:100000000C9450070C9475070C9475070C947507A5
:100010000C9475070C9475070C9475070C94750770
:100020000C9475070C9475070C94234B0C943F4B60
:100030000C9475070C9475070C9475070C94750750
:100040000C9475070C9475070C9475070C94750740
:100050000C9475070C9475070C9475070C94750730
:100060000C9475070C9475070C9475070C94750720
:100070000C9475070C9475070C9475070C94750710
:100080000C9475070C9475070C9475070C94750700
:100090000C9475070C9475070C9475070C94324DED
:1000A0000C946F4D0C94AC4D0C94E94D0C94750769
:1000B0000C9475070C9475070C9475070C947507D0
:1000C0000C9475070C9475070C9475070C947507C0
:1000D0000C9475070C9475070C9475070C947507B0
:1000E0000C9475070C9475070C9475070C947507A0
:1000F0000C9475070C9475070C9475070C94750790
:100100000C9475070C9475070C9475070C9475077F
:100110000C9475070C9475070C9475070C943E4C61
:100120000C947B4C0C94B84C0C94F54C0C947507C7
:100130000C9475070C9475070C9475070C9475074F
:100140000C9475070C9475070C9475070C9475073F
:100150000C9475070C9475070C9475070C9475072F
:100160000C9475070C9475070C9475070C9475071F
:100170000C9475070C9475070C9475070C9475070F
:100180000C9475070C9475070C9475070C947507FF
:100190000C9475070C9475070C9475070C947507EF
:1001A0000C9475070C9475070C9475070C947507DF
:1001B0000C9475070C9475070C9475070C947507CF
:1001C0000C9475070C9475070C9475070C947507BF
:1001D0000C9475070C9475070C9475070C947507AF
:1001E0000C9475070C9475070C9475070C9475079F
:1001F0000C9475073C696E70757420747970653D58
:10020000227375626D697422207374796C653D2266
:100210006865696768743A203530707822206E61AD
:100220006D653D22746F67676C65222076616C7521
:10023000653D224C454434223E266E627370266E24
:100240006273703C696E70757420747970653D22BC
:100250007375626D697422207374796C653D2268D0
:1002600065696768743A203530707822206E616D58
:10027000653D22746F67676C65222076616C7565D9
:100280003D224C454435223E266E627370266E62D6
:1002900073703C696E70757420747970653D22735B
:1002A00075626D697422207374796C653D2268658E
:1002B000696768743A203530707822206E616D6508
:1002C0003D22746F67676C65222076616C75653DB1
:1002D000224C454436223E266E627370266E62734F
:1002E000703C696E70757420747970653D22737509
:1002F000626D697422207374796C653D226865694A
:100300006768743A203530707822206E616D653DE3
:1003100022746F67676C65222076616C75653D227B
:100320004C454437223E266E627370266E627370AF
:100330003C2F6669656C647365743E3C2F666F7212
:100340006D3E3C2F74643E3C74643E266E62737056
:100350003B3C2F74643E3C2F74723E3C2F746162B0
:100360006C653E3C2F74643E3C7464207769647411
:10037000683D22323025223E3C2F74643E3C2F746F
:10038000723E3C2F7461626C653E3C2F626F6479F3
:100390003E3C2F68746D6C3E003C74723E3C74644D
:1003A0003E3C666F726D206D6574686F643D2267B8
:1003B00065742220616374696F6E3D22223E3C7039
:1003C0003E3C696E70757420747970653D2273755A
:1003D000626D697422207374796C653D2268656969
:1003E0006768743A2035307078222076616C7565C4
:1003F0003D2252656672657368223E3C2F703E3C1A
:100400002F666F726D3E3C2F74643E3C2F74723EBB
:100410003C2F7461626C653E3C62723E3C666F725A
:100420006D2069643D22666F726D226E616D653D5F
:1004300022666F726D22206D6574686F643D22675D
:1004400065742220616374696F6E3D22696E646514
:10045000782E68746D6C223E3C6669656C647365C9
:10046000743E3C6C6567656E643E4C454420636F2A
:100470006E74726F6C3C2F6C6567656E643E3C6990
:100480006E70757420747970653D227375626D6944
:100490007422207374796C653D226865696768749D
:1004A0003A203530707822206E616D653D22746F80
:1004B00067676C65222076616C75653D224C45440A
:1004C00030223E266E627370266E6273703C696ED7
:1004D00070757420747970653D227375626D6974EE
:1004E00022207374796C653D226865696768743A87
:1004F000203530707822206E616D653D22746F6703
:10050000676C65222076616C75653D224C454431EF
:10051000223E266E627370266E6273703C696E7046
:10052000757420747970653D227375626D697422EB
:10053000207374796C653D226865696768743A2038
:100540003530707822206E616D653D22746F67676B
:100550006C65222076616C75653D224C45443222E3
:100560003E266E627370266E6273703C696E7075A3
:100570007420747970653D227375626D69742220F0
:100580007374796C653D226865696768743A2035D3
:1005900030707822206E616D653D22746F67676CE4
:1005A00065222076616C75653D224C454433223EC0
:1005B000266E627370266E6273703C703E003C2F34
:1005C00074643E3C74643E3C623E3C2F623E3C2F71
:1005D00074643E3C2F74723E003C74723E3C746402
:1005E0003E4D414320416464726573733A20003C80
:1005F0002F74643E3C74643E3C623E3C2F623E3C41
:100600002F74643E3C2F74723E003C74723E3C7406
:10061000643E495020416464726573733A20004817
:100620005454502F312E3020323030204F4B0A534B
:1006300065727665723A20776C705F687474706466
:100640000A436F6E74656E742D747970653A207408
:100650006578742F68746D6C0A0A3C21444F4354CA
:100660005950452048544D4C205055424C49432048
:10067000222D2F2F5733432F2F4454442048544DBD
:100680004C20342E3031205472616E736974696F5E
:100690006E616C2F2F454E222022687474703A2FA1
:1006A0002F7777772E77332E6F72672F54522F68FC
:1006B000746D6C342F6C6F6F73652E647464223E9E
:1006C0003C68746D6C3E3C686561643E3C74697462
:1006D0006C653E6F574C207069636F2048545450CE
:1006E00020576562207365727665723C2F74697459
:1006F0006C653E3C2F686561643E3C626F647920A6
:100700007374796C653D666F6E742D66616D696C8E
:10071000793A617269616C3E3C7461626C653E3C21
:1007200074723E3C74642077696474683D22313091
:1007300030223E3C2F74643E3C74643E3C746162E3
:100740006C653E3C74722076616C69676E3D227404
:100750006F70223E3C74643E3C696D672073726327
:100760003D226C6F676F2E6769662220616C743D55
:10077000226C6F676F227469746C653D226C6F67C1
:100780006F223E3C2F74643E3C2F74723E3C747268
:100790003E3C74642077696474683D2235303022B1
:1007A0003E3C68323E576562205365727665722022
:1007B00072756E6E696E67206F6E206F574C207079
:1007C00069636F3C2F68323E3C703E546865207709
:1007D0006562207061676520697320736572766554
:1007E0006420627920776C705F687474706420751F
:1007F00073696E672074686520535042383030202A
:10080000574C414E206D6F64756C6520616E64209D
:10081000746865206F574C2D7069636F26636F7025
:10082000793B20536F667477617265204150493B74
:10083000206120756E697175652057692D466920A4
:10084000736F6C7574696F6E2066726F6D203C6299
:100850003E4826616D703B4420576972656C657334
:10086000732041423C2F623E2E3C2F703E3C68720A
:100870003E3C7461626C653E0047494638396145CB
:10088000017B00A10000FFFFFF006699000000FF50
:10089000FFFF21FE114372656174656420776974FE
:1008A000682047494D50002C0000000045017B00A6
:1008B0000002FE848FA9CBED0FA39CB4DA8BB3DECC
:1008C000BCFB0F86E24896E689A6EACAB6EE0BC7DD
:1008D000F24CD7F68DE7FACEF7FE0F0C0A87C4A2CA
:1008E000F1884C2A97CCA6F3098D4AA7D4AAF58A99
:1008F0006505B6DCAEF70B0E8BC76471F60C2DAB3D
:10090000D7EC36190D3FBAE7F4FA3B8EFFD9F77CE6
:100910007BFE9FD32738C80668384398A81876D836
:10092000D8B2081919E048792279A958A92982D999
:1009300029B809DAE139CA176A8A419A4A77CA3A64
:10094000A1FAEAD62AEB005BAB368BAB60BB6B96A9
:10095000EB0BC01BECF5EB2B6CBC458C7B6C9C3C17
:10096000BB2CDC2CFB1C1CDD3ACD5BCD7ABD9B7D0A
:10097000BA6DDB6DFA5D1B1E3A0E5B0E7AFE9ABEF7
:10098000B9AEDAAEF99E1A5F394F5A4F793F9AEFF6
:10099000B8EFD9AFD1BF4E010F0DC454D0D0C14B69
:1009A00009012D94D4F0CFC34811F34C845411CFD6
:1009B0001DFE5D601A8CF158A6421B04024A9A146F
:1009C000B0E0E4C9942A511E68290366B88D09185D
:1009D00031B0F980A6AB5B2465F6F4F9122800A1CA
:1009E0002D8836D3790027C761123E5EE01954A5E1
:1009F000829625A70A35BA022B31A40694D664DA6A
:100A0000B4D7539D5413503569F6AAD4185A7F7140
:100A100005D6F126D8B07151398DBAF26759BD6843
:100A2000F9BA84D1B6D8DDAF5F4072913B6969E114
:100A30000C64D59E4DBB7647E05C6FBD22987B1958
:100A40009962CC490FD3128BB7AF81B355FDFA9899
:100A5000AC6C70E6C50B58AFDECCB96B6CD996F7B1
:100A60000E255DFA76E4D07F47FBCCCB127883C9A4
:100A7000A879E77EF0B847E5BAB05B2726CC7C754D
:100A800017C4D17503C79DDB366FC82B8962EFCDC4
:100A9000FD7878ED56B10FFFCEE3ADC8D9CE414B0E
:100AA000F7DCDEB5EFC8E8E70BB72FBE2CD0EFF7C9
:100AB000FEF183F78F5B70FC95376020AAD9C5DE05
:100AC0007BD5D1361D75B1FD661E8004E6572080AA
:100AD000018E2760851692365E8438A847C182D081
:100AE000B9D7197B245A87964C2AEEB69D5FDAF166
:100AF000C7228AFFC1789F63C2D9289A0D20EE04CD
:100B00005F4E21C5D7E3880D7628A37F32FE57A418
:100B10008B10C6481E8EE21D69DA04C5DDB0235D68
:100B2000CF41009F8822C2B5A07E6BC1449E914AEE
:100B3000228995931866D85B98E7C5E84395110418
:100B400089E0950ACA39A7661DDAA6618BC62179A4
:100B5000248C51EE59619E63F6F7E1810C0EB914B5
:100B600007B36D79629F377A78E69E0CD0B81F8BF9
:100B700094EE46239A1CEAB09C7C9921C6239D875B
:100B8000DA091B9C1BE658DF84E0A9792AA44E668B
:100B90003A289BB016DAA8659D01F926A2733A3867
:100BA0005BAA8EE6F8A784935E8AAAA5C43EF9FEE6
:100BB0002BA1C9024B43A7268AEAA990BC1A262278
:100BC000A4AD0E5BA356AC3A60A6079B22F76D0D51
:100BD000CEEAFA2990A46E469D8FB69EAA2A9B491A
:100BE0001AB7A6B2DC1AEB6E0653BEABA3A15C3EED
:100BF0006B188F1BE8FB6BBBCCEA29ACA6AB762B42
:100C0000A98B146CABAA81B5322A2A63115BB9E5B2
:100C10008583C64B61BDCB7AC724B109EB991CC152
:100C2000E2EABB2E971E984A71C521DFC927BE5044
:100C3000622C28C794B21CAEC7B4AE5B32B916E8BA
:100C40009CAB7AE18E093391F3FAD9B0C02BB7FA95
:100C5000AAC554920C31CAEDBD37D68FD8BAFB73F2
:100C6000B02F83AB74A4460F0C28D5828EFC70B4D1
:100C7000A34EBC6F8309960AF0D59A0E0D2CC3457E
:100C8000B38DACD0111C0D73CBF95E94484671E066
:100C90009D89DE68F09DB7DF67004E88E08313FE14
:100CA00089E158209EB8E25630DE87E35740AD5EBA
:100CB0008AE45550BE87E597635E87E65470DEB9D7
:100CC000E75280BE8AE851903E87E9A7A33E92EAA8
:100CD0004FB0DEBAEB4DC05E88ECB3D30E95ED4A53
:100CE000E09EBBEE48F02EB5EFBF039FB6F040107C
:100CF0005FBCF16D225FB2F27A30BFA5F3CB437FC8
:100D0000B6F43B505FBDF59C62EFB4F6CA714FB6C6
:100D1000F7D7832F3E11E4976F3EF6E8A74FFDFA11
:100D2000EC23EF7E11CCC72F3FF1F41B01FCFDC378
:100D3000B3AE7F12A4F77F3BC601F0730719A00181
:100D40000F88C0042A70810C6CA0031F08C1084AD8
:100D5000708214ACA0052F8841CD1500003B48548B
:100D600054502F312E3020323030204F4B0A5365F3
:100D7000727665723A20776C705F68747470640A7A
:100D8000436F6E74656E742D747970653A20696D69
:100D90006167652F6769660A0A00485454502F310D
:100DA0002E30203430342046696C65206E6F7420FC
:100DB000666F756E640A5365727665723A20776C59
:100DC000705F68747470640A436F6E74656E742D1E
:100DD000747970653A20746578742F68746D6C0A44
:100DE0000A3C68746D6C3E3C686561643E3C7469A5
:100DF000746C653E6F574C207069636F2048545483
:100E00005020576562207365727665723C2F746955
:100E1000746C653E3C2F686561643E3C626F64792A
:100E20003E3C68323E343034202D205061676520CE
:100E30006E6F7420666F756E643C2F68323E3C7036
:100E40003E536F7272792C207468652070616765FB
:100E500020796F7520617265207265717565737494
:100E6000696E6720776173206E6F7420666F756E90
:100E700064206F6E20746869732073657276657282
:100E80002E3C2F703E3C2F626F64793E3C2F68747D
:100E90006D6C3E006364696E6F70737578585B00AB
:100EA00011241FBECFEFDFE3DEBFCDBF00E00CBFDC
:100EB00018BE19BE1ABE1BBE12E3A0E0B0E2EEE2FD
:100EC000FDEB00E00BBF02C007900D92AE3FB107F3
:100ED000D9F713E3AEEFB2E301C01D92A93EB1070B
:100EE000E1F70E94BF450C94955E0C9400009BB7FF
:100EF0008BBFFB018091CA014093CA017DE97093C9
:100F00003400E8958093CA019BBF08952091CF01DA
:100F100027FDFCCF9BB78BBFFB018091CA0123E269
:100F20002093CA010A01E89511248093CA019BBF4E
:100F30000895E0910033F091013308C020813181A0
:100F40002817390729F00380F481E02D3097B1F795
:100F5000CF0108959C01AB01A091FE32B091FF3208
:100F6000ED91FC91119716968D919C911797B9016F
:100F7000199508959C01AB01A091FE32B091FF320A
:100F80001296ED91FC91139716968D919C9117975F
:100F9000B90119950895A091FE32B091FF321496CF
:100FA000ED91FC911597309739F016968D919C91A3
:100FB000179761E070E019950895A091FE32B09105
:100FC000FF321496ED91FC911597309739F01696F3
:100FD0008D919C91179760E070E019950895E091CC
:100FE000FE32F091FF32808983FD0CC008951C967B
:100FF000ED91FC911D97309749F01E968D919C9133
:101000001F971995A091FE32B091FF3251968C91A5
:101010005197882361F351961C9251970895AF928E
:10102000BF92CF92DF92EF92FF920F931F93CF93D5
:10103000DF93EC015B016A01790188E090E0C80E62
:10104000D91EE80EF91EC6010E94341488839983C4
:101050001A82AB821C821D821E820115110579F055
:101060000E94CB07CE01B6010E94BA070E94EF078B
:10107000CE01B7010E94AA070E94DD070AC0CE0177
:10108000B6010E94BA070E94EF07CE01B7010E9485
:10109000AA07888199810E943814888399838C815A
:1010A0009D810E943814282F392F2C833D838881FD
:1010B00099818E159F0541F48A81813029F48B81B5
:1010C00090E08A159B0511F020EF3FEFC901DF91F9
:1010D000CF911F910F91FF90EF90DF90CF90BF9035
:1010E000AF900895CF92DF92EF92FF920F931F93EC
:1010F000CF93DF937C016B01EA018901A091FE325D
:10110000B091FF321896ED91FC911997309739F014
:101110001A968D919C911B9761E070E01995C7011B
:10112000B601AE01980101E010E00E940F08E82E20
:10113000092FA091FE32B091FF321896ED91FC91EB
:101140001997309739F01A968D919C911B9760E012
:1011500070E019958E2D902FDF91CF911F910F91F7
:10116000FF90EF90DF90CF9008954F925F926F9233
:101170007F928F929F92AF92BF92CF92DF92EF9227
:10118000FF920F931F93CF93DF935C014B013A01C2
:101190002901C091FE32D091FF32CE014E9669E016
:1011A00070E040E050E028E130E00E947208A114B5
:1011B000B10449F02EA13FA148A559A5F50120830E
:1011C0003183428353838114910449F02AA53BA5BE
:1011D0004CA55DA5F40120833183428353836114C0
:1011E000710449F02EA53FA548A959A9F301208310
:1011F0003183428353834114510449F02AA93BA906
:101200004CA95DA9F20120833183428353830115E8
:10121000110539F02BAD332727FD3095F8012083D8
:101220003183C114D10439F02AAD332727FD30951D
:10123000F60120833183E114F10449F02EA93FA97E
:1012400048AD59ADF7012083318342835383DF9149
:10125000CF911F910F91FF90EF90DF90CF90BF90B3
:10126000AF909F908F907F906F905F904F90089578
:10127000DF92EF92FF920F931F93FC01D02EA0916B
:10128000FE32B091FF32009759F0E080F180028188
:1012900013819696ED92FD920D931C93999706C03B
:1012A00096961D921D921D921C929997611571053B
:1012B00061F0FB0160817181828193819A966D93C7
:1012C0007D938D939C939D9706C09A961D921D9237
:1012D0001D921C929D974115510561F0FA014081C4
:1012E0005181628173819E964D935D936D937C9342
:1012F000D19706C09E961D921D921D921C92D19769
:101300002115310561F0F90120813181428153813C
:10131000D2962D933D934D935C93D59706C0D2966C
:101320001D921D921D921C92D597D696DC92D6974F
:10133000CD014E9668E070E044E150E020E030E0FE
:101340000E9472081F910F91FF90EF90DF90089517
:10135000CF92DF92EF92FF920F931F93CF93DF9381
:101360006C01EB010091FE321091FF32209709F4DD
:1013700056C0CB0183709070009731F09B012370B1
:10138000822F24E0281B01C020E08EE1E82EF12C02
:10139000E00EF11EF80124A3CE010896820F911DE4
:1013A0000E943414F801868F978F82E080A38BE12E
:1013B00081A312A213A2C70168E070E00E94BA07DD
:1013C000F80184A1C80FD11DC601BE010E94BA0751
:1013D0008C179D0739F50E94EF07C70168E070E0A0
:1013E0000E94AA07F801868D978D0E943814F80193
:1013F000868F978F82A193A10E943814282F392FAE
:10140000F80122A333A3868D978D8830910551F47E
:1014100080A1833039F481A18B3121F405C020E013
:1014200030E002C020EF3FEFC901DF91CF911F9163
:101430000F91FF90EF90DF90CF9008958F929F9241
:10144000AF92BF92CF92DF92EF92FF920F931F93D2
:10145000DF93CF930F92CDB7DEB74C016B015A01EA
:10146000790187E789838DE293E38093FE3290933D
:10147000FF3260E070E04EEA50E00E947816E091A2
:10148000FE32F091FF32C082D182A282B382E48226
:10149000F5820683178381E08816910421F4808900
:1014A0008860808B1DC00E94CB078E010F5F1F4F8D
:1014B000C80161E070E00E94BA07C80161E070E015
:1014C0000E94AA07E02E012F06C08E2D902F61E00A
:1014D00070E00E94AA0789818E32B9F30E94DD076D
:1014E00080E090E00F90CF91DF911F910F91FF90DE
:1014F000EF90DF90CF90BF90AF909F908F90089526
:101500000F931F93CF93DF938C01C091FE32D09144
:10151000FF32CE014E9663E270E040E050E024E0FE
:1015200030E00E9472089C0197FD05C08EA1F80171
:10153000808320E030E0C901DF91CF911F910F91AE
:101540000895EF92FF920F931F93CF93DF93EC01D7
:101550008B01E091FE32F091FF32009719F081E0AB
:1015600086A301C016A2CF014E966FE170E044E061
:1015700050E020E030E00E9472087C01E091FE32F1
:10158000F091FF32C087D18702871387C80160E0DE
:1015900070E0FE011995C701DF91CF911F910F9166
:1015A000FF90EF900895E091FE32F091FF32848732
:1015B0009587668777870895E091FE32F091FF3234
:1015C00081E0818B08950F931F93DF93CF930F9248
:1015D000CDB7DEB70091FE321091FF3249830E94F1
:1015E0003C14F80166A377A380A791A7498142A77D
:1015F0008091FE329091FF324E9660E070E048E0BC
:1016000050E024E030E00E9472080F90CF91DF910B
:101610001F910F910895AF92BF92CF92DF92EF92F8
:10162000FF920F931F93DF93CF930F920F92CDB73B
:10163000DEB787E78983A091FE32B091FF3218961A
:10164000ED91FC911997309739F01A968D919C91F4
:101650001B9761E070E019958091FE329091FF3206
:101660004E9668E170E040E050E020E030E00E94FB
:1016700072086C0197FD2FC0E091FE32F091FF32AD
:10168000808983FD28C00E94CB078E010F5F1F4F0A
:10169000C80161E070E00E94BA0792E0E92EF12CE7
:1016A000EC0EFD1EC70161E070E00E94AA07580120
:1016B0001E2D0F2D0BC0C50161E070E00E94BA071E
:1016C000812F902F61E070E00E94AA078A818737FE
:1016D00091F70E94DD07A091FE32B091FF3218967B
:1016E000ED91FC911997309739F01A968D919C9154
:1016F0001B9760E070E01995C6010F900F90CF9195
:10170000DF911F910F91FF90EF90DF90CF90BF90EE
:10171000AF9008956F927F928F929F92AF92BF92F7
:10172000CF92DF92EF92FF920F931F93CF93DF93AD
:101730003C016B015A014901C091FE32D091FF3248
:10174000CE014E9662E070E040E050E024E230E0EE
:101750000E9472087C0197FD3AC08EA190E0A0E043
:10176000B0E0DC01992788272FA130E040E050E06D
:10177000542F432F322F2227822B932BA42BB52BB0
:1017800028A530E040E050E0822B932BA42BB52B12
:10179000F30180839183A283B383C114D10451F0F8
:1017A000A114B10439F0BE01665D7F4FC601A501E9
:1017B0000E9487168114910451F00115110539F02A
:1017C000BE01665C7F4FC401A8010E948716C70155
:1017D000DF91CF911F910F91FF90EF90DF90CF900D
:1017E000BF90AF909F908F907F906F900895E09101
:1017F000FE32F091FF32828B938B648B758B089550
:1018000086EF9FEF089586EF9FEF0895AF92BF9206
:10181000CF92DF92EF92FF920F931F93CF93DF93BC
:101820006C017B015A010091FE321091FF32E801F8
:10183000A696CE0160E070E048E650E00E9478167F
:10184000C114D10431F0CE01B60141E250E00E9452
:101850007516E114F10461F081E0A816B10449F1B4
:10186000C7010E947E1608978833910510F113C0B6
:10187000F801E657FF4FA0828091FE329091FF322F
:101880004E9663E070E048E650E020E030E00E94D1
:1018900072089C0102C02EEF3FEFC901DF91CF918A
:1018A0001F910F91FF90EF90DF90CF90BF90AF907E
:1018B0000895C801865B9F4FB7014FE350E00E9437
:1018C0008716D6CF8091FE329091FF324E9664E01B
:1018D00070E040E050E020E030E00E94720808959F
:1018E0000F931F9300E010E00E9438091F910F91A1
:1018F0000895CF92DF92EF92FF920F931F9300E033
:1019000010E0EE24FF24CC24DD240E94B5081F91B2
:101910000F91FF90EF90DF90CF9008950F931F935A
:101920008C0180E090E060E070E040E050E020E07A
:1019300030E00E9438091F910F910895CF92DF92F5
:10194000EF92FF920F931F938C0180E090E060E094
:1019500070E040E050E020E030E0EE24FF24CC24B2
:10196000DD240E94B5081F910F91FF90EF90DF904A
:10197000CF900895E091FE32F091FF3286A3CF011F
:101980004E9669E170E044E050E020E030E00E94D3
:1019900072080895E091FE32F091FF32868B978BAA
:1019A000608F718F08950F931F93CF93DF938C01F6
:1019B000C091FE32D091FF32CE014E9666E070E0CB
:1019C00040E050E024E330E00E9472080115110568
:1019D00041F0BE016A5D7F4FC80146E050E00E94C1
:1019E000751680E090E0DF91CF911F910F910895DF
:1019F000EF92FF920F931F93CF93DF93EC0100912F
:101A0000FE321091FF32C8014E9666E070E040E071
:101A100050E024E330E00E9472087C01209741F1FD
:101A2000B801645D7F4FCE01819646E050E00E9490
:101A30007516B8016E5C7F4FCE0141E250E00E9406
:101A40007516F801EA5AFF4F808191810E9438147F
:101A50008FA398A7F801E85AFF4F808191810E94D7
:101A6000381489A79AA71DA61BA61CA61EA61FA6EA
:101A7000C701DF91CF911F910F91FF90EF900895D3
:101A8000AF92BF92CF92DF92FF920F931F93DF939B
:101A9000CF930F92CDB7DEB7F82E0091FE321091A2
:101AA000FF328FE090E069830E944D165C016981EE
:101AB000009779F1F801F6A267A38091FE32909128
:101AC000FF324E966BE070E044E050E020E030E002
:101AD0000E9472088C0197FF04C0C5010E94721613
:101AE0001AC0F5018083918313821482E091003340
:101AF000F0910133309731F4A0920033B09201336A
:101B00000AC0FC01838194810097D9F7A382B48233
:101B100002C00DEF1FEFC8010F90CF91DF911F9111
:101B20000F91FF90DF90CF90BF90AF9008950F93EB
:101B30001F93CF93DF93EB018A010E949907FC0169
:101B4000009739F0C783D0870387148720E030E0FF
:101B500002C02EEF3FEFC901DF91CF911F910F918E
:101B600008950F931F93CF93DF93EB018A010E9497
:101B70009907FC01009739F0C187D287058716873E
:101B800020E030E002C02EEF3FEFC901DF91CF919E
:101B90001F910F910895EF92FF920F931F93CF9390
:101BA000DF93EB017A010091FE321091FF320E9427
:101BB0003414F80182A793A788819981AA81BB81F7
:101BC00086A397A3A0A7B1A7C7010E943414F80168
:101BD00084A795A78091FE329091FF324E966CE0DB
:101BE00070E048E050E020E030E00E947208DF91B1
:101BF000CF911F910F91FF90EF900895BF92CF92D8
:101C0000DF92EF92FF920F931F93CF93DF93EC013C
:101C1000B62E6A0179010091FE321091FF320E94C6
:101C20009907FC010097D9F0C582D682E386F48635
:101C30001282CE010E943414F80186A397A3B0A6A5
:101C40008091FE329091FF324E966DE070E044E05C
:101C500050E020E030E00E9472089C0102C02EEFAC
:101C60003FEFC901DF91CF911F910F91FF90EF904E
:101C7000DF90CF90BF900895CF92DF92EF92FF92C6
:101C80000F931F93CF93DF93EC016B017A010091C7
:101C9000FE321091FF320E949907009739F1FC0142
:101CA0001282CE010E943414F80182A793A7F60194
:101CB00080819181A281B381F80186A397A3A0A717
:101CC000B1A7C7010E943414F80184A795A7809199
:101CD000FE329091FF324E966EE070E048E050E0A8
:101CE00020E030E00E9472089C0102C02EEF3FEF1E
:101CF000C901DF91CF911F910F91FF90EF90DF907D
:101D0000CF900895CF92DF92EF92FF920F931F939F
:101D1000CF93DF937C010091FE321091FF328FE070
:101D200090E00E944D16C82EE6016E01D92EE60104
:101D3000209771F1C7010E943414F80186A397A37C
:101D40008091FE329091FF324E9664E170E044E063
:101D500050E020E030E00E9472088C0197FF04C040
:101D6000C6010E94721616C0888399831B821C824A
:101D70008A8181608A83E0910033F091013301C050
:101D8000FC01838194810097D9F7C383D48302C077
:101D90000DEF1FEFC801DF91CF911F910F91FF90C1
:101DA000EF90DF90CF9008950F931F93CF93DF9321
:101DB000EC010091FE321091FF320E943414D801E0
:101DC00096968D939C9397978091FE329091FF32D7
:101DD0004E966FE070E044E050E020E030E00E947A
:101DE00072088091003390910133FC01A0E0B0E0D3
:101DF0002DC0208131812C173D0719F5228122FD4C
:101E000020C0C091FE32D091FF32388932FF03C02A
:101E1000246022831DC0109751F4DC0113968D912C
:101E20009C911497809300339093013306C0838173
:101E3000948113968D939C931497CF010E947216F0
:101E400007C0DF0133812481E32FF22F309789F619
:101E500080E090E0DF91CF911F910F910895AF92B4
:101E6000BF92CF92DF92EF92FF920F931F93DF9377
:101E7000CF9300D0CDB7DEB75B017A010091FE327F
:101E80001091FF320E943414F80186A397A3C70172
:101E90000E943414F80180A791A7A091FE32B0915E
:101EA000FF321896ED91FC911997309739F01A96F8
:101EB0008D919C911B9761E070E019950E94CB0772
:101EC0008091FE329091FF324E9660E170E044E0E6
:101ED00050E020E030E000E010E00E940F088C01AC
:101EE00097FD43C0E816F906F4F1C090FE32D09099
:101EF000FF320E94EF07C6014E9668E070E00E9434
:101F0000AA077C01F601868D978D0E943814F60190
:101F1000868F978FF8E0EF16F10429F5F60120A1DE
:101F2000243009F521A12B31F1F424A1E8EFEE2EA4
:101F3000EFEFFE2EE21AF108E80EF91EE016F106A8
:101F400091F4C501B7010E94AA078C018E159F0567
:101F500051F4F60164A1662341F0CE01019670E0D0
:101F60000E94AA0702C000EF1FEF0E94DD07A091A8
:101F7000FE32B091FF321896ED91FC91199730978F
:101F800039F01A968D919C911B9760E070E019953D
:101F9000C8012396CDBFDEBFCF91DF911F910F9176
:101FA000FF90EF90DF90CF90BF90AF900895CF92C9
:101FB000DF92EF92FF920F931F93CF93DF936B010A
:101FC0007A01C091FE32D091FF320E9434148EA368
:101FD0009FA3C7010E94341488A799A7A091FE323D
:101FE000B091FF321896ED91FC911997309739F026
:101FF0001A968D919C911B9761E070E019950E9453
:10200000CB078091FE329091FF324E9661E170E0F5
:1020100044E050E020E030E000E010E00E940F08D3
:10202000EC0197FD0BC0E816F90634F0C601BE01BD
:102030000E94A809EC0102C0C0EFDFEF0E94DD079B
:10204000A091FE32B091FF321896ED91FC91199754
:10205000309739F01A968D919C911B9760E070E053
:102060001995CE01DF91CF911F910F91FF90EF90C5
:10207000DF90CF900895AF92BF92CF92DF92EF9210
:10208000FF920F931F93CF93DF935B016A01E901E6
:10209000E090FE32F090FF320E943414F70182A7E4
:1020A00093A7C6010E943414F70184A795A78881DD
:1020B0009981AA81BB8186A397A3A0A7B1A7C801D4
:1020C0000E943414F70186A797A7A091FE32B09121
:1020D000FF321896ED91FC911997309739F01A96C6
:1020E0008D919C911B9761E070E019950E94CB0740
:1020F0008091FE329091FF324E9662E170E04CE0AA
:1021000050E020E030E000E010E00E940F08EC0119
:1021100097FD0BC0C816D90634F0C501BE010E9458
:10212000A809EC0102C0C0EFDFEF0E94DD07A0911B
:10213000FE32B091FF321896ED91FC9119973097CD
:1021400039F01A968D919C911B9760E070E019957B
:10215000CE01DF91CF911F910F91FF90EF90DF9013
:10216000CF90BF90AF9008950F931F93CF93DF93BD
:102170008B01C091FE32D091FF320E9434148EA3A5
:102180009FA38091FE329091FF324E9665E170E000
:1021900044E050E024E030E00E947208BC0197FD6A
:1021A00009C02EA13FA148A559A5F801208331837C
:1021B00042835383CB01DF91CF911F910F910895FB
:1021C000CF92DF92EF92FF920F931F93CF93DF9303
:1021D000EC018B016A01E090FE32F090FF32009733
:1021E00059F10E947E168038910530F5E091FE325B
:1021F000F091FF32828D938D009709F5C701869685
:10220000BE010E9490168091FE329091FF324E9650
:102210006AE070E040E850E020E030E00E947208A0
:102220009C0197FD0EC0E091FE32F091FF32028FCB
:10223000138FC48ED58E05C02EEF3FEF02C022EF64
:102240003FEFC901DF91CF911F910F91FF90EF9068
:10225000DF90CF900895AF92BF92CF92DF92EF922E
:10226000FF920F931F93DF93CF93CDB7DEB72A97DB
:10227000CDBFDEBF8091FE329091FF32009709F40E
:10228000A9C14E9661E070E040E050E020E030E00F
:102290000E947208009709F49DC18091FE329091CE
:1022A000FF324E9665E070E040E050E020E030E024
:1022B0000E9472080097D1F4A091FE32B091FF32D3
:1022C0005296ED91FC915397309761F150968C9115
:1022D000509780FD27C0816050968C9350975496FC
:1022E0008D919C91559761E070E01BC097FF1AC0DB
:1022F000A091FE32B091FF325296ED91FC9153972E
:10230000309781F050968C91509780FF0BC08E7F54
:1023100050968C93509754968D919C91559760E070
:1023200070E01995A3E0AA2EB12CAC0EBD1EC5011C
:1023300060E070E040E050E020E030E000E010E0DD
:10234000F7E0EF2EF12CEC0EFD1E6E010894C11C7F
:10235000D11C0E94B5080097D1F4A091FE32B09133
:10236000FF325696ED91FC915797309769F1509650
:102370008C91509781FD28C0826050968C93509725
:1023800058968D919C915997B50119951DC097FF4D
:1023900042C0A091FE32B091FF325696ED91FC9171
:1023A00057973097C1F150968C91509781FF33C069
:1023B0008D7F50968C93509758968D919C915997FC
:1023C00060E070E0199527C0A091FE32B091FF3215
:1023D0005A96ED91FC915B973097E9F089819A814B
:1023E000009741F45C968D919C915D97BE01695F69
:1023F0007F4F0AC02FEF8F3F920769F45C968D9153
:102400009C915D9760E070E01995E091FE32F0914B
:10241000FF32128E138EE091FE32F091FF328089EE
:102420008460808B009100331091013393C0D801F8
:102430008D919C910E943414F70186A397A38091FB
:10244000FE329091FF324E9663E170E044E050E03E
:1024500024E030E00E947208AC0197FD22C0D70151
:1024600096968C9196978130D1F4F801928190FDE7
:1024700042C00780F085E02D3097E9F1892F816017
:102480008D7FD80112968C9312976D917C91119744
:102490001B968D919C911C9741E050E057C0843071
:1024A000B9F4F801828181FD25C00780F085E02D17
:1024B000309701F18E7F8260D80112968C9312972B
:1024C0006D917C9111971B968D919C911C973CC0AE
:1024D000833089F4D8011596ED91FC9116973097C9
:1024E00051F06D917C9111971B968D919C911C9749
:1024F00019952DC084E0141615067CF4D8011996A0
:10250000ED91FC911A97309741F06D917C91119764
:102510001D968D919C911E9719C08823C1F4F801D6
:10252000828180FF14C00184F285E02D309779F01C
:102530008E7FD80112968C9312976D917C91119792
:102540001D968D919C911E9740E050E01995F801E1
:1025500003811481E090FE32F090FF3201151105E5
:1025600009F065CFD70150968C9150978B7F50968C
:102570008C935097E0910033F091013300E010E02C
:1025800027C0828182FF1FC00115110569F4A09147
:102590000033B091013313968D919C9114978093E1
:1025A00000339093013307C083819481D80113963F
:1025B0008D939C931497A380E480CF010E947216A0
:1025C0009A2D8E2D03C08F0193818481E92FF82FDE
:1025D0003097B9F62A96CDBFDEBFCF91DF911F911C
:1025E0000F91FF90EF90DF90CF90BF90AF90089544
:1025F000E091FE32F091FF3286A3CF014E9666E164
:1026000070E044E050E020E030E00E94720808955D
:102610000F931F93CF93DF938C01C091FE32D09123
:10262000FF32CE014E966AE170E040E050E024E0D7
:1026300030E00E9472089C0197FD03C08EA1F80152
:102640008083C901DF91CF911F910F910895E0918F
:10265000FE32F091FF3286A3CF014E9667E170E023
:1026600044E050E020E030E00E9472080895E091DC
:10267000FE32F091FF3221E0009709F420E026A31A
:10268000CF014E966EE170E044E050E020E030E093
:102690000E94720808958F929F92AF92BF92CF923C
:1026A000DF92EF92FF920F931F93CF93DF93F82E59
:1026B0004A015B01C901B801C091FE32D091FF32DD
:1026C0000E943C146EA37FA388A799A7C501B401FB
:1026D0000E943C146AA77BA78CA79DA7C6010E94F5
:1026E00034148EA79FA7F8AAE9AA8091FE32909190
:1026F000FF324E966DE170E04FE050E020E030E0B8
:102700000E947208DF91CF911F910F91FF90EF907F
:10271000DF90CF90BF90AF909F908F900895BF9221
:10272000CF92DF92EF92FF920F931F93CF93DF939D
:10273000B82E7B016A018901C091FE32D091FF322F
:10274000CE01869660E070E048E850E00E9478167E
:10275000E114F10449F0F70180819181A281B381F4
:102760008EA39FA3A8A7B9A7C6010E9434148AA765
:102770009BA7BCA60115110579F0C8010E947E1621
:102780008F379105C0F4C8010E947E16AC01CE01BE
:102790008E96B8010E9475168091FE329091FF329C
:1027A0004E966CE170E048E850E020E030E00E9496
:1027B00072089C0102C02EEF3FEFC901DF91CF915B
:1027C0001F910F91FF90EF90DF90CF90BF900895F1
:1027D000E091FE32F091FF3221E0009709F420E011
:1027E00026A3CF014E9660E270E044E050E020E086
:1027F00030E00E9472080895CF93DF93C091FE32BB
:10280000D091FF320E943C146EA37FA388A799A7A2
:102810008091FE329091FF324E9661E270E044E08A
:1028200050E020E030E00E947208DF91CF910895DF
:10283000CF93DF93C091FE32D091FF320E943C14BF
:102840006EA37FA388A799A78091FE329091FF3253
:102850004E9662E270E044E050E020E030E00E94FA
:102860007208DF91CF910895382F292FC90108955B
:10287000382F292FC9010895AF92BF92CF92DF92CE
:10288000EF92FF920F931F93292F33274427552749
:10289000162F0027FF24EE242E293F29402B512BF1
:1028A000EE24F62E072F182FA12CB12CFFEFCF2EE0
:1028B000D12CEA20FB200C211D212E293F29402B61
:1028C000512B672F782F892F992760708070907017
:1028D000262B372B482B592BB901CA011F910F9179
:1028E000FF90EF90DF90CF90BF90AF9008950E943F
:1028F0003C1408952F923F924F925F926F927F9275
:102900008F929F92AF92BF92CF92DF92EF92FF92FF
:102910000F931F93DF93CF93CDB7DEB76097CDBFF3
:10292000DEBFDC011B010C91112707FD10958DE026
:10293000482E512C4C0E5D1E5E010894A11CB11C4A
:10294000802F80538A3008F028C100331105A1F48C
:1029500011960C91112707FD10950837110519F0F4
:102960000835110569F411960C91112707FD109592
:10297000F0E1CF2ED12C07C0EAE0CE2ED12C03C03F
:1029800078E0C72ED12C7D010894E11CF11C60E099
:1029900070E0CB013601882477FC8094982CF701F5
:1029A0003197202F302F30533A30A0F4A4019301F7
:1029B0000E9453539B01AC0100531040B80188277B
:1029C00077FD8095982F620F731F841F951FD70185
:1029D0000C912BC0B0E1CB16D10471F5A02FA156FC
:1029E000A63020F0302F3154363030F59B01AC0149
:1029F00064E0220F331F441F551F6A95D1F7065F0D
:102A00001F4FAA3118F481E690E002C081E490E003
:102A1000081B190BB801882777FD8095982F622B2A
:102A2000732B842B952BF7010081112707FD10953F
:102A30000894E11CF11CB3CF0E32110589F4A414E3
:102A4000B50409F4AAC0D5016D937D938D939D9330
:102A50005D01DF0111960181112707FD109570CFEF
:102A600001151105C1F0203208F497C007FD95C08B
:102A70000032110581F00C30110569F00A301105A2
:102A800051F00D30110539F00930110521F00B30EE
:102A9000110509F082C09E012F5F3F4FA21AB30AB1
:102AA000B594A794B594A7940894A11CB11CB2E066
:102AB000AB16B10499F0E3E0AE16B1042CF4A11406
:102AC000B10409F46AC05EC0F3E0AF16B104C1F00E
:102AD00024E0A216B10409F055C02BC0603030E0EC
:102AE000730730E0830731E0930708F056C029816F
:102AF0003A814B815C81522F4427332722273EC0E5
:102B00006030A0E07A07A1E08A07A0E09A0708F009
:102B100044C02D813E814F815885A901332722274A
:102B2000E980FA800B811C811E2D0027FF24EE24F2
:102B300021C06F3F71058105910509F070F52D8168
:102B40003E814F815885A90133272227E980FA80E9
:102B50000B811C811E2D0027FF24EE242E293F29E6
:102B6000402B512BE984FA840B851C85102F0F2DE7
:102B7000FE2CEE242E293F29402B512B622B732B48
:102B8000842B952B2114310459F00E943C14F1013F
:102B9000608371838283938303C020E030E002C0AE
:102BA00021E030E0C9016096CDBFDEBFCF91DF915B
:102BB0001F910F91FF90EF90DF90CF90BF90AF905B
:102BC0009F908F907F906F905F904F903F902F904D
:102BD0000895AF92BF92DF92EF92FF920F931F93EF
:102BE000DF93CF93CDB7DEB72797CDBFDEBFFC0114
:102BF00080819181A281B3818C839D83AE83BF83C9
:102C0000DE011496AD014C5F5F4F32E0A32E33E33B
:102C1000B32E2AE0D22E9E012F5F3F4F9EE2E92E77
:102C20008C91FF246D2D0E94725389010F0D111D8F
:102C3000905DF8019083F3948823A1F76F2D1D9286
:102C4000C50109C0FA9489010F0D111DF8017081A9
:102C5000FC017193CF01FF20A9F7C501860F911DDB
:102C6000FC01E1925F01A417B507D1F6FC011082C7
:102C700082E093E32796CDBFDEBFCF91DF911F9116
:102C80000F91FF90EF90DF90BF90AF90089580E09C
:102C900090E008950E94E2530895EF92FF920F93FF
:102CA0001F93DF93CF930F920F92CDB7DEB7AC0196
:102CB00049835A830E94E2538C0149815A810097CB
:102CC00021F060E070E00E94A257C8010F900F90C1
:102CD000CF91DF911F910F91FF90EF9008950E9487
:102CE000155508950E947C5408950E9487570895B1
:102CF0000E94A25708950E9490570895FC010190E8
:102D00000020E9F73197E81BF90BCF0108950E94E5
:102D1000E55708950E94D75708950E94C757089510
:102D20000E94D05708950E9453570895CF92DF9282
:102D3000EF92FF920F931F93CF93DF937C018B0150
:102D4000CB0101960E94E253C82EE6016E01D92EF6
:102D5000E601209749F0C601B701A8010E94E55796
:102D6000F601E00FF11F1082CE01DF91CF911F918C
:102D70000F91FF90EF90DF90CF9008950E947A57C7
:102D800008950E94EE5508950E94BC5708950E9430
:102D9000F45708950E94A95708950E94FF57089577
:102DA000DF93CF93CDB7DEB7FE013C968E819F8136
:102DB000688579854A855B859F010E947658CF9109
:102DC000DF9108950E9476580895AF92BF92CF92F6
:102DD000DF92EF92FF920F931F93DF93CF93CDB7C4
:102DE000DEB78E01025F1F4FF801A190B1908F01F5
:102DF00080EA90E00E94E253D82EC92EE82EF92EE8
:102E0000E114F104E9F0C70160EA70E0A50198015E
:102E10000E9476588C0197FD04C0C601C92ED82E99
:102E200006C0C7010E947C540BC00E943749F601BE
:102E300081916F018823C9F7C7010E947C5402C0A9
:102E40000FEF1FEFC801CF91DF911F910F91FF90FE
:102E5000EF90DF90CF90BF90AF900895CF93DF9326
:102E60009C01009741F420911233309113332115C6
:102E7000310509F440C0F9019F018191992787FD2F
:102E800090957E2F6F2FA0E0B0E203C084179507C6
:102E900099F34D91552747FD509541155105B1F7CF
:102EA000009739F4109212331092133320E030E07F
:102EB00022C0CB01E92FF62FEF014191552747FDA5
:102EC0005095CF01A0E0B0E26D91772767FD709536
:102ED0006417750761F44115510511F0188202C09D
:102EE00080E090E0809312339093133304C0611517
:102EF000710551F7E1CFC901DF91CF910895CF93CB
:102F0000DF93EC01009749F08A859B85009711F0CB
:102F10000E947216CE010E947216DF91CF91089521
:102F2000CF93DF93FC01DB0116964D935C931797CB
:102F3000C281D381209721F46283738307C0EC019F
:102F4000888599850097D9F7A887B98718961D9223
:102F50001C921997DF91CF910895FB014683578307
:102F6000FC0166A777A70895FC01808191810895EF
:102F7000CF92DF92EF92FF920F931F93CF93DF9345
:102F80007C016A01062F172FC0E0D0E011C0D801E4
:102F90006D918D01772767FD7095D7011696ED919C
:102FA000FC91179718968D919C91199719952196D8
:102FB000CC15DD0564F3DF91CF911F910F91FF9048
:102FC000EF90DF90CF900895AF92BF92CF92DF92B3
:102FD000EF92FF920F931F93DF93CF93CDB7DEB79E
:102FE000AE84BF848E010E5E1F4F80E590E00E948C
:102FF0004A166C017C01009721F160E570E0488978
:10300000598998010E94E2168C0197FF11C0C601F0
:103010000E94721616C0772767FD7095D501169627
:10302000ED91FC91179718968D919C911997199590
:10303000F60161916F01662371F7C7010E94721654
:1030400002C00DEF1FEFC801CF91DF911F910F91CB
:10305000FF90EF90DF90CF90BF90AF900895EF92E8
:10306000FF920F931F93CF93DF938C01DC01129695
:10307000CD91DC91139783E0E82E80E2F82E24C0F6
:10308000288139818C819D81009711F482E090E242
:10309000EDB7FEB73897EDBFFEBF3196ADB7BEB7FF
:1030A00011960D931C931297E282F3822483358349
:1030B000868397830E94E4170884D985C02DEDB7D5
:1030C000FEB73896EDBFFEBF2097D1F6DF91CF91C6
:1030D0001F910F91FF90EF9008952F923F924F9282
:1030E0005F926F927F928F929F92AF92BF92CF9298
:1030F000DF92EF92FF920F931F93DF93CF93CDB7A1
:10310000DEB7C655D040CDBFDEBF65968EAF9FAF50
:1031100065971A0149012DB73EB7285030402DBFA1
:103120003EBFEDB7FEB73196ADB7BEB711968D93E2
:103130009C9312978EE090E28283938364837583DD
:10314000868297820E94E417EDB7FEB73896EDBFEE
:10315000FEBFEE24FF249E012F5A3F4F67962EAFED
:103160003FAF67972E010894411C511C8701B1C0E5
:103170008DB79EB708978DBF9EBFEDB7FEB731964E
:10318000ADB7BEB711964D925C92129720E530E034
:103190002283338386E290E28483958306831783B8
:1031A0000E94D016D201A80FB91F6396AEAFBFAF71
:1031B00063973801EDB7FEB73896EDBFFEBF6801E3
:1031C000AA24BB2478018D01C814D9044CF52DB76D
:1031D0003EB7285030402DBF3EBFEDB7FEB7319609
:1031E000ADB7BEB711960D931C93129767968EAD2F
:1031F0009FAD6797801B910B828393832DE230E212
:1032000024833583D101AC0DBD1D8C91868317823B
:103210000E94D0168DB79EB708968DBF9EBF05C081
:10322000C80163E370E20E9490160D5F1F4F08947F
:10323000A11CB11C0894C11CD11C90E1A916B104B9
:1032400019F687016396EEACFFAC6397A0E3B0E09C
:10325000EA0EFB1EC70167E370E20E94901680E051
:1032600090E0F7016814790474F4D101A60DB71D3C
:103270004C919F012F5F3F4F403214F0408302C0BA
:10328000BEE2B083F90101960894611C711C803183
:10329000910541F7108200D000D0EDB7FEB731960E
:1032A00065962EAD3FAD6597ADB7BEB711962D9320
:1032B0003C9312978AE390E28283938344825582FF
:1032C0000E94E417005F1F4FADB7BEB71696ADBFA3
:1032D000BEBF081519050CF44BCFCA5ADF4FCDBF3E
:1032E000DEBFCF91DF911F910F91FF90EF90DF90A4
:1032F000CF90BF90AF909F908F907F906F905F9096
:103300004F903F902F9008956F927F928F929F924F
:10331000AF92BF92CF92DF92EF92FF920F931F93E3
:10332000DF93CF930F92CDB7DEB73C01DC0150960F
:103330008D919C9151970097B9F11E968D919C911A
:103340001F978F3491052CF050961D921C92519727
:10335000AEC16E3671F0623719F06C35E1F413C00E
:10336000D3011A96ED91FC911B97E80FF91F8DE0A0
:1033700008C0D3011A96ED91FC911B97E80FF91F35
:103380008AE0808308C0D3011A96ED91FC911B97C7
:10339000E80FF91F6083F30186859785019686877C
:1033A0009787108A118A83C16A30E1F16B3024F467
:1033B000683009F038C112C06D30A1F16C3509F0E8
:1033C00032C1D30152968C91529782FF07C081E09F
:1033D00090E050968D939C93519769C1F301868537
:1033E0009785009709F463C1828981FD14C000D0DC
:1033F0000F92ADB7BEB711966D927C92129782E490
:1034000090E213968D939C9314970E94E4170F906B
:103410000F900F900F90F30186859785019786870F
:10342000978745C1D3011A96ED91FC911B971E9683
:103430008D919C911F97E80FF91F108252968C91E5
:10344000529781FD10C000D00F92EDB7FEB7618298
:10345000728286E490E2838394830E94E4170F9043
:103460000F900F900F90D3011A968D919C911B97FE
:1034700054961D921C92559722E030E256962D9359
:103480003C93579717C0F30124893589F9013B967E
:10349000EE0FFF1FE60DF71D80839183C901019692
:1034A000D30154968D939C9355978C30910531F0B0
:1034B00080E090E00E942E17009729F7F301C6885C
:1034C000D788C6010E947E16009709F447C0D30131
:1034D00012960D911C911397AA24BB24EE24FF246D
:1034E00021C0F80180819181B6010E948D1600975C
:1034F00019F1D8018D909C90C6010E947E16AC01F6
:10350000C401B6010E948A16009749F4E114F1043F
:1035100011F4780104C0780191E0A92EB12CF801D2
:103520000085118501151105E1F6A114B104B1F46E
:10353000E114F10499F08701D80116968D919C91C0
:103540001797F3018083918364897589A3014A5E8B
:103550005F4F1296ED91FC91139716C0D3019E9682
:10356000ED91FC919F97309791F0868197818D9393
:103570009C93119754966D917C915597A3014A5E47
:103580005F4F0280F381E02DC301199524C0F30140
:10359000868997890E947E160097E9F000D000D0B6
:1035A000EDB7FEB73196ADB7BEB711966D927C926E
:1035B000129789E490E282839383D30156968D918A
:1035C0009C915797848395830E94E417EDB7FEB7CB
:1035D0003696EDBFFEBFD3011E961D921C921F971B
:1035E00052968C91529780FD62C000D000D0EDB70A
:1035F000FEB73196ADB7BEB711966D927C92129719
:1036000080E690E282839383D30114968D919C91FE
:103610001597848395830E94E417EDB7FEB736961D
:10362000EDBFFEBF44C0D3011E968D919C911F97A4
:103630008F349105E4F5862F80528F35C0F5529670
:103640008C91529781FD1EC000D000D0EDB7FEB71F
:103650003196ADB7BEB711966D927C92129784E603
:1036600090E282839383862F992787FD90958483A8
:10367000958369830E94E417EDB7FEB73696EDBFD8
:10368000FEBF6981D3011A96ED91FC911B971E969E
:103690008D919C911F97E80FF91F60831E968D9165
:1036A0009C911F9701961E968D939C931F970F9048
:1036B000CF91DF911F910F91FF90EF90DF90CF900E
:1036C000BF90AF909F908F907F906F9008956F9272
:1036D0007F928F929F92AF92BF92CF92DF92EF92A2
:1036E000FF920F931F93CF93DF937C016B014A01ED
:1036F000B22EA32E6115710509F455C080E390E048
:103700000E944A16682EE3013E01792EE3018301EF
:10371000209709F44AC0C30160E070E040E350E044
:103720000E947816E114F10421F457E6E52E50E2E8
:10373000F52EEC82FD8280E590E08C879D870E94CB
:103740004A168A879B87009721F4CE010E94721641
:103750002AC04C855D8560E070E00E947816BA8AC8
:10376000AB8ACE82DF8288869986B0FC1EC000D0EC
:1037700000D0EDB7FEB73196ADB7BEB71196CD9379
:10378000DC93129780E690E2828393838C819D8103
:10379000848395830E94E4172DB73EB72A5F3F4F7D
:1037A0002DBF3EBF02C000E010E0C801DF91CF9105
:1037B0001F910F91FF90EF90DF90CF90BF90AF904F
:1037C0009F908F907F906F9008952F923F924F928D
:1037D0005F926F927F928F929F92AF92BF92CF92A1
:1037E000DF92EF92FF920F931F93DF93CF930F928D
:1037F0000F92CDB7DEB75C0181E090E069837A83F8
:103800000E944D16282E392E69817A8121143104A7
:1038100009F44CC0062F172FEE24FF24250108942D
:10382000410851083FC061E0C62ED12CE414F504D4
:1038300014F0CC24DD24C1010E947E164C01380115
:10384000F801808191810E947E16B6016F5F7F4FE3
:10385000680D791D680F791FC1010E946F160097CE
:1038600031F4C1010E947216222433241FC01C01AE
:103870000E947E160E5F1F4FF30160817181820DE1
:10388000931D0E949016C114D10449F0C1010E94F9
:103890007E16820D931D60E070E20E9490160894DF
:1038A000E11CF11CEA14FB040CF4BDCFC1010F9024
:1038B0000F90CF91DF911F910F91FF90EF90DF90CC
:1038C000CF90BF90AF909F908F907F906F905F90C0
:1038D0004F903F902F9008952F923F924F925F927A
:1038E0006F927F928F929F92AF92BF92CF92DF9210
:1038F000EF92FF920F931F93DF93CF93CDB7DEB775
:10390000C455D040CDBFDEBF1B014A0100D000D05E
:10391000EDB7FEB7319625E830E2ADB7BEB71196E8
:103920002D933C93129782839383448355830E9403
:10393000E516EDB7FEB73696EDBFFEBFEE24FF24C9
:103940009E012F5A3F4F65962EAF3FAF65972E01D0
:103950000894411C511C8701A5C08DB79EB70897DC
:103960008DBF9EBFEDB7FEB73196ADB7BEB711960E
:103970004D925C92129720E530E0228333838DE9EB
:1039800090E284839583068317830E94D016D20128
:10399000A80FB91F6396AEAFBFAF63973801EDB7FD
:1039A000FEB73896EDBFFEBF6801AA24BB2478019C
:1039B0008D01C814D9044CF52DB73EB728503040BE
:1039C0002DBF3EBFEDB7FEB73196ADB7BEB711966E
:1039D0000D931C93129765968EAD9FAD6597801BD6
:1039E000910B8283938324EA30E224833583D101CF
:1039F000AC0DBD1D8C91868317820E94D0168DB7A9
:103A00009EB708968DBF9EBF05C0C8016AEA70E2E6
:103A10000E9490160D5F1F4F0894A11CB11C0894C2
:103A2000C11CD11C90E1A916B10419F68701639657
:103A3000EEACFFAC6397A0E3B0E0EA0EFB1EC7015B
:103A40006EEA70E20E94901680E090E0F701681440
:103A5000790474F4D101A60DB71D4C919F012F5F1D
:103A60003F4F403214F0408302C0BEE2B083F90100
:103A700001960894611C711C8031910541F71082F8
:103A800000D00F9221EB30E2EDB7FEB721833283F5
:103A9000438254820E94E516005F1F4F0F900F90E3
:103AA0000F900F90081519050CF457CFCC5ADF4F23
:103AB000CDBFDEBFCF91DF911F910F91FF90EF90AF
:103AC000DF90CF90BF90AF909F908F907F906F903E
:103AD0005F904F903F902F900895FC0197FF0BC08F
:103AE0007696E631F10550F4EE0FFF1FE957FD4CD5
:103AF0002081318105C029EB30E202C021EC30E2A7
:103B0000C901089586E090E00E944D168093143319
:103B100090931533009719F42DEF3FEF02C020E08A
:103B200030E0C9010895CF92DF92EF92FF920F9398
:103B30001F93CF93DF936C018B01EA0179012097EA
:103B4000A1F18CE090E00E944D16FC019C010097D1
:103B500071F1C283D383E482F5820115110529F046
:103B600086819781826086839783C0911433D09138
:103B70001533A881B981109721F4E883F98309C02E
:103B8000DC018D919C9111970097D1F7ED93FC93F7
:103B900011978A819B8180879187C286D38686818F
:103BA00097818E7F8683978302C020E030E0C90131
:103BB000DF91CF911F910F91FF90EF90DF90CF9009
:103BC0000895CF93DF930097D1F1A0911433B09172
:103BD000153314962C91149720FF0BC0DC01169618
:103BE0002D913C911797246016962D933C9317972F
:103BF00026C0CD91DC9111979E01E0E0F0E019C064
:103C00002817390731F0F90150814181252F342FD0
:103C100010C0309731F4288139812D933C9311974E
:103C200005C0DC012D913C91208331830E947216E6
:103C300006C02115310521F72EEF3FEF02C020E02D
:103C400030E0C901DF91CF910895FC01A0911433B8
:103C5000B091153312968D919C911397808791871F
:103C600062877387868197818E7F86839783089585
:103C7000E0911433F091153322813381C901089505
:103C8000E0911433F0911533309731F02281338174
:103C9000280F391F2283338308954115510519F0E8
:103CA00086179707A1F06817790740F0681B790B12
:103CB00021E030E06417750760F409C080959095A5
:103CC000860F971F21E030E08417950710F420E05D
:103CD00030E0C90108950F931F93CF93DF93E091D4
:103CE0001433F091153384819581816084839583A9
:103CF000C081D18130C00E811F81C8018570907054
:103D0000009731F5E0911433F0911533628173819E
:103D10004A855B85888599850E944D1E0097C1F074
:103D200001600E831F836C817D81EA81FB81CE015E
:103D300019958E819F8181FF0BC0E0911433F09122
:103D4000153322813381288739878E7F8E839F8325
:103D50000990D881C02D209771F6E0911433F0912D
:103D60001533848195818E7F848395830190F081C2
:103D7000E02DC0E0D0E024C0868182FF1CC02097E7
:103D800079F42091143330911533D9018D919C91A0
:103D9000DC018D919C91D9018D939C93119704C066
:103DA000808191818883998310810181CF010E9454
:103DB0007216C80103C0EF0190818181E92FF82FAD
:103DC0003097D1F6DF91CF911F910F910895EF9227
:103DD000FF920F931F93CF93DF938C01C091143305
:103DE000D0911533EA80FB806A817B81C701A801ED
:103DF0000E944D1E0097C1F3DF91CF911F910F914B
:103E0000FF90EF9008956817790730F49C01209592
:103E10003095260F371F03C09B01281B390BC901A2
:103E20000895CF93DF93FC01DB018D939C93DC011C
:103E300020E030E026C0863271F410822417350766
:103E4000FCF4E901CC0FDD1FCC0FDD1FC60FD71F1F
:103E5000A883B98315C08D3399F4E901CC0FDD1F18
:103E6000CC0FDD1FC60FD71F88819981009741F0C5
:103E700010822417350724F4AA83BB832F5F3F4F9A
:103E800031968D918823B9F6C901DF91CF910895BC
:103E9000AF92BF92CF92DF92EF92FF920F931F9358
:103EA000CF93DF935C016A01E62EE7017E01F72ED6
:103EB000E701EE24FF2400E010E00FC06881798163
:103EC0006115710569F0C5010E948D16009711F406
:103ED000EA80FB800F5F1F4F24960C151D0574F3BD
:103EE000C701DF91CF911F910F91FF90EF90DF906D
:103EF000CF90BF90AF9008958DE290E061E070E0C8
:103F00000E946A498EE290E062E070E00E946A4995
:103F10008EE290E00E94A94989E290E062E070E0C0
:103F20000E946A4989E290E00E94944984EF91E0FE
:103F30000E94294989E290E00E94A94984EF91E01A
:103F40000E94294980E090E0089589E290E062E0D3
:103F500070E00E946A4989E290E00E94944980E002
:103F600090E008952DB73EB72A5030402DBF3EBF98
:103F7000EDB7FEB73196ADB7BEB711968D939C9352
:103F8000129787EF91E28283938381E090E08483AC
:103F9000958323E030E026833783808791870E94D2
:103FA000E4172DB73EB7265F3F4F2DBF3EBF0895A4
:103FB0002DB73EB7285030402DBF3EBFEDB7FEB7FE
:103FC0003196ADB7BEB711968D939C9312978DE045
:103FD00092E28283938364837583468357830E942E
:103FE000E4172DB73EB7285F3F4F2DBF3EBF089562
:103FF0000F931F93CF93DF93EC018B010E947E16EA
:10400000482FF80180A3C801BE0150E00E94751638
:1040100081E090E0DF91CF911F910F910895CF92B1
:10402000DF92EF92FF920F931F93DF93CF93CDB761
:10403000DEB7A197CDBFDEBF7C01623071057CF099
:10404000DA0112968D919C9113978E010F5F1F4F8D
:10405000B8010E94F81F0097B1F1C80102C080E0CA
:1040600090E063E870E2A7010E94000C8C0197FDCC
:1040700005C09EE2C92E92E2D92E04C081E3C82E6B
:1040800082E2D82EC8010E946D1DEDB7FEB73A97A7
:10409000EDBFFEBF3196ADB7BEB71196ED92FC9263
:1040A000129725E332E222833383C482D5820683CA
:1040B0001783808791870E94E417EDB7FEB73A9681
:1040C000EDBFFEBF14C000D00F92ADB7BEB71196C2
:1040D000ED92FC92129782E492E213968D939C9358
:1040E00014970E94E4170F900F900F900F90A196D5
:1040F000CDBFDEBFCF91DF911F910F91FF90EF9069
:10410000DF90CF9008952F923F924F925F926F92DF
:104110007F928F929F92AF92BF92CF92DF92EF9257
:10412000FF920F931F93DF93CF93CDB7DEB7A39783
:10413000CDBFDEBF5C016115710571F400D00F9237
:10414000EDB7FEB73196ADB7BEB711968C93119708
:10415000B18282E692E212C0CE0101960E94030C67
:104160000097A9F000D00F92EDB7FEB73196ADB72A
:10417000BEB71196AC92B18282E792E282839383BA
:104180000E94E4170F900F900F900F9088C100D0FD
:104190000F92EDB7FEB73196ADB7BEB71196AC92A0
:1041A000B1828FE892E2828393830E94E417EDB795
:1041B000FEB73196ADB7BEB71196AC92B18287EC1F
:1041C00092E2828393830E94E4170F900F900F90E6
:1041D0000F90EE24FF24CC24DD245FE0652E53E213
:1041E000752E4FE2442E43E2542E37E4232E33E261
:1041F000332E23E0822E912C8C0E9D1E48C102810D
:1042000013810E0D1F1DEDB7FEB77097EDBFFEBFFA
:104210003196ADB7BEB71196AC92B182628273820D
:10422000D80191968C9191978483158292968C9166
:1042300092978683178293968C91939780871186A5
:1042400094968C9194978287138695968C919597E6
:104250008487158696968C91868717860E94E41728
:10426000EDB7FEB77096EDBFFEBFD8019E968D915B
:104270009C919F97009719F486E592E202C08CE525
:1042800092E2EDB7FEB73A97EDBFFEBF3196ADB7FC
:10429000BEB71196AC92B1824282538284839583D9
:1042A000D8019D968C919D978683178297968D91C4
:1042B0009C919897808791870E94E417F80181A5C7
:1042C00092A52DB73EB7265F3F4F2DBF3EBF3FEFB4
:1042D00080389307C1F000D000D0EDB7FEB731961B
:1042E000ADB7BEB71196AC92B1822FE333E2228311
:1042F0003383848395830E94E4178DB79EB7069617
:104300008DBF9EBF12C000D00F92EDB7FEB73196A1
:10431000ADB7BEB71196AC92B182228233820E94B1
:10432000E4170F900F900F900F90F80183A594A5BC
:104330008230910591F18330910538F4009789F02E
:104340008130910509F067C01AC08430910509F4E5
:1043500040C08430910578F18530910509F05BC04B
:1043600046C000D00F92EDB7FEB73196ADB7BEB7DD
:104370001196AC921197B1822DE433E244C000D083
:104380000F92EDB7FEB73196ADB7BEB71196AC92AE
:104390001197B18228E533E236C000D00F92EDB715
:1043A000FEB73196ADB7BEB71196AC921197B182F8
:1043B00023E633E228C000D00F92EDB7FEB7319666
:1043C000ADB7BEB71196AC921197B1822EE633E22B
:1043D0001AC000D00F92EDB7FEB73196ADB7BEB799
:1043E0001196AC921197B18229E733E20CC000D04C
:1043F0000F92EDB7FEB73196ADB7BEB71196AC923E
:10440000B18224E833E2228333830E94E4170F90C1
:104410000F900F900F90C40160E070E041E250E017
:104420000E947816D80190964C91C401B80150E0D2
:104430000E94751600D000D0EDB7FEB73196ADB72B
:10444000BEB71196AC92B1822FE833E22283338358
:10445000848295820E94E4170F900F90EDB7FEB70B
:104460003196ADB7BEB71196AC92B18222E933E274
:10447000228333830E94E4170894C11CD11C80E37B
:1044800090E0E80EF91E0F900F900F900F90E981C9
:10449000FA8180819181C816D9060CF4B0CEA3961A
:1044A000CDBFDEBFCF91DF911F910F91FF90EF90B5
:1044B000DF90CF90BF90AF909F908F907F906F9044
:1044C0005F904F903F902F900895EF92FF920F933F
:1044D0001F93DF93CF930F920F92CDB7DEB78C016E
:1044E0007B01BE016F5F7F4F40E050E00E94C1162C
:1044F000F701608371838283938321E030E040E0A1
:1045000050E089819A818017910719F420E030E00A
:10451000A901B901CA010F900F90CF91DF911F91AE
:104520000F91FF90EF900895CF92DF92EF92FF925C
:104530000F931F93DF93CF9300D00F92CDB7DEB7C9
:104540006C01623071050CF442C0DA0112968D9153
:104550009C911397BE016F5F7F4F0E94652261158A
:1045600071058105910599F169817A818B819C8121
:104570000E9418148C0197FD05C07EE2E72E72E2BE
:10458000F72E04C061E3E62E62E2F62EC8010E9417
:104590006D1DEDB7FEB73A97EDBFFEBF3196ADB7D3
:1045A000BEB71196CD92DC92129725E332E22283B8
:1045B0003383E482F58206831783808791870E9484
:1045C000E417EDB7FEB73A96EDBFFEBF14C000D0BA
:1045D0000F92ADB7BEB71196CD92DC92129785E9D6
:1045E00093E213968D939C9314970E94E4170F9077
:1045F0000F900F900F902496CDBFDEBFCF91DF912B
:104600001F910F91FF90EF90DF90CF900895EF9260
:10461000FF920F931F93DF93CF930F920F92CDB71B
:10462000DEB78C017B01BE016F5F7F4F40E050E041
:104630000E94C116F7016083718321E030E0898117
:104640009A818017910711F420E030E0C9010F90A2
:104650000F90CF91DF911F910F91FF90EF900895F0
:10466000EF92FF920F931F93DF93CF930F920F92CE
:10467000CDB7DEB78C017B01BE016F5F7F4F40E09D
:1046800050E00E94C11629813A812017310741F07C
:1046900077FD06C0F7016083718321E030E002C03E
:1046A00020E030E0C9010F900F90CF91DF911F9172
:1046B0000F91FF90EF900895CF92DF92EF92FF92CB
:1046C0000F931F93DF93CF9300D00F92CDB7DEB738
:1046D0006C01623071050CF460C0DA0112968D91A4
:1046E0009C911397BE016F5F7F4F0E9465226115F9
:1046F00071058105910509F450C069817A818B812A
:104700009C810E94FC138C0100D000D0EDB7FEB755
:104710003196ADB7BEB71196CD92DC9212978DEB64
:1047200093E28283938389819A81848395830E9413
:10473000E417EDB7FEB73696EDBFFEBF17FD05C017
:10474000FEE2EF2EF2E2FF2E04C0E1E3EE2EE2E203
:10475000FE2EC8010E946D1D2DB73EB72A50304075
:104760002DBF3EBFEDB7FEB73196ADB7BEB71196C0
:10477000CD92DC92129725E332E222833383E482E6
:10478000F58206831783808791870E94E417EDB72F
:10479000FEB73A96EDBFFEBF14C000D00F92ADB782
:1047A000BEB71196CD92DC92129789EC93E21396E4
:1047B0008D939C9314970E94E4170F900F900F9085
:1047C0000F902496CDBFDEBFCF91DF911F910F9147
:1047D000FF90EF90DF90CF900895CF92DF92EF920D
:1047E000FF920F931F93DF93CF930F920F92CDB74A
:1047F000DEB76C0162307105ECF1DA0112968D9131
:104800009C911397BE016F5F7F4F0E940723009713
:1048100089F189819A810E94E8138C0197FD05C076
:10482000BEE2EB2EB2E2FB2E04C0A1E3EA2EA2E22E
:10483000FA2EC8010E946D1DEDB7FEB73A97EDBF85
:10484000FEBF3196ADB7BEB71196CD92DC921297EE
:1048500025E332E222833383E482F58206831783E1
:10486000808791870E94E417EDB7FEB73A96EDBFB7
:10487000FEBF14C000D00F92ADB7BEB71196CD9257
:10488000DC92129786EE93E213968D939C93149785
:104890000E94E4170F900F900F900F900F900F90C1
:1048A000CF91DF911F910F91FF90EF90DF90CF900C
:1048B0000895CF92DF92EF92FF920F931F93DF93B1
:1048C000CF930F92CDB7DEB76C01CE0101960E9457
:1048D000800A8C0197FD05C09EE2E92E92E2F92E36
:1048E00004C081E3E82E82E2F82EC8010E946D1D0B
:1048F0002DB73EB72A5030402DBF3EBFEDB7FEB7B3
:104900003196ADB7BEB71196CD92DC92129725E3E2
:1049100032E222833383E482F58206831783808721
:1049200091870E94E4170F900F900F900F90EDB7B2
:10493000FEB73196ADB7BEB71196CD92DC92129705
:104940008DEF93E2828393838981848315820E9411
:10495000E4172DB73EB72A5F3F4F2DBF3EBF0F90E4
:10496000CF91DF911F910F91FF90EF90DF90CF904B
:104970000895CF92DF92EF92FF920F931F93DF93F0
:10498000CF93CDB7DEB7A497CDBFDEBF6C01CE010C
:104990000196BE016B5F7F4F40E150E09E012B5EB0
:1049A0003F4F00E110E00E948A0B8C0197FD05C08B
:1049B0004EE2E42E42E2F42E04C031E3E32E32E272
:1049C000F32EC8010E946D1D2DB73EB72A5030400E
:1049D0002DBF3EBFEDB7FEB73196ADB7BEB711964E
:1049E000CD92DC92129725E332E222833383E48274
:1049F000F58206831783808791870E94E417898157
:104A00009A81AB81BC810F920F926DB77EB76F5FB9
:104A10007F4FEDB7FEB7C182D28223E134E2FB01C2
:104A2000228333832A2F30E024833583292F3A2FA2
:104A30004B2F55273070268337839070808791875E
:104A4000CE010596828793870E94E4172DB73EB763
:104A5000245F3F4F2DBF3EBF8E010B5E1F4FC8012D
:104A60000E947E16009711F40BE014E200D000D0F3
:104A7000EDB7FEB73196ADB7BEB71196CD92DC92C9
:104A8000129782E394E282839383048315830E94C6
:104A9000E417EDB7FEB73696EDBFFEBFA496CDBFC7
:104AA000DEBFCF91DF911F910F91FF90EF90DF90CC
:104AB000CF9008958F929F92AF92BF92CF92DF9244
:104AC000EF92FF920F931F93DF93CF9300D00F923B
:104AD000CDB7DEB74C018B017A016E010894C11C81
:104AE000D11CC60160E070E040E050E020E030E022
:104AF0000E94790CC80101978530910508F097C094
:104B00000130110509F4A8C0D70112968D919C912E
:104B1000139764E474E20E948D16009709F087C031
:104B20000230110509F498C0F70184819581B6011E
:104B30000E947A14009709F47AC00330110509F431
:104B40008BC0D70116968D919C91179760E070E00D
:104B50004AE050E00E94C1165B010530110521F4C6
:104B6000F7010085118502C000E010E080E0BE0181
:104B70006F5F7F4FA50198010E948F137C0197FD05
:104B800005C07EE2C72E72E2D72E04C061E3C62EB6
:104B900062E2D62EC7010E946D1D2DB73EB72A5086
:104BA00030402DBF3EBFEDB7FEB73196ADB7BEB7B3
:104BB00011968D929C92129725E332E222833383E1
:104BC000C482D582E682F782808791870E94E417AB
:104BD000EDB7FEB73A96EDBFFEBFCE0101960E943B
:104BE000E9150115110511F403E414E22DB73EB7E0
:104BF0002A5030402DBF3EBFEDB7FEB73196ADB75E
:104C0000BEB711968D929C9212972EE434E22283C5
:104C1000338384839583A682B782008711870E949D
:104C2000E417EDB7FEB73A96EDBFFEBF1AC000D04D
:104C30000F92ADB7BEB711968D929C92129786E6F1
:104C400094E213968D939C9314970E94E4170F900F
:104C50000F900F900F9005C050E9A52E5FE1B52E83
:104C600083CF2496CDBFDEBFCF91DF911F910F91EF
:104C7000FF90EF90DF90CF90BF90AF909F908F907C
:104C800008950F931F938C0161157105A9F400D04D
:104C90000F92EDB7FEB73196ADB7BEB711968C93B4
:104CA00011838AEA94E2828393830E94E4170F902F
:104CB0000F900F900F901AC0CB010E94E91500D001
:104CC00000D0EDB7FEB73196ADB7BEB711960C93D5
:104CD000118326EC34E222833383848395830E94FC
:104CE000E4178DB79EB706968DBF9EBF1F910F919B
:104CF00008950F931F93DF93CF93CDB7DEB76097DF
:104D0000CDBFDEBF8C01CE010196BE016B5F7F4F30
:104D1000AE01475F5F4F9E01235F3F4F0E94790CBA
:104D200097FD03C02EE232E202C021E332E24DB72A
:104D30005EB7485050404DBF5EBFEDB7FEB73196ED
:104D4000ADB7BEB711960D931C93129748ED54E280
:104D50004283538324833583868397830E94E41799
:104D60004DB75EB7485F5F4F4DBF5EBFCE01019646
:104D70000E94E91500D000D0EDB7FEB73196ADB76F
:104D8000BEB711960D931C93129720EE34E2228346
:104D90003383848395830E94E4174DB75EB74A5FDF
:104DA0005F4F4DBF5EBFCE0105960E94E91500D052
:104DB00000D0EDB7FEB73196ADB7BEB711960D93E3
:104DC0001C93129727EE34E22283338384839583E6
:104DD0000E94E4174DB75EB74A5F5F4F4DBF5EBF9D
:104DE000CE0109960E94E91500D000D0EDB7FEB7BC
:104DF0003196ADB7BEB711960D931C93129720EF65
:104E000034E222833383848395830E94E4174DB771
:104E10005EB74A5F5F4F4DBF5EBFCE010D960E94E9
:104E2000E91500D000D0EDB7FEB73196ADB7BEB7EB
:104E300011960D931C93129727EF34E2228333834C
:104E4000848395830E94E4174DB75EB74A5F5F4F36
:104E50004DBF5EBF6096CDBFDEBFCF91DF911F918A
:104E60000F910895EF92FF920F931F93CF93DF93CB
:104E7000EC0162307105BCF1DA0112968D919C91C2
:104E8000139761E476E2AE010E94E0108C0197FD79
:104E900005C0FEE2EF2EF2E2FF2E04C0E1E3EE2EAB
:104EA000E2E2FE2EC8010E946D1DEDB7FEB73A97F3
:104EB000EDBFFEBF3196ADB7BEB71196CD93DC9373
:104EC000129725E332E222833383E482F58206835C
:104ED0001783808791870E94E417EDB7FEB73A9653
:104EE000EDBFFEBF14C000D00F92ADB7BEB7119694
:104EF0008D939C93129781E095E213968D939C93EA
:104F000014970E94E4170F900F900F900F90DF916D
:104F1000CF911F910F91FF90EF900895CF92DF9264
:104F2000EF92FF920F931F93DF93CF9300D000D0A7
:104F3000CDB7DEB76C01623071050CF45DC0DA01EB
:104F400012968D919C911397BE016F5F7F4F0E94C7
:104F50000723009709F450C089819A81BE016D5FD3
:104F60007F4F0E94B4108C0197FD05C0BEE2EB2E6E
:104F7000B2E2FB2E04C0A1E3EA2EA2E2FA2EC8019F
:104F80000E946D1DEDB7FEB73A97EDBFFEBF31969B
:104F9000ADB7BEB71196CD92DC92129723E235E2FF
:104FA00022833383E482F582068317838087918787
:104FB0000E94E417EDB7FEB73A96EDBFFEBFCE01F3
:104FC00003960E94E91500D000D0EDB7FEB73196E8
:104FD000ADB7BEB71196CD92DC9212972FE235E2B3
:104FE00022833383848395830E94E417EDB7FEB751
:104FF0003696EDBFFEBF14C000D00F92ADB7BEB75E
:105000001196CD92DC92129789E395E213968D93D7
:105010009C9314970E94E4170F900F900F900F909D
:105020002696CDBFDEBFCF91DF911F910F91FF90EC
:10503000EF90DF90CF9008952F923F924F925F9222
:105040006F927F928F929F92AF92BF92CF92DF9298
:10505000EF92FF920F931F93DF93CF93CDB7DEB7FD
:105060002897CDBFDEBF4C017B018A0164307105FA
:105070000CF4CEC0DA0112968D919C911397BE016B
:105080006F5F7F4F0E940723009709F4C1C035E08E
:10509000A32EB12CAC0EBD1EF80184819581B50103
:1050A0000E947A14009709F4B3C0D80116968D9126
:1050B0009C911797BE016D5F7F4F0E943023009730
:1050C00009F4A6C0B801685F7F4FC70104970E942A
:1050D000E51B6C01009709F471C00E947E163C012B
:1050E000C5010E94E915EDB7FEB73A97EDBFFEBFC7
:1050F0003196ADB7BEB711968D929C92129728E566
:1051000035E22283338364827582868397838B8121
:105110009C81808791870E94E417EDB7FEB73A968D
:10512000EDBFFEBFEE24FF243A2C2B2C24E7422EA9
:1051300025E2522E36C05301AE18BF08B6016E0DDF
:105140007F1D0B811C8189819A81A501232D322D20
:105150000E943B108C0197FF04C0C6010E947C5442
:105160002FC02DB73EB7285030402DBF3EBFEDB702
:10517000FEB73196ADB7BEB711968D929C9212973D
:105180004282538284839583A81AB90AA682B78281
:105190000E94E417E00EF11EEDB7FEB73896EDBFA2
:1051A000FEBFE614F7043CF2C6010E947C5400E006
:1051B00010E09EE2E92E92E2F92E06C00DEF1FEFFD
:1051C00081E3E82E82E2F82EC8010E946D1D2DB702
:1051D0003EB72A5030402DBF3EBFEDB7FEB73196E7
:1051E000ADB7BEB711968D929C92129725E332E22D
:1051F00022833383E482F582068317838087918735
:105200000E94E417EDB7FEB73A96EDBFFEBF14C09B
:1052100000D00F92ADB7BEB711968D929C921297A7
:1052200089E895E213968D939C9314970E94E41756
:105230000F900F900F900F902896CDBFDEBFCF91AB
:10524000DF911F910F91FF90EF90DF90CF90BF9073
:10525000AF909F908F907F906F905F904F903F9016
:105260002F9008954F925F926F927F928F929F92AC
:10527000AF92BF92CF92DF92EF92FF920F931F9364
:10528000DF93CF930F920F92CDB7DEB74C017B0126
:105290008A01633071050CF4A1C0DA0112968D9178
:1052A0009C911397BE016F5F7F4F0E940723009769
:1052B00009F494C0B8016C5F7F4FC70102970E9448
:1052C000E51B6C01009709F45FC00E947E165C012B
:1052D00000D000D0EDB7FEB73196ADB7BEB711968E
:1052E0008D929C92129789EB95E282839383A4829C
:1052F000B5820E94E417EDB7FEB73696EDBFFEBF4C
:1053000000E010E054E7452E55E2552E32C035013D
:10531000601A710AB601600F711F89819A81A30119
:105320000E94D70F7C0197FF04C0C6010E947C54E5
:105330002FC02DB73EB7285030402DBF3EBFEDB730
:10534000FEB73196ADB7BEB711968D929C9212976B
:105350004282538284839583681A790A66827782AF
:105360000E94E4170E0D1F1DEDB7FEB73896EDBF76
:10537000FEBF0A151B055CF2C6010E947C54EE2498
:10538000FF240EE212E206C04DEFE42E4FEFF42EA2
:1053900001E312E2C7010E946D1D2DB73EB72A50EE
:1053A00030402DBF3EBFEDB7FEB73196ADB7BEB7AB
:1053B00011968D929C92129725E332E222833383D9
:1053C00004831583E682F782808791870E94E41721
:1053D000EDB7FEB73A96EDBFFEBF14C000D00F92F6
:1053E000ADB7BEB711968D929C9212978CEC95E258
:1053F00013968D939C9314970E94E4170F900F902F
:105400000F900F900F900F90CF91DF911F910F9100
:10541000FF90EF90DF90CF90BF90AF909F908F90D4
:105420007F906F905F904F900895CF92DF92EF92B0
:10543000FF920F931F93DF93CF930F920F92CDB7ED
:10544000DEB76C0162307105ECF1DA0112968D91D4
:105450009C911397BE016F5F7F4F0E9407230097B7
:1054600089F189819A810E94D40E8C0197FD05C033
:105470007EE2E72E72E2F72E04C061E3E62E62E2DE
:10548000F62EC8010E946D1DEDB7FEB73A97EDBF2D
:10549000FEBF3196ADB7BEB71196CD92DC92129792
:1054A00025E332E222833383E482F5820683178385
:1054B000808791870E94E417EDB7FEB73A96EDBF5B
:1054C000FEBF14C000D00F92ADB7BEB71196CD92FB
:1054D000DC9212978EEE95E213968D939C9314971F
:1054E0000E94E4170F900F900F900F900F900F9065
:1054F000CF91DF911F910F91FF90EF90DF90CF90B0
:105500000895CF92DF92EF92FF920F931F93DF9354
:10551000CF93CDB7DEB72897CDBFDEBF6C018A0130
:10552000643071050CF45BC0DA0112968D919C9188
:105530001397BE016F5F7F4F0E940723009709F406
:105540004EC0A5E0EA2EF12CEC0EFD1EF801848180
:105550009581B7010E947A14009709F440C0D801E0
:1055600016968D919C911797BE016D5F7F4F0E949B
:1055700030230097A1F14B815C8189819A81B70129
:105580000E943C0E8C0197FD05C0FEE2EF2EF2E278
:10559000FF2E04C0E1E3EE2EE2E2FE2EC8010E94DF
:1055A0006D1DEDB7FEB73A97EDBFFEBF3196ADB7B3
:1055B000BEB71196CD92DC92129725E332E2228398
:1055C0003383E482F58206831783808791870E9464
:1055D000E417EDB7FEB73A96EDBFFEBF14C000D09A
:1055E0000F92ADB7BEB71196CD92DC92129786E0BE
:1055F00096E213968D939C9314970E94E4170F9054
:105600000F900F900F902896CDBFDEBFCF91DF9106
:105610001F910F91FF90EF90DF90CF900895CF9260
:10562000DF92EF92FF920F931F93DF93CF9300D0FF
:105630000F92CDB7DEB76C017B018A0181E090E06B
:105640008B839C83623071050CF454C0DA0112968E
:105650008D919C911397BE016F5F7F4F0E9407232E
:10566000009709F447C0B2E0EB16F10451F0F801DD
:1056700084819581BE016D5F7F4F0E940723009753
:10568000C9F16B817C8189819A814AE95BE296014B
:105690000E94FE0D8C0197FD05C08EE2E82E82E28D
:1056A000F82E04C0B1E3EB2EB2E2FB2EC8010E943B
:1056B0006D1D2DB73EB72A5030402DBF3EBFEDB710
:1056C000FEB73196ADB7BEB71196CD92DC92129768
:1056D00025E332E222833383E482F5820683178353
:1056E000808791870E94E417EDB7FEB73A96EDBF29
:1056F000FEBF14C000D00F92ADB7BEB71196CD92C9
:10570000DC9212978CE296E213968D939C931497F9
:105710000E94E4170F900F900F900F902496CDBF2A
:10572000DEBFCF91DF911F910F91FF90EF90DF903F
:10573000CF900895EF92FF920F931F93CF93DF9333
:105740007C01EB0100D000D0EDB7FEB73196ADB7CC
:10575000BEB711968C93F1828FE496E28283938395
:10576000648375830E94E4172DB73EB72A5F3F4FCD
:105770002DBF3EBFCE010E94820EEC011816190605
:1057800064F468ED7FE1A7010E94970DCE016BEFF5
:105790007BE2A7010E94B10D02C0009719F40EE24E
:1057A00012E202C001E312E2CE010E946D1DADB70C
:1057B000BEB71A97ADBFBEBFEDB7FEB73196119613
:1057C000EC92F18225E332E2228333830483158352
:1057D000C683D783808791870E94E4172DB73EB791
:1057E000265F3F4F2DBF3EBFDF91CF911F910F919D
:1057F000FF90EF900895AF92BF92CF92DF92EF9219
:10580000FF920F931F93DF93CF93CDB7DEB7C054B2
:10581000D040CDBFDEBFB82EA92E6B018A01411545
:10582000510519F083E494E202C083E796E22DB7B4
:105830003EB72A5030402DBF3EBFEDB7FEB7319680
:10584000ADB7BEB71196BC92A18225E836E222839D
:105850003383C482D58206831783808791870E9411
:10586000E4172DB73EB7265F3F4F2DBF3EBF7E01E9
:105870000894E11CF11C18C00134110518F040E433
:1058800050E001C0A801C601B7010E942F0F9C0182
:10589000181619068CF7081B190B8B2D9A2D63EA25
:1058A00076E2A7010E946D18101611062CF3C05C59
:1058B000DF4FCDBFDEBFCF91DF911F910F91FF90E2
:1058C000EF90DF90CF90BF90AF900895CF92DF928E
:1058D000EF92FF920F931F93DF93CF93CDB7DEB775
:1058E0002897CDBFDEBF6C018A01643071050CF4CE
:1058F0005BC0DA0112968D919C911397BE016F5F88
:105900007F4F0E940723009709F44EC035E0E32E35
:10591000F12CEC0EFD1EF80184819581B7010E94E7
:105920007A14009709F440C0D80116968D919C9185
:105930001797BE016D5F7F4F0E9430230097A1F142
:105940004B815C8189819A81B7010E94CB0D8C01CA
:1059500097FD05C02EE2E22E22E2F22E04C091E372
:10596000E92E92E2F92EC8010E946D1DEDB7FEB737
:105970003A97EDBFFEBF3196ADB7BEB71196CD9247
:10598000DC92129725E332E222833383E482F582AC
:1059900006831783808791870E94E417EDB7FEB7CF
:1059A0003A96EDBFFEBF14C000D00F92ADB7BEB7A0
:1059B0001196CD92DC92129786EA96E213968D9319
:1059C0009C9314970E94E4170F900F900F900F90E4
:1059D0002896CDBFDEBFCF91DF911F910F91FF9031
:1059E000EF90DF90CF900895AF92BF92CF92DF9269
:1059F000EF92FF920F931F93DF93CF930F920F922B
:105A0000CDB7DEB76C015B018A0119821A82623060
:105A100071050CF479C0DA0112968D919C9113975F
:105A200069EC76E20E948D160097C9F0F801828138
:105A3000938160ED76E20E948D16009799F0D8016F
:105A400012968D919C91139766ED76E20E948D16C9
:105A5000009709F059C072E0E72EF12C06C0EE2441
:105A6000FF2403C061E0E62EF12CB2E0AB16B104D6
:105A700059F0F80184819581BE016F5F7F4F0E94CC
:105A80000723009709F440C069817A81C7010E9409
:105A9000400D8C0168ED7FE1A6010E94970DC801C1
:105AA0006BEF7BE2A6010E94B10D17FD05C05EE21F
:105AB000E52E52E2F52E04C041E3E42E42E2F42E3C
:105AC000C8010E946D1D2DB73EB72A5030402DBF32
:105AD0003EBFEDB7FEB73196ADB7BEB71196CD92CA
:105AE000DC92129725E332E222833383E482F5824B
:105AF00006831783808791870E94E417EDB7FEB76E
:105B00003A96EDBFFEBF14C000D00F92ADB7BEB73E
:105B10001196CD92DC9212978AED96E213968D93B0
:105B20009C9314970E94E4170F900F900F900F9082
:105B30000F900F90CF91DF911F910F91FF90EF90F9
:105B4000DF90CF90BF90AF900895CF92DF92EF9209
:105B5000FF920F931F93DF93CF930F920F92CDB7C6
:105B6000DEB76C0162307105ECF1DA0112968D91AD
:105B70009C911397BE016F5F7F4F0E940723009790
:105B800089F189819A810E94BA0C8C0197FD05C028
:105B9000FEE2EF2EF2E2FF2E04C0E1E3EE2EE2E29F
:105BA000FE2EC8010E946D1DEDB7FEB73A97EDBFFE
:105BB000FEBF3196ADB7BEB71196CD92DC9212976B
:105BC00025E332E222833383E482F582068317835E
:105BD000808791870E94E417EDB7FEB73A96EDBF34
:105BE000FEBF14C000D00F92ADB7BEB71196CD92D4
:105BF000DC92129788E097E213968D939C9314970A
:105C00000E94E4170F900F900F900F900F900F903D
:105C1000CF91DF911F910F91FF90EF90DF90CF9088
:105C200008950F931F93DF93CF930F920F92CDB7E9
:105C3000DEB78C01CE0101960E949E0C97FD03C039
:105C40002EE232E202C021E332E24DB75EB74A50A3
:105C500050404DBF5EBFEDB7FEB73196ADB7BEB792
:105C600011960D931C93129741E257E2428353839E
:105C7000248335838683978389819A81808791875E
:105C80000E94E4174DB75EB7465F5F4F4DBF5EBFE2
:105C90000F900F90CF91DF911F910F910895CF92A8
:105CA000DF92EF92FF920F931F93DF93CF930F92A8
:105CB0000F92CDB7DEB76C0162307105ECF1DA01FD
:105CC00012968D919C911397BE016F5F7F4F0E943A
:105CD0000723009789F189819A810E948E0C8C019B
:105CE00097FD05C0BEE2EB2EB2E2FB2E04C0A1E39D
:105CF000EA2EA2E2FA2EC8010E946D1DEDB7FEB792
:105D00003A97EDBFFEBF3196ADB7BEB71196CD92B3
:105D1000DC92129725E332E222833383E482F58218
:105D200006831783808791870E94E417EDB7FEB73B
:105D30003A96EDBFFEBF14C000D00F92ADB7BEB70C
:105D40001196CD92DC92129786E397E213968D938B
:105D50009C9314970E94E4170F900F900F900F9050
:105D60000F900F90CF91DF911F910F91FF90EF90C7
:105D7000DF90CF900895CF92DF92EF92FF920F9332
:105D80001F93DF93CF93CDB7DEB76097CDBFDEBF54
:105D90006C017B018A0180917F3290918032A091C9
:105DA0008132B09182328D839E83AF83B887898799
:105DB0009A87AB87BC878D879E87AF87B88B623009
:105DC00071050CF478C0DA0112968D919C911397AD
:105DD000BE016F5F7F4F0E947A14009709F46BC079
:105DE000B2E0EB16F10451F1F80184819581BE0116
:105DF0006B5F7F4F0E947A14009709F45CC0F3E058
:105E0000EF16F104D9F0D80116968D919C91179751
:105E1000BE01675F7F4F0E947A14009709F44BC060
:105E2000B4E0EB16F10451F0F80180859185BE01D4
:105E3000635F7F4F0E947A140097E9F1CE010196CB
:105E4000BE016B5F7F4FAE01475F5F4F9E01235FD7
:105E50003F4F0E94700C8C0197FD05C09EE2E92E19
:105E600092E2F92E04C081E3E82E82E2F82EC80106
:105E70000E946D1D2DB73EB72A5030402DBF3EBF4A
:105E8000EDB7FEB73196ADB7BEB71196CD92DC92A5
:105E9000129725E332E222833383E482F58206837C
:105EA0001783808791870E94E417EDB7FEB73A9673
:105EB000EDBFFEBF14C000D00F92ADB7BEB71196B4
:105EC000CD92DC9212978EE497E213968D939C9379
:105ED00014970E94E4170F900F900F900F90609608
:105EE000CDBFDEBFCF91DF911F910F91FF90EF905B
:105EF000DF90CF9008958F929F92AF92BF92CF92F2
:105F0000DF92EF92FF920F931F93DF93CF93CDB762
:105F1000DEB7C155D040CDBFDEBF8C0132E2E32EEB
:105F2000F12CEC0EFD1EC7010E94F80C4C0122E47E
:105F3000C22ED12CCC0EDD1ED6014C915E010894F0
:105F4000A11CB11CC501B70150E00E947516F601F5
:105F50008081F501E80FF11D108297FC03C08EE2ED
:105F600092E202C081E392E22DB73EB72850304062
:105F70002DBF3EBFEDB7FEB73196ADB7BEB7119698
:105F80000D931C9312972DE737E22283338384838A
:105F90009583868297820E94E417EDB7FEB7389604
:105FA000EDBFFEBFFE01EE5BFF4F8081882319F03D
:105FB000CE01019602C089E797E22DB73EB7225184
:105FC00030402DBF3EBFEDB7FEB73196ADB7BEB77F
:105FD00011960D931C93129724E837E222833383A2
:105FE00084839583DE01AD5BBF4F8C9186831782DE
:105FF000DE01AC5BBF4F8C9180871186DE01AB5B0D
:10600000BF4F8C9182871386DE01AA5BBF4F8C91B4
:1060100084871586DE01A95BBF4F8C918687178622
:10602000DE01A85BBF4F8C91808B118A0E94E41720
:10603000FE01E75BFF4F80819181EDB7FEB772965D
:10604000EDBFFEBFFFEF80389F07C9F000D000D042
:10605000EDB7FEB73196ADB7BEB711960D931C9351
:10606000129727EA37E222833383848395830E9441
:10607000E417EDB7FEB73696EDBFFEBF14C000D0F3
:106080000F92ADB7BEB711960D931C93129780EB8C
:1060900097E213968D939C9314970E94E4170F90A8
:1060A0000F900F900F90FE01E55BFF4F8081918173
:1060B000BFEF80389B07C9F000D000D0EDB7FEB726
:1060C0003196ADB7BEB711960D931C9312972AEB7C
:1060D00037E222833383848395830E94E417EDB7EC
:1060E000FEB73696EDBFFEBF14C000D00F92ADB71D
:1060F000BEB711960D931C93129781EC97E21396FD
:106100008D939C9314970E94E4170F900F900F901B
:106110000F9000D00F92EDB7FEB70183128389EC88
:1061200097E2838394830E94E4170F900F900F905F
:106130000F90CF5ADF4FCDBFDEBFCF91DF911F91C0
:106140000F91FF90EF90DF90CF90BF90AF909F9016
:106150008F9008950F931F93DF93CF9300D000D0BB
:10616000CDB7DEB78C01CE0101960E94D30C97FD0E
:1061700003C02EE232E202C021E332E24DB75EB745
:10618000445150404DBF5EBFEDB7FEB73196ADB73D
:10619000BEB711960D931C9312974DEC57E24283B4
:1061A00053832483358386839783898180871186EF
:1061B0008A81828713868B81848715868C81868766
:1061C00017868D81808B118A8E81828B138A0E9423
:1061D000E4174DB75EB74C5E5F4F4DBF5EBF26966E
:1061E000CDBFDEBFCF91DF911F910F910895CF9268
:1061F000DF92EF92FF920F931F93DF93CF930F9253
:106200000F92CDB7DEB76C0162307105E4F1DA01AF
:1062100012968D919C911397BE016F5F7F4F0E94E4
:106220000723009781F189810E9427138C0197FD34
:1062300005C05EE2E52E52E2F52E04C041E3E42EF5
:1062400042E2F42EC8010E946D1DEDB7FEB73A97E9
:10625000EDBFFEBF3196ADB7BEB71196CD92DC92C1
:10626000129725E332E222833383E482F5820683A8
:106270001783808791870E94E417EDB7FEB73A969F
:10628000EDBFFEBF14C000D00F92ADB7BEB71196E0
:10629000CD92DC92129785EF97E213968D939C93A3
:1062A00014970E94E4170F900F900F900F900F908B
:1062B0000F90CF91DF911F910F91FF90EF90DF90A2
:1062C000CF900895AF92BF92CF92DF92EF92FF925C
:1062D0000F931F93DF93CF93CDB7DEB76097CDBFFA
:1062E000DEBF5C018A016630710509F0AFC0DA01DA
:1062F00012968D919C911397BE016F5F7F4F0E9404
:106300000723009709F4A2C0F80184819581BE019A
:106310006B5F7F4F0E9465226115710581059105B4
:1063200009F494C0D80116968D919C911797BE01DF
:10633000675F7F4F0E946522611571058105910598
:1063400009F484C0F80180859185BE016D5F7F4F9F
:106350000E940723009709F479C0D8011A968D91FD
:106360009C911B97BE01635F7F4F0E946522611560
:1063700071058105910509F469C0EDB7FEB73E9737
:10638000EDBFFEBF3196ADB7BEB71196AD92BC92D0
:10639000129784E198E28283938389819A8184832E
:1063A00095838D819E818683978389859A85808751
:1063B00091878B819C81828793878D859E85848739
:1063C00095870E94E417EDB7FEB73E96EDBFFEBF7E
:1063D0004D815E816F81788509851A852B853C8585
:1063E000CD84DE848981EB800E944B138C0197FD64
:1063F00005C07EE2E72E72E2F72E04C061E3E62ECE
:1064000062E2F62EC8010E946D1D2DB73EB72A50DC
:1064100030402DBF3EBFEDB7FEB73196ADB7BEB72A
:106420001196AD92BC92129725E332E22283338318
:10643000E482F58206831783808791870E94E417A0
:10644000EDB7FEB73A96EDBFFEBF1EC000D00F926B
:10645000ADB7BEB71196AD92BC92129785E298E2A5
:1064600013968D939C9314970E94E417EDB7FEB793
:10647000A182B28289E598E2838394830E94E41723
:106480000F900F900F900F906096CDBFDEBFCF9111
:10649000DF911F910F91FF90EF90DF90CF90BF9011
:1064A000AF900895CF92DF92EF92FF920F931F93D8
:1064B000DF93CF930F920F92CDB7DEB76C016230AE
:1064C0007105ECF1DA0112968D919C911397BE0142
:1064D0006F5F7F4F0E940723009789F189819A811E
:1064E0000E9437138C0197FD05C0FEE2EF2EF2E209
:1064F000FF2E04C0E1E3EE2EE2E2FE2EC8010E9470
:106500006D1DEDB7FEB73A97EDBFFEBF3196ADB743
:10651000BEB71196CD92DC92129725E332E2228328
:106520003383E482F58206831783808791870E94F4
:10653000E417EDB7FEB73A96EDBFFEBF14C000D02A
:106540000F92ADB7BEB71196CD92DC92129785E946
:1065500098E213968D939C9314970E94E4170F90E2
:106560000F900F900F900F900F90CF91DF911F9190
:106570000F91FF90EF90DF90CF9008950F931F93AE
:10658000DF93CF930F92CDB7DEB78C01CE0101968A
:106590000E940813E981E43040F4F0E0EE0FFF1FA1
:1065A000ED54FD4C2081318102C020E030E097FFA6
:1065B00005C041E352E229E737E202C04EE252E26F
:1065C0006DB77EB76A5070406DBF7EBFEDB7FEB746
:1065D0003196ADB7BEB711960D931C93129765E334
:1065E00072E2628373834483558386839783208713
:1065F00031870E94E4176DB77EB7665F7F4F6DBF2E
:106600007EBF0F90CF91DF911F910F910895EF9270
:10661000FF920F931F93CF93DF938C01EA016230B7
:1066200071050CF459C08A819B816BEA78E20E9463
:106630008D160097D1F08A819B816FEA78E20E94E3
:106640008D160097A1F08A819B8162EB78E20E940F
:106650008D16009771F08A819B8168EB78E20E9429
:106660008D160097C9F583E005C080E003C081E086
:1066700001C082E00E94F812EC0197FD05C08EE295
:10668000E82E82E2F82E04C0B1E3EB2EB2E2FB2E3C
:10669000CE010E946D1D2DB73EB72A5030402DBF50
:1066A0003EBFEDB7FEB73196ADB7BEB711960D93AD
:1066B0001C93129725E332E222833383E482F5822E
:1066C000C683D783808791870E94E417EDB7FEB712
:1066D0003A96EDBFFEBF14C000D00F92ADB7BEB763
:1066E00011960D931C9312978CEB98E213968D9351
:1066F0009C9314970E94E4170F900F900F900F90A7
:10670000DF91CF911F910F91FF90EF900895EF923D
:10671000FF920F931F93CF93DF937C010E94620C33
:10672000EC0197FD03C00EE212E202C001E312E2A7
:10673000CE010E946D1D2DB73EB72A5030402DBFAF
:106740003EBFEDB7FEB73196ADB7BEB71196ED922D
:10675000FC92129725E332E222833383048315836C
:10676000C683D783808791870E94E4172DB73EB7F1
:10677000265F3F4F2DBF3EBFDF91CF911F910F91FD
:10678000FF90EF900895AF92BF92CF92DF92EF9279
:10679000FF920F931F93DF93CF93CDB7DEB7A197EF
:1067A000CDBFDEBF5C016B018A017E010894E11C54
:1067B000F11CC70160E070E041E250E00E947816F1
:1067C00024E0C216D104A4F1D80112968D919C91B7
:1067D0001397B7010E94F81F009709F487C0F801CA
:1067E000E680F780C7016DED78E20E948D16009774
:1067F00091F0C70162EE78E20E948D16009771F069
:10680000C70166EE78E20E948D16009709F06EC00F
:1068100041E050E005C043E050E002C042E050E0FB
:10682000D80114966D917C911597CE0101962CC0DC
:10683000B3E0CB16D10481F4F80182819381B701D2
:106840000E94F81F009709F451C0D80114966D9169
:106850007C911597C70116C0B2E0CB16D10451F454
:10686000F80182819381B7010E94F81F0097F1F12E
:10687000C70106C0F1E0CF16D104C1F580E090E079
:1068800060E070E040E050E00E94060C8C0197FD53
:1068900005C02EE2E22E22E2F22E04C091E3E92EA0
:1068A00092E2F92EC8010E946D1D2DB73EB72A5005
:1068B00030402DBF3EBFEDB7FEB73196ADB7BEB786
:1068C0001196AD92BC92129725E332E22283338374
:1068D000E482F58206831783808791870E94E417FC
:1068E000EDB7FEB73A96EDBFFEBF14C000D00F92D1
:1068F000ADB7BEB71196AD92BC9212978AEE98E2F0
:1069000013968D939C9314970E94E4170F900F9009
:106910000F900F90A196CDBFDEBFCF91DF911F9159
:106920000F91FF90EF90DF90CF90BF90AF900895C0
:106930008F929F92AF92BF92CF92DF92EF92FF928F
:106940000F931F93DF93CF9300D000D0CDB7DEB766
:106950004C016A011B821C821D821E8219821A82CE
:1069600063307105DCF0DA0112968D919C911397DA
:10697000BE016D5F7F4F0E94652261157105810523
:10698000910509F469C0F60184819581BE016F5FAC
:106990007F4F0E9407230097A9F45EC06230710503
:1069A00009F05AC0DA0112968D919C911397BE019D
:1069B0006D5F7F4F0E94652261157105810591050C
:1069C00009F44AC06B817C818D819E8149810E943E
:1069D000E30A5C010097D1F48AEF90E00E94294914
:1069E0004B815C816D817E81C980DA8080911C330E
:1069F00090911D3328E030E000E010E0E1E0EE2E61
:106A0000F12C0E94974797FF03C03BC097FD03C03E
:106A10000EE212E202C001E312E2C5010E946D1D06
:106A2000EDB7FEB73A97EDBFFEBF3196ADB7BEB733
:106A300011968D929C92129725E332E22283338342
:106A400004831583A682B782808791870E94E4170A
:106A5000EDB7FEB73A962BC000D00F92ADB7BEB7D8
:106A600011968D929C92129786E199E213968D93DE
:106A70009C9314970E94E4170F900F900F900F9023
:106A800018C000D000D0EDB7FEB73196ADB7BEB795
:106A900011968D929C92129720E439E222833383DF
:106AA000848395830E94E417EDB7FEB73696EDBF59
:106AB000FEBF2696CDBFDEBFCF91DF911F910F9114
:106AC000FF90EF90DF90CF90BF90AF909F908F900E
:106AD0000895EF92FF920F931F93CF93DF937C0162
:106AE0000E940B0BEC0197FD03C00EE212E202C004
:106AF00001E312E2CE010E946D1D2DB73EB72A5070
:106B000030402DBF3EBFEDB7FEB73196ADB7BEB733
:106B10001196ED92FC92129725E332E222833383A1
:106B200004831583C683D783808791870E94E417E7
:106B30002DB73EB7265F3F4F2DBF3EBFDF91CF91B0
:106B40001F910F91FF90EF900895CF93DF93EC0189
:106B500088819981009721F00E94D40E18821982B1
:106B6000DF91CF9108950F931F93CF93DF938C0103
:106B7000FC0182819381009721F0C80102960E9456
:106B8000A535F801808191810E94820EEC0197FD6C
:106B90000EC06CED75E3A8010E94970DCE0165EF64
:106BA00075E3A8010E94B10DF801C283D383DF9180
:106BB000CF911F910F910895DF93CF9300D00F9243
:106BC000CDB7DEB74115510539F0CB01BE016F5F7E
:106BD0007F4F0E94B41003C002960E94A5352496F0
:106BE000CDBFDEBFCF91DF910895AF92BF92CF921C
:106BF000DF92EF92FF920F931F93CF93DF935B018E
:106C00006A01E82EE7017E01F92EE70141155105E1
:106C100009F453C086E0E82EF12CEC0EFD1ECB01EA
:106C2000B70140E850E00E942F0F8C01A601481BDD
:106C3000590BC50160E070E00E942F0F17FD41C0A5
:106C40008A819B810097E9F1FE01E00FF11F158217
:106C5000C7016BE67DE20E94CD16009791F1C70156
:106C60006EE67DE244E050E00E948A16009729F526
:106C7000FE013A96CF0121912C30E1F32A30D1F375
:106C80002D30C1F32930B1F32B30A1F3203291F331
:106C9000E82FF92FDF0121912C3051F02A3041F0FB
:106CA0002D3031F0293021F02B3011F0203291F7C6
:106CB0001C926A817B810E94C943CE0102960E9488
:106CC000A535DF91CF911F910F91FF90EF90DF904D
:106CD000CF90BF90AF900895CF92DF92EF92FF9246
:106CE0000F931F93CF93DF937C0186E890E00E947F
:106CF0004D16C82EE6016E01D92EE60186012097B9
:106D000039F180E090E060E070E00E94400D8883FF
:106D1000998397FD12C06FE772E3A7010E94CB0D24
:106D2000009759F48881998161E070E043EB55E365
:106D300096010E94FE0D009759F088819981009775
:106D400011F00E94D40ECE010E94721600E010E0F5
:106D5000C801DF91CF911F910F91FF90EF90DF90CD
:106D6000CF900895CF93DF93EC0102960E94A53552
:106D700088819981009711F00E94D40ECE010E9463
:106D80007216DF91CF910895EF92FF920F931F93A8
:106D9000CF93DF938C01CB01EA0179010E94E915C1
:106DA00000D000D0EDB7FEB73196ADB7BEB71196A3
:106DB0000C93118323E73DE22283338384839583FD
:106DC0000E94E4170F920F92EDB7FEB73196ADB760
:106DD000BEB711960C93118380E99DE28283938361
:106DE000C483D583E682F7820E94E4178DB79EB7ED
:106DF00008968DBF9EBFDF91CF911F910F91FF909D
:106E0000EF900895CF92DF92EF92FF920F931F932E
:106E1000CF93DF93D82EC92E7B01CA01E90101155A
:106E20001105A1F40E94E9152DB73EB72A50304054
:106E30002DBF3EBFEDB7FEB73196ADB7BEB71196C9
:106E4000DC921197C18226EB3DE212C0033011059E
:106E5000F1F40E94E915ADB7BEB71A97ADBFBEBF3A
:106E6000EDB7FEB731961196DC92C18226ED3DE278
:106E700022833383E482F58286839783C087D18718
:106E80000E94E4172DB73EB7265F3F4F1FC00E94F8
:106E9000E915ADB7BEB71C97ADBFBEBFEDB7FEB726
:106EA00031961196DC92C18223E13EE22283338344
:106EB000E482F58286839783C087D1870287138710
:106EC0000E94E4172DB73EB7245F3F4F2DBF3EBF52
:106ED000DF91CF911F910F91FF90EF90DF90CF90B6
:106EE0000895CF93DF93EC01888D998D18161906BC
:106EF00014F40E94D40E8A8D9B8D009711F00E948D
:106F0000E11D8C819D810E947216CE010E94721635
:106F1000DF91CF910895CF92DF92EF92FF920F937E
:106F20001F93CF93DF93E62EE7017E01F72EE70153
:106F30000C811D81288939898A899B8928173907FD
:106F400081F4EA85FB85309741F04C895D892E8973
:106F50003F898C859D85B7011995CE010E947137B7
:106F60007DC0EE80FF80E8E0F0E0EE0EFF1E88E0DE
:106F7000F80180831182128213828E859F850E9480
:106F80003414F80184839583888999890E94341484
:106F9000F80186839783B70180E090E0DC010FC0A1
:106FA000D080CC24218130E02C293D29329640E04C
:106FB00050E0820F931FA41FB51F625070406230D3
:106FC000710570F7970136952795F901EE0FFF1FB0
:106FD000E00FF11F220F331FE216F30641F030815C
:106FE00020E040E050E0820F931FA41FB51F9D01D9
:106FF00044275527A070B070820F931FA41FB51FA0
:10700000A0FF09C09D0144275527A070B070820FD2
:10701000931FA41FB51F0E94341480959095F8010A
:1070200082839383888D998DB801A7019E0100E02A
:1070300010E00E943B108E159F0529F48C899D89D4
:1070400001968C8B9D8B8A8D9B8D68EE73E00E94E0
:10705000251E888999890196888B998BDF91CF911C
:107060001F910F91FF90EF90DF90CF9008958F9236
:107070009F92AF92BF92CF92DF92EF92FF920F93C7
:107080001F93CF93DF93C82EA92E7B018A01CA01DB
:107090000E944A16882EE4014E01992EE4012097A1
:1070A000C9F1C701B401A8010E942F0F7C0180170C
:1070B000910781F58C31910568F10C2D1A2D74E141
:1070C000C72ED12CC80CD91CF601848195810E9451
:1070D0003814F8012685378582179307D9F48689F5
:1070E00097890196868B978B808491848114910473
:1070F00089F0A484B584F601868197810E943814B2
:107100009C01AE01445F5F4F0C89C501B70110E0DF
:10711000F4011995CE010E947216DF91CF911F9153
:107120000F91FF90EF90DF90CF90BF90AF909F9026
:107130008F9008952F923F924F925F926F927F921D
:107140008F929F92AF92BF92CF92DF92EF92FF9277
:107150000F931F93DF93CF930F920F92CDB7DEB7AC
:107160005C013B01490168018CE190E049835A834D
:107170000E944D161C0149815A81009709F442C0B2
:107180008A01C80108960E944D16F10184839583F7
:107190000097A9F182E090E061E070E00E94400D6C
:1071A000F101808F918F181619064CF567E378E38B
:1071B000A1010E94B10DF50180819181A281B3816D
:1071C000F10180839183A283B383628A738A0683E9
:1071D00017831686178680869186C286D386E486B4
:1071E000F58680E090E060E070E04BE857E39101C5
:1071F0000E94931DF101828F938F009731F4C1019A
:107200000E9471372DEF3FEF02C020E030E0C9014E
:107210000F900F90CF91DF911F910F91FF90EF9002
:10722000DF90CF90BF90AF909F908F907F906F90A6
:107230005F904F903F902F9008952F923F924F92E2
:107240005F926F927F928F929F92AF92BF92CF92F6
:10725000DF92EF92FF920F931F93DF93CF9300D0B3
:107260000F92CDB7DEB72C015B016A0180917F32AE
:1072700090918032A0918132B091823289839A8339
:10728000AB83BC8331E0E32EF12C20E2622E712C23
:1072900093E0892E912C1E010894211C311C47C0BB
:1072A0008701000F111F0C0D1D1DD8018D919C91A0
:1072B00062E47EE20E948D16009791F40894E11C2E
:1072C000F11CEA14FB040CF076C0F701EE0FFF1F6F
:1072D000EC0DFD1D808191810E941B574C0124C043
:1072E000F8018081918165E47EE20E948D1600970D
:1072F00091F40894E11CF11CEA14FB040CF05BC04F
:10730000F701EE0FFF1FEC0DFD1D808191810E94A2
:107310001B573C0109C0D8018D919C91B1010E947D
:107320007A14009709F447C00894E11CF11CEA1490
:10733000FB040CF4B5CF89819A81AB81BC810097A5
:10734000A105B105C1F1CE010196B401A30122E06E
:1073500037E304EC16E372010E949A388C0197FD22
:1073600005C0FBE3EF2EFEE2FF2E04C0EEE3EE2E9F
:10737000EEE2FE2EC8010E946D1DEDB7FEB73A97F2
:10738000EDBFFEBF3196ADB7BEB711964D925C9280
:10739000129728E43EE222833383E482F582068357
:1073A0001783808791870E94E417EDB7FEB73A965E
:1073B000EDBFFEBF14C000D00F92ADB7BEB711969F
:1073C0004D925C92129785E59EE213968D939C9365
:1073D00014970E94E4170F900F900F900F9024962F
:1073E000CDBFDEBFCF91DF911F910F91FF90EF9046
:1073F000DF90CF90BF90AF909F908F907F906F90D5
:107400005F904F903F902F900895AF92BF92CF9290
:10741000DF92EF92FF920F931F93CF93DF93B82EDB
:10742000A92EEB016A017801890100D00F92EDB716
:10743000FEB73196ADB7BEB711968C93918386E8AF
:107440009EE2828393830E94E4170F900F900F9027
:107450000F902097E1F0CE010E946D1DEDB7FEB7B1
:107460003897EDBFFEBF3196ADB7BEB71196BC924F
:10747000A18229E83EE222833383C483D5838683B5
:1074800097830E94E417EDB7FEB7389645C0E11424
:10749000F1040105110559F12DB73EB72E503040CA
:1074A0002DBF3EBFCDB7DEB72196ADB7BEB71196A3
:1074B000BC92A9828CE99EE28A839B83CC82DD8286
:1074C000EE82FF8208871987B601882777FD8095AD
:1074D000982FA80197010E9491532A873B874C87D8
:1074E0005D870E94E417EDB7FEB73E9615C000D049
:1074F00000D0EDB7FEB73196ADB7BEB71196BC92CE
:10750000A1828EEC9EE282839383C482D5820E9404
:10751000E417EDB7FEB73696EDBFFEBFDF91CF9112
:107520001F910F91FF90EF90DF90CF90BF90AF90A1
:1075300008950F931F93CF93DF938C01EB0100D03D
:107540000F92EDB7FEB73196ADB7BEB711968C93DB
:10755000118384EF9EE2828393830E94E4170F904D
:107560000F900F900F901C161D06DCF4CE0160E505
:1075700070E00E947E530097A1F400D00F92EDB707
:10758000FEB73196ADB7BEB711960C93118386E85E
:107590009EE2828393830E94E4170F900F900F90D6
:1075A0000F90DF91CF911F910F910895AF92BF92ED
:1075B000CF92DF92EF92FF920F931F93CF93DF93BF
:1075C000EC01B62EA72E88899989009761F02C814D
:1075D0003D818E819F81289F6001299FD00C389F1B
:1075E000D00C112404C0CA88DB88EC88FD886C8527
:1075F0007D85888599850E94031FEA8DFB8D3097D4
:1076000049F08C0120E030E08C8D9D8D6B2D7A2D22
:10761000A60119958A819B810E94721688819981A1
:107620000E94D40E88899989009721F48E899F89B8
:107630000E94D40ECE010E9472168B2D9A2DDF91DE
:10764000CF911F910F91FF90EF90DF90CF90BF905F
:10765000AF900895EF92FF92CF93DF93E82EE7016A
:107660007E01F92EE701CB010E94820EBC018E8BB8
:107670009F8B97FF04C0C7010E94D63A14C065EAE9
:107680007BE3A7010E94970D8E899F8968E57BE3C4
:10769000A7010E94B10D0E94381EA0E0B0E08887CB
:1076A0009987AA87BB87DF91CF91FF90EF900895CC
:1076B000EF92FF92CF93DF939B01E82EE7017E01CB
:1076C000F92EE701888999890097D1F5411551056F
:1076D00061F40E94381EA0E0B0E08C879D87AE87E1
:1076E000BF87C70160E070E00BC06A817B814C817D
:1076F0005D81C9010E942F0FBC0197FF04C0C70123
:107700000E94D63A1DC0AE81BF811196AE83BF8361
:10771000882777FD8095982F2A893B894C895D8938
:10772000260F371F481F591F2A8B3B8B4C8B5D8BB5
:10773000E88DF98D309721F08C8D9D8DBD011995C7
:10774000DF91CF91FF90EF900895EF92FF920F930A
:107750001F93CF93DF93E82EE7017E01F92EE70117
:107760004115510521F4C7016CEF7FEF3CC00E9429
:10777000381EA0E0B0E088879987AA87BB87EE24EF
:10778000FF241EC06A817B81600F711F401B510B5B
:10779000888199810E94D70FBC0197FD08C0080F0E
:1077A000191F4C815D810417150760F325C0CE01B8
:1077B0001AC08C8D9D8DB70119950894E11CF11CA0
:1077C0008E819F81E816F90618F400E010E0E9CFF9
:1077D0000E94381EA0E0B0E08C879D87AE87BF87EF
:1077E000CE0160E070E00E94D63ADF91CF911F9108
:1077F0000F91FF90EF900895E88DF98D3097C9F6BD
:10780000DCCF2F923F924F925F926F927F928F9236
:107810009F92AF92BF92CF92DF92EF92FF920F931F
:107820001F93CF93DF932C013B014A01590141156E
:10783000510509F455C02115310509F451C06115F0
:10784000710509F44DC08EE190E00E944D16282E7E
:10785000E1011E01392EE101209709F444C08E8216
:107860009F82AC82BD82088F198FEA8EFB8ECC8EF0
:10787000DD8E81E090E0888B998BC5010E944A16CD
:107880008A839B83009721F4C1016DEF7FEF0CC0C9
:1078900080E090E060E070E00E94400DBC018883D1
:1078A000998397FF05C0CE010E94D63A9C011DC066
:1078B000B201A3010E943C0EBC0197FDF4CF888168
:1078C000998165EA7BE3A1010E94970D88819981E6
:1078D00068E57BE3A1010E94B10D2881398105C0D3
:1078E0002EEF3FEF02C02DEF3FEFC901DF91CF91A7
:1078F0001F910F91FF90EF90DF90CF90BF90AF90CE
:107900009F908F907F906F905F904F903F902F90BF
:1079100008956F927F928F929F92AF92BF92CF9273
:10792000DF92EF92FF920F931F93CF93DF934C015F
:107930007B015A0169018EE190E00E944D16682E8C
:10794000E3013E01792EE301209719F480E090E0F5
:1079500010C0EC82FD82A88EB98ECA8EDB8E0C8F91
:107960001D8FC7010E944A168A839B83009731F4BA
:10797000C3016DEF7FEF0E94D63A23C080E090E014
:1079800060E070E00E94400DBC018883998397FD00
:1079900014C06FE772E3A4010E94CB0DBC0197FDF8
:1079A0000CC08881998161E070E04AE25BE3930159
:1079B0000E94FE0DBC0197FF02C0CE01DCCF888182
:1079C0009981DF91CF911F910F91FF90EF90DF9000
:1079D000CF90BF90AF909F908F907F906F900895C1
:1079E0002F923F924F925F926F927F928F929F92CF
:1079F000AF92BF92CF92DF92EF92FF920F931F93BD
:107A0000DF93CF9300D000D0CDB7DEB75C014B0140
:107A10006A0180917F3290918032A0918132B09141
:107A2000823289839A83AB83BC8322243324412C02
:107A300034E0532E20E034E02D833E8328E8622E8C
:107A400023E1722E91E0E92EF12C81C08701000F15
:107A5000111F0C0D1D1DD8018D919C9166EF7EE2CA
:107A60000E948D16009799F40894E11CF11CE8140B
:107A7000F9040CF002C1F701EE0FFF1FEC0DFD1D24
:107A8000808191810E941B57682E792E5DC0F8017C
:107A90008081918169EF7EE20E948D160097A9F4A2
:107AA0000894E11CF11CE814F9040CF0E6C0F7019D
:107AB000EE0FFF1FEC0DFD1D808191810E941B5771
:107AC000282F392F2D833E833FC0D8018D919C9163
:107AD0006CEF7EE20E948D16009799F40894E11CE9
:107AE000F11CE814F9040CF0C8C0F701EE0FFF1FF9
:107AF000EC0DFD1D808191810E941B57482E592E4F
:107B000023C0F801808191816FEF7EE20E948D1683
:107B10000097A1F0D8018D919C9162E07FE20E94D4
:107B20008D16009779F0F80180819181BE016F5F19
:107B30007F4F0E947A14009739F49FC0F1E02F2EF6
:107B4000312C02C0222433240894E11CF11CE814D7
:107B5000F9040CF47BCF21143104C9F089819A8196
:107B6000AB81BC810097A105B10509F486C0CE01A7
:107B70000196B3014D815E81920109E91AE3E5E0C6
:107B8000EE2EEAE3FE2E65010E94013C09C0C3010E
:107B9000B20149E95AE325E03AE385010E94893CB4
:107BA0008C0197FF1EC00E946D1D2DB73EB72A5055
:107BB00030402DBF3EBFEDB7FEB73196ADB7BEB773
:107BC0001196AD92BC92129725E03FE22283338357
:107BD00022E13FE2248335830683178380879187E0
:107BE00044C02114310459F1CE0101960E94E915D7
:107BF0002DB73EB72E5030402DBF3EBFEDB7FEB77C
:107C00003196ADB7BEB71196AD92BC92129726E1F0
:107C10003FE22283338384839583668277822D813A
:107C20003E812087318742865386048715870E94CC
:107C3000E4178DB79EB70E968DBF9EBF32C0ADB70D
:107C4000BEB71A97ADBFBEBFEDB7FEB7319611965E
:107C5000AD92BC92129787E49FE282839383648201
:107C6000758246825782008711870E94E417EDB71C
:107C7000FEB73A96EDBFFEBF14C000D00F92ADB76D
:107C8000BEB71196AD92BC92129782E79FE213960F
:107C90008D939C9314970E94E4170F900F900F9070
:107CA0000F902696CDBFDEBFCF91DF911F910F9130
:107CB000FF90EF90DF90CF90BF90AF909F908F900C
:107CC0007F906F905F904F903F902F9008950F930B
:107CD0001F93CF93DF938C01FB01EA01309709F5E5
:107CE000CA010E946D1D2DB73EB7285030402DBFF0
:107CF0003EBFEDB7FEB73196ADB7BEB711960C9348
:107D0000118323EA3FE22283338384839583C683EE
:107D1000D7830E94E417CDB7DEB72896CDBFDEBF6C
:107D200047C02DB73EB7205130402DBF3EBFADB745
:107D3000BEB71196CDB7DEB7898311961C93119704
:107D400083EC9FE212968D939C9313978581968185
:107D50008459984F14968D939C931597848190E045
:107D6000019616968D939C931797838118968C9302
:107D7000189719961C92199782811A968C931A97C4
:107D80001B961C921B9781811C968C931C971D96A9
:107D90001C921D9780811E968C931E971F961C9295
:107DA0000E94E4172DB73EB7205F3F4F2DBF3EBF67
:107DB000DF91CF911F910F910895CF93DF93EC0145
:107DC0008C819D811816190614F40E94D40E8E81A0
:107DD0009F81009711F00E94E11DCE010E94721652
:107DE000DF91CF910895EF92FF92CF93DF93E62E2C
:107DF000E7017E01F72EE701E881F981309739F03C
:107E00008A819B8160E070E04FEE5FEF1995CE01B3
:107E10000E94DD3EDF91CF91FF90EF9008956F9229
:107E20007F928F929F92AF92BF92CF92DF92EF920A
:107E3000FF920F931F93DF93CF93CDB7DEB7E097F9
:107E4000CDBFDEBF3C018B014A015E010894A11C3D
:107E5000B11CC50160E070E040E350E00E9478167C
:107E600083E2898388E090E00E944D167C010097B0
:107E700009F441C081E090E060E070E00E94400DB4
:107E80006C01181619067CF5F701008311838282B4
:107E900093828483958388E893E160E070E043EF08
:107EA0005EE397010E94931DF701868397830097F5
:107EB000D1F0C601B3014BE750E00E943C0E8C01AB
:107EC0000097A9F4C6016BE072E4A7010E94B10D0E
:107ED00097FD0CC0C601B50140E350E00E94D70FEA
:107EE00097FF0BC003C00DEF1FEF01C08C01C7014E
:107EF0000E94DD3E02C00DEF1FEFC801E096CDBF2E
:107F0000DEBFCF91DF911F910F91FF90EF90DF9037
:107F1000CF90BF90AF909F908F907F906F9008957B
:107F2000CF92DF92EF92FF920F931F93DF93CF9345
:107F300000D00F92CDB7DEB76C01623071050CF442
:107F400040C0DA0112968D919C9113978E010F5FBC
:107F50001F4FB8010E947A14009799F1C80167E693
:107F60007EE3A6010E940F3F8C0197FD05C09DEEA8
:107F7000E92E9FE2F92E04C080EFE82E8FE2F82E62
:107F8000C8010E946D1DEDB7FEB73A97EDBFFEBF69
:107F90003196ADB7BEB71196CD92DC92129724EF11
:107FA0003FE222833383E482F5820683178380874E
:107FB00091870E94E417EDB7FEB73A96EDBFFEBF7A
:107FC00014C000D00F92ADB7BEB71196CD92DC921F
:107FD000129781E090E313968D939C9314970E94DF
:107FE000E4170F900F900F900F902496CDBFDEBF37
:107FF000CF91DF911F910F91FF90EF90DF90CF9085
:1080000008952F923F924F925F926F927F928F923C
:108010009F92AF92BF92CF92DF92EF92FF920F9317
:108020001F93DF93CF93CDB7DEB7C254D040CDBFFF
:10803000DEBF6DAB7EABDE011196EBEBF2E324E32A
:1080400001900D922150E1F7DC016D917D918D91B0
:108050009C9120E831E541E050E00E949153790184
:108060008A0120E13EE040E050E00E94B353EDA9D8
:10807000FEA922832CE330E040E050E00E94B3539D
:10808000ADA9BEA911962C9311976C93C801B701A5
:108090006C5F7F4F8F4F9F4F27E030E040E050E014
:1080A0000E94B353EDA9FEA96187A2EBAA2EA7E017
:1080B000BA2EC12CD12CFEC0C801B7012DE631E08B
:1080C00040E050E00E94B353662797FD6395772701
:1080D0008827992739014A01661A770A880A990A76
:1080E0006A0C7B1C8C1C9D1C6FAA78AE89AE9AAE64
:1080F00035014601089461087108810891082FA88C
:1081000038AC49AC5AAC08942108310841085108F0
:10811000C401B30124E030E040E050E00E94B353DA
:108120002BAF3CAF4DAF5EAF23966CAF7DAF8EAF44
:108130009FAF2397C401B3012CE93FEF4FEF5FEFEF
:108140000E94B3538BAD9CADADADBEAD280F391FB2
:108150004A1F5B1FE20EF31E041F151FC401B3016B
:1081600020E931E040E050E00E94B3536BAF7CAFB8
:108170008DAF9EAFE20EF31E041F151FC401B301A5
:1081800024E630E040E050E00E94B353662797FDBC
:108190006395772788279927E60EF71E081F191F72
:1081A0008BAD9CADADADBEAD8827B7FD839599274E
:1081B000AA27BB27E81AF90A0A0B1B0B23968CADDA
:1081C0009DADAEADBFAD23978827B7FD83959927A9
:1081D000AA27BB27E81AF90A0A0B1B0BC201B10137
:1081E00020E73EEF4FEF5FEF0E94B353E20EF31E26
:1081F000041F151FC201B10124E630E040E050E049
:108200000E94B3536BAF7CAF8DAF9EAFE20EF31EF7
:10821000041F151FC201B10124E030E040E050E02E
:108220000E94B3533B014C01E21AF30A040B150BF5
:10823000C201B10120E931E040E050E00E94B353B7
:10824000662797FD6395772788279927E60EF71EFF
:10825000081F191FD401C3018827B7FD83959927EB
:10826000AA27BB27E80EF91E0A1F1B1FC601B5016E
:108270006FA878AC89AC9AAC661977098809990916
:108280002DE631E040E050E00E945353E60EF71E29
:10829000081F191F8BAD9CADADADBEAD8827B7FDD6
:1082A00083959927AA27BB27E81AF90A0A0B1B0B03
:1082B0006401530117FD00CF23E0622E712C812C45
:1082C000912C6A207B208C209D20611471048104F4
:1082D0009104D1F4C601B50124E630E040E050E05D
:1082E0000E94B353611571058105910591F4C60192
:1082F000B50120E931E040E050E00E94B353611540
:1083000071058105910529F08DE691E0A0E0B0E0CE
:1083100004C08EE691E0A0E0B0E0E816F9060A0796
:108320001B070CF0C9CEC5018C569740ADA9BEA95C
:1083300015968D939C9316971796ED92FC9218972D
:10834000611471048104910401F5C601B50124E6AC
:1083500030E040E050E00E94B353611571058105A3
:108360009105B1F4C601B50120E931E040E050E0EB
:108370000E94B35321E030E061157105810591053C
:1083800011F020E030E0C90105C080E090E002C0BB
:1083900081E090E02AE130E0829FF001839FF00DC0
:1083A000929FF00D1124CE010196E80FF91F7896E7
:1083B0008BE090E0A0E0B0E003C00197A109B10913
:1083C0003291229140E050E0E216F30604071507CF
:1083D000A4F3EDA9FEA98483E21AF30A040B150B9A
:1083E000E394E38281E090E0CE5BDF4FCDBFDEBF60
:1083F000CF91DF911F910F91FF90EF90DF90CF9081
:10840000BF90AF909F908F907F906F905F904F90B4
:108410003F902F900895AF92BF92CF92DF92EF924C
:10842000FF920F931F93DF93CF93CDB7DEB7609783
:10843000CDBFDEBF5B017A016C014033510580F195
:10844000CA010E944A16082F192F0115110569F15A
:10845000C501B801A7010E942F0FAC018E159F0521
:1084600031F5D80190966D917D918D919C91939766
:108470004F87588B0E94771460587E478A4A9348EA
:1084800069837A838B839C83F894CE010196BE0125
:108490006B5F7F4F0E94014078944F85588907C0D9
:1084A00040EF5FEF00E010E002C04DEF5FEFD6015C
:1084B000ED91FC911197309741F012968D919C911E
:1084C0001397BE016B5F7F4F1995C8010E9472160A
:1084D000C6010E94DD3E6096CDBFDEBFCF91DF9129
:1084E0001F910F91FF90EF90DF90CF90BF90AF90D2
:1084F0000895CF92DF92EF92FF920F931F93CF9345
:10850000DF936C018B01CB010E947E167C01C0E0E1
:10851000D0E00EC0B8016C0F7D1FA7014C1B5D0B96
:10852000C6010E94D70F9C0197FD07C0C80FD91F35
:10853000CE15DF057CF320E030E0C901DF91CF915B
:108540001F910F91FF90EF90DF90CF9008958F9241
:108550009F92AF92BF92CF92DF92EF92FF920F93D2
:108560001F93CF93DF934C015B016A0180E490E09D
:108570000E944A167C01C0E0D0E01DC086010C1BA1
:108580001D0B0134110514F000E410E0B5016C0F6F
:108590007D1FC701A8010E944157C401B701A8016E
:1085A0000E94D70F8C0197FF04C0C7010E9472166A
:1085B0000AC0C80FD91FCC15DD0504F3C7010E94FE
:1085C000721600E010E0C801DF91CF911F910F916A
:1085D000FF90EF90DF90CF90BF90AF909F908F90E3
:1085E00008950F931F93CF93DF93EC018B01CB0181
:1085F0000E944A57AC01CE01B8010E94A742DF9108
:10860000CF911F910F910895EF92FF920F931F93B7
:10861000DF93CF93CDB7DEB76C97CDBFDEBF7C01C4
:108620008EE49FE2A1E4B0E08B879C87AD87BE8794
:10863000FE013F968EE0DF011D928A95E9F7E11475
:10864000F10409F499C0C7016FE176E00E94F1429C
:108650009C0197FD93C08E010F5F1F4FC80160E022
:1086600070E040E050E020E030E00E94790C00979C
:1086700029F4C8010E94E9158C0102C008E310E347
:10868000C7016AE076E00E94F1429C0197FD76C046
:10869000C701B8010E9479429C0197FD6FC0C701D4
:1086A0006FEE75E00E94F1429C0197FD67C0CE011C
:1086B00005960E94D30C009789F58DB79EB7429717
:1086C0008DBF9EBFEDB7FEB73196CE010B96ADB70D
:1086D000BEB711968D939C93129782E190E08283AE
:1086E00093838CE390E3848395838D8186831782C3
:1086F0008E81808711868F81828713868885848703
:1087000015868985868717868A85808B118A0E94BF
:1087100021588DB79EB742968DBF9EBFC70169EDA8
:1087200075E00E94F1429C0197FD28C0C701BE017F
:10873000655F7F4F0E9479429C0197FD1FC0C70172
:108740006EEB75E00E94F1429C0197FD17C0C701D6
:1087500069E973E00E94F1429C0197FD0FC0C701D7
:1087600064EF71E00E94F142282F392F1216130690
:108770002CF420E030E002C02FEF3FEFC9016C96EF
:10878000CDBFDEBFCF91DF911F910F91FF90EF9092
:108790000895EF92FF920F931F93DF93CF930F9261
:1087A0000F92CDB7DEB77C018B016AE570E30E94C2
:1087B0008D16009709F471C0C7016CE570E30E9443
:1087C0008D16009709F469C0C7016FE570E34CE0AE
:1087D00050E00E948A16009709F058C000D000D0DF
:1087E000EDB7FEB73196C7010C96ADB7BEB711967F
:1087F0008D939C9312978CE690E382839383CE01B2
:108800000196848395830E9459582DB73EB72A5FFD
:108810003F4F2DBF3EBF009709F43FC089819A8129
:108820008330910511F1843091054CF4813091052C
:10883000B1F082309105B4F4009771F02EC085300C
:108840009105C9F0853091059CF086309105B1F015
:108850008730910511F515C080E290E014C081E2E7
:1088600090E011C082E290E00EC083E290E00BC085
:1088700084E290E008C085E290E005C086E290E0E6
:1088800002C087E290E00E94D44807C0C70169E7B0
:1088900070E30E948D16009729F4C8010E940443DA
:1088A0009C0129C0C70165E870E30E948D160097FE
:1088B00081F4C8016EE57DE00E94F1429C0197FDC4
:1088C0001AC0C80169E778E045EE54E00E94A7426B
:1088D00008C00115110569F0C8016AE97DE00E9430
:1088E000F142282F392F121613062CF420E030E025
:1088F00002C02FEF3FEFC9010F900F90CF91DF9192
:108900001F910F91FF90EF9008951F93CF93DF93E6
:10891000EC01162FBA0180E090E026E631E040E05D
:1089200050E00E945353209118333091193340E0A6
:1089300050E00E94915320931633309317332FB792
:10894000F894388181E090E002C0880F991F1A9551
:10895000E2F7880F880F832B88832FBFDF91CF9199
:108960001F9108950F931F93DF93CF93CDB7DEB779
:108970002A97CDBFDEBFBE016C5F7F4F87E0FB0152
:1089800011928A95E9F78E010F5F1F4F83E0F8017E
:1089900011928A95E9F786E0888781E08E8380E0EE
:1089A00092E00E94574E80E092E065E874E40E94F5
:1089B000384F19821A828B81807F81608B8380E09F
:1089C00092E060E0A8010E94BC4E82E06FE270E09D
:1089D0000E94BE49182F00E082E06EE270E00E9423
:1089E000BE4990E0802B912B8093183390931933DC
:1089F00080E092E00E94264E9FB7F894E0E0F2E01B
:108A00008081846080839FBF2A96CDBFDEBFCF91D7
:108A1000DF911F910F9108952091163330911733F4
:108A200021513140C90108956115710529F08FB7B1
:108A3000F89480931E33089580911E338FBF08955C
:108A400000D000D0EDB7FEB73196ADB7BEB71196E6
:108A50008D939C9312978FE890E382839383648332
:108A600075830E94E4178DB79EB706968DBF9EBF93
:108A700008950F931F938C016115710579F500D04E
:108A80000F92EDB7FEB73196ADB7BEB711968C9386
:108A9000118381EA90E3828393830E94E41780919B
:108AA0001A3390911B330F900F900F900F900097F7
:108AB00009F44CC00E94B23610921A3310921B3344
:108AC00000D00F92EDB7FEB73196ADB7BEB7119695
:108AD0000C931197118383EB90E330C0CB010E947C
:108AE000E91500D000D0EDB7FEB73196ADB7BEB7EF
:108AF00011960C93118323EC30E322833383848318
:108B000095830E94E4178DB79EB706968DBF9EBFD2
:108B100080E590E00E946C3680931A3390931B336B
:108B20000097A1F000D00F92EDB7FEB73196ADB728
:108B3000BEB711960C93118383ED90E382839383E8
:108B40000E94E4170F900F900F900F901F910F91BC
:108B500008956115710549F08EE290E00E94A949DF
:108B60008EE190E00E94294908958EE290E00E94F3
:108B7000944908950E94CF480E94401E0895AF92E4
:108B8000BF92CF92DF92EF92FF920F931F93DF93EA
:108B9000CF93CDB7DEB7AB97CDBFDEBF19820E94B2
:108BA000044980E490E06AEB75E40E94A6480E94C4
:108BB000821D97FDACC180EA99E040E052EC61E093
:108BC00070E028E030E000E010E0E1E0EE2EF12C73
:108BD000CC24DD240E94974797FD99C180E090E066
:108BE00067EF77E440EA59E024E030E00E94671B39
:108BF0005C01009709F48BC10E947C1F80EA9BE016
:108C000040E052EC61E070E028E030E00E949747DD
:108C100097FD7DC180E090E066E178E44DE258E4A4
:108C200024E135E400EA1BE00E941E0A97FD6FC1B3
:108C300080EA9BE080931C3390931D330E94B244E2
:108C400089EA95E4B5010E94A10ACE0101960E942D
:108C5000800ACE0102960E94081380E295E4B501D5
:108C60000E94F70B89E395E4B5010E94CA0CC50187
:108C70006BE271E340E050E00E949017C50165E3AC
:108C800071E340E050E00E949017C50161E771E395
:108C900040E050E00E949017C5016BE771E340E0AF
:108CA00050E00E949017C50165E871E340E050E094
:108CB0000E949017C5016FE871E340E050E00E9408
:108CC0009017C50169E971E340E050E00E949017F8
:108CD000C50163EA71E340E050E00E949017C501CE
:108CE0006DEA71E340E050E00E949017C50167E033
:108CF00072E340E050E00E949017C50167EB71E31A
:108D000040E050E00E949017C50161EC71E340E043
:108D100050E00E949017C5016BEC71E340E050E019
:108D20000E949017C50165ED71E340E050E00E949C
:108D30009017C5016FED71E340E050E00E9490177D
:108D4000C50169EE71E340E050E00E949017C50153
:108D500063EF71E340E050E00E949017C5016DEFB2
:108D600071E340E050E00E949017C5016BE172E3AF
:108D700040E050E00E949017C50165E272E340E0D8
:108D800050E00E949017C5016FE272E340E050E0AE
:108D90000E949017C5016FE371E340E050E00E942C
:108DA0009017C50169E471E340E050E00E9490171C
:108DB000C50163E571E340E050E00E949017C501F2
:108DC0006DE571E340E050E00E949017C50167E651
:108DD00071E340E050E00E949017C50167E171E344
:108DE00040E050E00E949017C50161E271E340E06D
:108DF00050E00E949017C50161E172E340E050E04D
:108E00000E949017C50169E372E340E050E00E94C0
:108E10009017C50163E472E340E050E00E949017B0
:108E2000C5016DE472E340E050E00E949017C50177
:108E30006BE672E340E050E00E949017C50165E7E1
:108E400072E340E050E00E949017C50161E672E3D2
:108E500040E050E00E949017C5016DE071E340E0F2
:108E600050E00E9490178A81882399F566E172E0AC
:108E700088EA90EC0E943C146B837C838D839E83F4
:108E800060E07FEF8FEF9FEF0E943C146F83788745
:108E900089879A878E01055F1F4FC80163EE70E3D3
:108EA0000E94901683EE90E30E947E168BA7C80165
:108EB0006EEE70E340E050E00E94060CCE01039697
:108EC000BE01695F7F4F40E050E020E030E00E944B
:108ED000700C80EA99E00E945348009751F080EAB4
:108EE00099E060E070E00E94FD47682FC5010E9494
:108EF0008419898180FF06C08DE290E00E94784944
:108F0000009711F40E942B110E946B1EE2CF8FEF8D
:108F10009FEFAB96CDBFDEBFCF91DF911F910F9139
:108F2000FF90EF90DF90CF90BF90AF900895AF92F9
:108F3000BF92CF92DF92EF92FF920F931F93B82EC2
:108F4000A92EC801C114D10409F045C025503040F4
:108F50002530310528F421513D4CF901108101C023
:108F600010E08130910539F08130910538F0823080
:108F7000910589F502C0106201C01063F2E0EF169E
:108F8000F10409F418609A01AB0184E0220F331F49
:108F9000441F551F8A95D1F7213088E4380788EEA1
:108FA000480781E0580750F460E078E488EE91E0EB
:108FB0000E9491532150304088E103C02FEF3FEFD2
:108FC0008CE1EB2DFA2D148215832683378384835D
:108FD00020E030E002C026EF3FEFC9011F910F9162
:108FE000FF90EF90DF90CF90BF90AF900895FC017D
:108FF000818185FFFDCF608308950F931F93CF93E9
:10900000DF938C01EB010E94381EF801209731F4A8
:10901000818187FFFDCF208130E002C026EF3FEF46
:10902000C901DF91CF911F910F910895FC0180E05C
:1090300090E00EC0218127FFFDCF6115710511F46D
:10904000208105C02081DB01A80FB91F2C93019658
:10905000841795077CF3CA010895CF92DF92EF92AF
:10906000FF920F931F93CF93DF936C017A01062F2A
:10907000172FC0E0D0E00AC0F80161918F01772777
:1090800067FD7095C6010E94F7472196CE15DF0552
:109090009CF3C701DF91CF911F910F91FF90EF904B
:1090A000DF90CF900895FC01218130E0207830706E
:1090B000C90108958530910540F4FC01EE0FFF1FB2
:1090C000EC50FD4C2081318102C02CEF30E3C9010E
:1090D0000895EF92FF920F931F937B018C01E09113
:1090E0001F33F0912033309709F0199560912333A5
:1090F0007091243380912533909126336E0D7F1D1E
:10910000801F911F0E94F14A1F910F91FF90EF90D5
:10911000089580932133909322339C01B9018827CD
:1091200077FD8095982F28EE33E040E050E00E94D4
:1091300053530E949153209323333093243340930D
:1091400025335093263380E090E00895EF92FF920C
:109150000F931F937C0160931F33709320330E9401
:109160000F4B89E698E40E940A4BC7010E94894888
:10917000E0902333F090243300912533109126336F
:109180000E94D04A6E0D7F1D801F911F0E94F14AE0
:1091900080E090E01F910F91FF90EF9008958091F3
:1091A0002133909122330895CF93DF93EC010E94F5
:1091B0007849009721F0CE010E94A94903C0CE0151
:1091C0000E949449DF91CF9108950E949449089597
:1091D0000E94A9490895AB01282F2695269526952A
:1091E00030E0205D3F4F877061E070E002C0660FA5
:1091F000771F8A95E2F7C90125E0880F991F2A9504
:10920000E1F70E948E4A089587E0E0EAF0E0828369
:109210000E94C8490E941F4A8BE260E073E00E94EE
:10922000EB488AE260E070E00E94EB4883E090E067
:1092300060E10E94F14984E090E060E10E94F14920
:1092400086E090E060E10E94F149789480E090E04F
:109250000895282F392FC90107C0EFE3FFE13197A7
:10926000F1F700C0000001970097B9F708951F9328
:10927000182F8A3031F480EA99E06DE070E00E94A6
:10928000F747612F772767FD709580EA99E00E9484
:10929000F7471F91089587E293E30895AB01282FC4
:1092A00026952695269530E0205D3F4F877061E03A
:1092B00070E002C0660F771F8A95E2F7C90125E0CA
:1092C000880F991F2A95E1F70E948E4A089580E041
:1092D00090E0089560FF03C060E070E004C061FFAB
:1092E00004C060E071E00E944E4980E090E0089583
:1092F000E82FE695E695E695F0E0F09635E0EE0F7E
:10930000FF1F3A95E1F79085877021E030E002C0B9
:10931000220F331F8A95E2F7922321E030E011F407
:1093200020E030E0C9010895E82FE695E695E6953E
:10933000F0E0F09645E0EE0FFF1F4A95E1F78770E9
:1093400021E030E002C0220F331F8A95E2F7258327
:109350000895E82FE695E695E695F0E0F09655E05D
:10936000EE0FFF1F5A95E1F7877021E030E002C051
:10937000220F331F8A95E2F7268308954091CA0190
:10938000E62FF72F8093CA0184914093CA01089574
:109390008FEF8093700080937100809372008093B0
:1093A00073008093740080937500809376009FB75C
:1093B000F894809150008260809350009FBF80910C
:1093C000510081FFFCCF80E490E061E00E94B84B47
:1093D0009FB7F894809150008E7F809350009FBF7C
:1093E0000895FC019FB7F894E059FF4F6095808184
:1093F000862380839FBF0895FC019FB7F894E059AE
:10940000FF4F8081862B80839FBF0895AB01282F5B
:1094100026952695269530E0205D3F4F877061E0C8
:1094200070E002C0660F771F8A95E2F7C90125E058
:10943000880F991F2A95E1F70E948E4A089580E2CD
:1094400060E073E00E94064A81E260E073E00E94FF
:10945000064A82E260E073E00E94064A83E260E02E
:1094600073E00E94064A84E260E073E00E94064ACC
:1094700085E260E073E00E94064A86E260E073E005
:109480000E94064A87E260E073E00E94064A88E193
:1094900068E170E00E94064A89E168E170E00E949C
:1094A000064A8AE168E170E00E94064A8BE168E1C1
:1094B00070E00E94064A8CE168E170E00E94064A72
:1094C0008DE168E170E00E94064A88E768E170E09B
:1094D0000E94064A89E768E170E00E94064A88E037
:1094E00067E070E00E94064A8BE060E071E00E9455
:1094F000064A83E160E073E00E94064A82E160E090
:1095000070E00E94064A8BE160E073E00E94064A28
:109510008AE160E070E00E94064A08950F931F936D
:10952000CF93DF93FC01DC0180E090E0262F30E058
:10953000E901082E02C0D595C7950A94E2F7C0FF4D
:1095400003C050964C935097019611968830910520
:1095500079F750FF07C051FF02C0658301C06683E1
:10956000618301C06283DF91CF911F910F910895B4
:109570009091020481E092FD80E008951092000431
:109580002091010420FDFCCFE0E0F4E060877187CA
:109590008093DB339093DC3381E080930004089563
:1095A0004FB7F8942091DB333091DC33809108047D
:1095B00090910904009731F45091030450FF02C0C8
:1095C0002F5F3F4F4FBF40E050E0A90133272227D4
:1095D000A0E0B0E0282B392B4A2B5B2BB901CA0144
:1095E0000895E0E0F4E021E02283648775876093CA
:1095F000DF337093E0338093DD339093DE33E0E02C
:10960000F4E08091010480FDFACF82E0838385E05D
:10961000828308958093E1339093E233089580E04C
:1096200090E064E00E94F14921E0E0E4F0E023836F
:10963000E0E0F4E08FEF9FEF82879387108611863A
:109640002283208308951F920F920FB60F9208B6BF
:109650000F92112418BE8F939F938091DB339091CA
:10966000DC3301968093DB339093DC339F918F91B1
:109670000F9008BE0F900FBE0F901F9018951F926D
:109680000F920FB60F9208B60F9209B60F920BB653
:109690000F92112418BE19BE1BBEEF92FF920F93BA
:1096A0001F932F933F934F935F936F937F938F936A
:1096B0009F93AF93BF93EF93FF936091DB337091D0
:1096C000DC334091DD335091DE3364177507A8F128
:1096D00081E0E0E0F4E08283E091E133F091E23375
:1096E000309759F1009108041091090480E090E04E
:1096F000CB017727662720E030E0602B712B822B8F
:10970000932B9A0140E050E0A90133272227E090F3
:10971000DF33F090E03300E010E02E293F29402BAA
:10972000512B261737074807590730F0CA01B901EE
:109730006F5F7F4F8F4F9F4F1995FF91EF91BF91B3
:10974000AF919F918F917F916F915F914F913F91D9
:109750002F911F910F91FF90EF900F900BBE0F90E4
:1097600009BE0F9008BE0F900FBE0F901F90189566
:109770001BBEFC0128ED24BF6083089522E08030E9
:10978000920771F480912B33982F9F5F90932B3326
:109790008823B9F481E090E062E00E94F1490895E5
:1097A00022E08034920769F480912C33982F9F5FD8
:1097B00090932C33882329F482E090E062E00E94A9
:1097C000F149089522E08030920769F480912B33AB
:1097D000815080932B338823B1F481E090E062E0E4
:1097E0000E94FC49089522E08034920761F4809140
:1097F0002C33815080932C33882329F482E090E02D
:1098000062E00E94FC490895682F82E070E00E94A7
:10981000BE490895EF92FF92CF93DF938130910577
:1098200079F08130910520F082309105F9F410C073
:1098300081E20E94044C982F80E0EC0180E20FC08E
:1098400085E20E94044C982F80E0EC0184E207C07E
:109850008FE20E94044C982F80E0EC018EE20E947F
:10986000044C282F30E02C2B3D2B02C020E030E0B0
:10987000C901DF91CF91FF90EF9008951F920F9251
:109880000FB60F9208B60F9209B60F920BB60F9251
:10989000112418BE19BE1BBE2F933F934F935F93A5
:1098A0006F937F938F939F93AF93BF93EF93FF93A8
:1098B000E0E0F2E044A155A1E0912733F091283394
:1098C00080E092E061E01995FF91EF91BF91AF9137
:1098D0009F918F917F916F915F914F913F912F91C8
:1098E0000F900BBE0F9009BE0F9008BE0F900FBED9
:1098F0000F901F9018951F920F920FB60F9208B6F7
:109900000F9209B60F920BB60F92112418BE19BE12
:109910001BBE2F933F934F935F936F937F938F93D0
:109920009F93AF93BF93EF93FF93E8E2F2E04481FC
:109930005581E0912733F091283380E092E062E096
:109940001995FF91EF91BF91AF919F918F917F9169
:109950006F915F914F913F912F910F900BBE0F90A0
:1099600009BE0F9008BE0F900FBE0F901F90189564
:109970001F920F920FB60F9208B60F9209B60F9270
:109980000BB60F92112418BE19BE1BBE2F933F9326
:109990004F935F936F937F938F939F93AF93BF93F7
:1099A000EF93FF93E0E3F2E044815581E0912733A8
:1099B000F091283380E092E064E01995FF91EF91F7
:1099C000BF91AF919F918F917F916F915F914F91D7
:1099D0003F912F910F900BBE0F9009BE0F9008BEC4
:1099E0000F900FBE0F901F9018951F920F920FB6F9
:1099F0000F9208B60F9209B60F920BB60F92112470
:109A000018BE19BE1BBE2F933F934F935F936F9366
:109A10007F938F939F93AF93BF93EF93FF93E8E36D
:109A2000F2E044815581E0912733F091283380E0C2
:109A300092E068E01995FF91EF91BF91AF919F91EE
:109A40008F917F916F915F914F913F912F910F90E7
:109A50000BBE0F9009BE0F9008BE0F900FBE0F9067
:109A60001F9018951F920F920FB60F9208B60F9283
:109A700009B60F920BB60F92112418BE19BE1BBE69
:109A80002F933F934F935F936F937F938F939F9306
:109A9000AF93BF93EF93FF93E0E4F2E044A155A1AD
:109AA000E0912933F0912A3380E492E061E0199546
:109AB000FF91EF91BF91AF919F918F917F916F91A6
:109AC0005F914F913F912F910F900BBE0F9009BE68
:109AD0000F9008BE0F900FBE0F901F9018951F9209
:109AE0000F920FB60F9208B60F9209B60F920BB6EF
:109AF0000F92112418BE19BE1BBE2F933F934F9394
:109B00005F936F937F938F939F93AF93BF93EF93E5
:109B1000FF93E8E6F2E044815581E0912933F0912A
:109B20002A3380E492E062E01995FF91EF91BF91B2
:109B3000AF919F918F917F916F915F914F913F91E5
:109B40002F910F900BBE0F9009BE0F9008BE0F9083
:109B50000FBE0F901F9018951F920F920FB60F9285
:109B600008B60F9209B60F920BB60F92112418BEC9
:109B700019BE1BBE2F933F934F935F936F937F93B9
:109B80008F939F93AF93BF93EF93FF93E0E7F2E040
:109B900044815581E0912933F0912A3380E492E0A9
:109BA00064E01995FF91EF91BF91AF919F918F91D3
:109BB0007F916F915F914F913F912F910F900BBECD
:109BC0000F9009BE0F9008BE0F900FBE0F901F9010
:109BD00018951F920F920FB60F9208B60F9209B602
:109BE0000F920BB60F92112418BE19BE1BBE2F93F5
:109BF0003F934F935F936F937F938F939F93AF9315
:109C0000BF93EF93FF93E8E7F2E044815581E09141
:109C10002933F0912A3380E492E068E01995FF91AE
:109C2000EF91BF91AF919F918F917F916F915F91D4
:109C30004F913F912F910F900BBE0F9009BE0F9047
:109C400008BE0F900FBE0F901F9018951F93CF93D3
:109C5000DF93EC011FB7F8940E94BE4B88818160AE
:109C600088831FBFDF91CF911F9108951F931FB766
:109C7000F894FC0120812E7F20830E94E24B1FBFBD
:109C80001F91089522E08030920721F481E09091A5
:109C90002B3307C022E08034920739F481E09091A1
:109CA0002C33992319F480E0089580E00895DF9221
:109CB000EF92FF920F931F93CF93DF93EC018B01F1
:109CC00082E0C030D80719F480E090E006C0E2E0FE
:109CD000C034DE0721F581E090E00E940A4C7C014F
:109CE000DFB6F894CE010E94BE4B288182E08883C3
:109CF000EC86FD86F80185819681888F998F828117
:109D00008A8384818C8383818B8381818983217081
:109D10008081282B2883CE010E94E24BDFBEDF9199
:109D2000CF911F910F91FF90EF90DF900895FF92D8
:109D30000F931F93CF93DF93EC018B01FFB6F89441
:109D40000E94BE4B8881807CF8018083888D998D2C
:109D5000858396838A8182838C8184838B818383AC
:109D600089818183CE010E94E24BFFBEDF91CF91BA
:109D70001F910F91FF900895DF92EF92FF920F9342
:109D80001F93CF93DF93EC017A01862F90E08370CD
:109D90009070009721F46695669582E001C080E09E
:109DA00060FF8F5F8E01005E1F4F90E023E0880F01
:109DB000991F2A95E1F7080F191FDFB6F894CE0115
:109DC0000E94BE4BF7018081F8018083F7018281F8
:109DD000F8018283F7018181F8018183CE010E941D
:109DE000E24BDFBEDF91CF911F910F91FF90EF907B
:109DF000DF900895DF92EF92FF920F931F93CF931E
:109E0000DF93EC017A01862F90E0837090700097C9
:109E100021F46695669582E001C080E060FF8F5F67
:109E20008E01005E1F4F90E033E0880F991F3A9536
:109E3000E1F7080F191FDFB6F894CE010E94BE4B60
:109E4000F8018081F7018083F8018281F701828324
:109E5000F8018181F7018183CE010E94E24BDFBED0
:109E6000DF91CF911F910F91FF90EF90DF900895B8
:109E70002FB7F89432E08030930729F460932733AA
:109E80007093283308C032E08034930721F4609344
:109E9000293370932A332FBF08958091CF0187FD16
:109EA000FCCF08951F93CF93DF93C0ECD1E01A85C8
:109EB0008A878BEC91E061E00E94B84B1A87DF91B2
:109EC000CF911F9108958BEC91E061E00E94B84B17
:109ED0000895682F82E070E00E94BE490895CF93F4
:109EE000DF93EC0188E00E94694F888389E00E943B
:109EF000694F89838AE00E94694F8A838BE00E94C0
:109F0000694F8B838CE00E94694F8C838DE00E94A7
:109F1000694F8D8380E10E94694F8E8382E10E94A8
:109F2000694F8F8383E10E94694F888784E10E9493
:109F3000694F898785E10E94694F8A87DF91CF91B8
:109F400008950F931F93DF93CF930F920F92CDB786
:109F5000DEB789839A830E944D4F00EC11E0F8012F
:109F600012829A8191838981808386E090E00E94A9
:109F7000524FF80184810F900F90CF91DF911F9184
:109F80000F910895EF92FF920F931F93DF93CF935A
:109F900000D00F92CDB7DEB78C01CB014B835C8331
:109FA00069839A830E944D4F8CECE82E81E0F82E55
:109FB000F7012081286020830050104F89819A8109
:109FC000B8014B815C810E948757F7018081877FB0
:109FD00080832496CDBFDEBFCF91DF911F910F917B
:109FE000FF90EF9008950E944D4F8091CF0181FF27
:109FF00006C086E3E0ECF1E082870E94634F08959B
:10A00000EF92FF921F93DF93CF9300D0CDB7DEB7CF
:10A0100020ECE22E21E0F22EF701128569838A837B
:10A020009B830E94F34F0E944D4F23E3F701228749
:10A0300012829B8191838A8180836981648385E315
:10A0400082870E94634FF70112872396CDBFDEBF40
:10A05000CF91DF911F91FF90EF900895EF92FF92C3
:10A060001F93DF93CF930F920F92CDB7DEB730ECF3
:10A07000E32E31E0F32EF70112856A8389830E9473
:10A080004D4F93E3F7019287128211828981808379
:10A090006A81648312870F900F90CF91DF911F9197
:10A0A000FF90EF900895FF920F931F93CF93DF934C
:10A0B0008C01C0ECD1E0F090CA010E944D4F83E3C7
:10A0C0008A871A82198280E0E0ECF1E08093C00177
:10A0D000D8019D918D0194838F5F8032B9F7E0ECB8
:10A0E000F1E0F286DF91CF911F910F91FF900895DB
:10A0F000DF93CF930F92CDB7DEB789830E944D4F88
:10A10000898190E045E0880F991F4A95E1F7E0ECDE
:10A11000F1E012829183808385E390E00E94524FA8
:10A120000F90CF91DF910895CF92DF92EF92FF923F
:10A130000F931F93CF93DF937C016B01EA0126C03D
:10A14000C7018F7190700097B1F4C032D10598F0BB
:10A15000C6010E945350C70155E0969587955A95C0
:10A16000E1F70E94785080E290E0E80EF91EC80EF8
:10A17000D91EA0970BC087010F5F1F4FC701F601C3
:10A1800061916F010E940050219778012097C1F6DC
:10A19000DF91CF911F910F91FF90EF90DF90CF90C3
:10A1A0000895DF93CF930F92CDB7DEB789830E94D6
:10A1B0004D4F898190E065E0880F991F6A95E1F71E
:10A1C000E0ECF1E012829183808384E390E00E94CE
:10A1D000524F0F90CF91DF910895EF92FF921F930E
:10A1E000DF93CF930F92CDB7DEB770ECE72E71E01F
:10A1F000F72E1091CA0189830E94F34F0E944D4FA0
:10A2000093E3D7011A969C931A9712961C92129771
:10A2100011961C92119790E0E0ECF1E08981909307
:10A22000C00184839F5F9032D1F7E0ECF1E01287A8
:10A230000F90CF91DF911F91FF90EF900895DF93E2
:10A24000CF930F92CDB7DEB789830E944D4F89819E
:10A2500090E0E5E0880F991FEA95E1F7E0ECF1E086
:10A2600012829183808382E390E00E94524F0F908C
:10A27000CF91DF9108951F93182F8FEF0E94ED501B
:10A28000812F0E941F511F9108950E944D4F80E31E
:10A2900090E00E94524F08958FEF0E94ED500E946F
:10A2A00045510895DF92EF92FF920F931F93CF9342
:10A2B000DF937B018C01C0ECD1E0DA848AE38A87EA
:10A2C000E882BB27A12F902F8F2D8983780100274B
:10A2D0001127EA822C83BB27A52F942F832F8D83F0
:10A2E0009A01442755272E838BEC91E061E00E9470
:10A2F000B84BDA86DF91CF911F910F91FF90EF90CD
:10A30000DF900895EF92FF920F931F93DF93CF9307
:10A3100000D00F92CDB7DEB77A01890169837A83C5
:10A320008B839C830E944D4F69817A818B81382F6A
:10A330009C81292F862F972FA32FB22F0DC00BB6EC
:10A34000ABBFFC0127910BBEF70121937F01019662
:10A35000A11DB11D015010400115110581F7249672
:10A36000CDBFDEBFCF91DF911F910F91FF90EF9096
:10A370000895EF92FF920F931F93CF93DF937A018B
:10A380008901EB01D1700AC081E0BE010E94BE4983
:10A39000F70181937F0121960150104001151105AD
:10A3A00099F7DF91CF911F910F91FF90EF90089552
:10A3B0002F923F924F925F926F927F928F929F92D5
:10A3C000AF92BF92CF92DF92EF92FF920F931F93C3
:10A3D000DF93CF930F920F92CDB7DEB74A01790189
:10A3E000702E6B0166242E010894411C511C2224FE
:10A3F0002A94322C53C0A12C91E0B92E00E010E039
:10A400007720A9F081E0B8010E94BE49F201808363
:10A41000B8016F5F7F4F81E00E94BE49F2018183E6
:10A4200089819A81FFEF8F3F9F0721F405C0298220
:10A430003A8202C066246394E114F104F9F0C01674
:10A44000D10669F40894E108F1080894C11CD11CF4
:10A45000F40181914F018983E114F10479F0C8017D
:10A460000196C816D90651F40894E108F108089439
:10A47000C11CD11CF40181914F018A83B80180E095
:10A4800090E049815A810E9486070E5F1F4F089411
:10A49000A108B108A114B10409F0B2CFE114F1048C
:10A4A00009F0A9CF662041F00E944D4F60E070E0B6
:10A4B000CB0148E10E9477070E944D4F60E070E0B9
:10A4C000CB014AE10E9477070F900F90CF91DF9167
:10A4D0001F910F91FF90EF90DF90CF90BF90AF90C2
:10A4E0009F908F907F906F905F904F903F902F90B4
:10A4F00008952F923F924F925F926F927F928F9228
:10A500009F92AF92BF92CF92DF92EF92FF920F9302
:10A510001F93DF93CF93CDB7DEB72897CDBFDEBFB4
:10A520001A0149010F83412C2EEF522E2FEF622E7C
:10A530002FEF722E46225722682279225B016C018E
:10A540007DC00E944D4FD301C20180509E4FAF4F3E
:10A55000BF4F8B839C83AD83BE838301720120E058
:10A560009F81992369F00BB60BBFF70187919691F4
:10A570000BBE89839A83AFEF8F3F9A0731F406C0F1
:10A58000EFEFFFEFE983FA8301C021E0811491042A
:10A5900051F1AE14BF04C006D10679F408948108C5
:10A5A00091080894A11CB11CC11CD11CD1018D9132
:10A5B0001D01898381149104B1F0D801C70101966E
:10A5C000A11DB11DA816B906CA06DB0661F40894E0
:10A5D000810891080894A11CB11CC11CD11CF10177
:10A5E00081911F018A8349815A81C801B701288757
:10A5F0000E94860782E090E0A0E0B0E0E80EF91E3D
:10A600000A1F1B1F28858B819C81AD81BE81E816A6
:10A61000F9060A071B0709F0A3CF222331F00E9495
:10A620004D4FC301B20145E205C00E944D4FC30129
:10A63000B20144E20E947707270138018114910496
:10A6400009F07FCF2896CDBFDEBFCF91DF911F915C
:10A650000F91FF90EF90DF90CF90BF90AF909F90C1
:10A660008F907F906F905F904F903F902F900895C4
:10A670000F931F93DF93CF930F92CDB7DEB78983EC
:10A680000E944D4F00EC11E08981F801808387E042
:10A6900090E00E94524FF80184810F90CF91DF919A
:10A6A0001F910F910895629FD001739FF001829FC7
:10A6B000E00DF11D649FE00DF11D929FF00D839F51
:10A6C000F00D749FF00D659FF00D9927729FB00DEE
:10A6D000E11DF91F639FB00DE11DF91FBD01CF0101
:10A6E00011240895991B79E004C0991F961708F06A
:10A6F000961B881F7A95C9F78095089597FB092EB8
:10A7000007260AD077FD04D049D006D000201AF4DD
:10A71000709561957F4F0895F6F7909581959F4FBD
:10A720000895A1E21A2EAA1BBB1BFD010DC0AA1F92
:10A73000BB1FEE1FFF1FA217B307E407F50720F0AA
:10A74000A21BB30BE40BF50B661F771F881F991F25
:10A750001A9469F760957095809590959B01AC016E
:10A76000BD01CF01089597FB092E05260ED057FD98
:10A7700004D0D7DF0AD0001C38F4509540953095AE
:10A7800021953F4F4F4F5F4F0895F6F79095809575
:10A79000709561957F4F8F4F9F4F0895AA1BBB1BEC
:10A7A00051E107C0AA1FBB1FA617B70710F0A61BD1
:10A7B000B70B881F991F5A95A9F780959095BC01F2
:10A7C000CD010895CF93DF938230910510F482E09C
:10A7D00090E0E091E533F091E63340E050E020E096
:10A7E00030E026C06081718168177907E0F0681752
:10A7F000790781F4828193812115310531F0D901E6
:10A8000012968D939C9313972BC08093E53390936E
:10A81000E63326C04115510519F06417750718F481
:10A82000AB01E901DF019F0172816381E72FF62F00
:10A830003097C1F64115510501F1481B590B4430C1
:10A84000510580F412968D919C911397209719F0E1
:10A850008A839B8304C08093E5339093E633FD01A4
:10A86000329646C0FD01E40FF51F8193919342504B
:10A8700050404D935C9311973BC02091E33330914E
:10A88000E4332115310541F42091093130910A3129
:10A890002093E3333093E43320910B3130910C312A
:10A8A0002115310541F42DB73EB740910731509144
:10A8B0000831241B350BE091E333F091E433E217C8
:10A8C000F307A0F42E1B3F0B2817390778F0AC01D3
:10A8D0004E5F5F4F2417350748F04E0F5F1F4093C0
:10A8E000E3335093E4338193919302C0E0E0F0E0CE
:10A8F000CF01DF91CF910895CF93DF93009709F4B3
:10A9000091C0FC013297128213826091E5337091FD
:10A91000E6336115710581F420813181280F391FDB
:10A920008091E3339091E4338217930799F5E09394
:10A93000E333F093E43376C0DB0180E090E002C0C3
:10A94000CD01D901AE17BF0748F412962D913C9165
:10A95000139721153105A1F7CD0121C0A283B3833F
:10A96000EF01499159919E01240F351FA217B3079A
:10A9700079F42D913C911197240F351F2E5F3F4F95
:10A980002083318312962D913C9113972283338338
:10A99000009729F4E093E533F093E63343C0DC01FC
:10A9A0001296ED93FC9313974D915D91A40FB51FF3
:10A9B000EA17FB0769F420813181240F351F2E5FD0
:10A9C0003F4FEC0128833983228133812A833B83E3
:10A9D000E0E0F0E002C0FB01BC01DB0112968D91CA
:10A9E0009C9113970097B9F79B012E5F3F4F8D9174
:10A9F0009C911197820F931F4091E3335091E43360
:10AA00004817590779F4309729F41092E5331092DA
:10AA1000E63302C012821382225030402093E33387
:10AA20003093E433DF91CF9108958F929F92AF924C
:10AA3000BF92CF92DF92EF92FF920F931F93CF932B
:10AA4000DF938C01CB010115110529F40E94E2531B
:10AA5000082F192FB5C0D80112979801260F371F5C
:10AA60002A173B0708F4AAC0ED90FC901197E61650
:10AA7000F706D0F045E0E416F10408F4A1C0A70100
:10AA8000445050404617570708F49AC0A701425057
:10AA90005040461B570BF901419351936D937C93A2
:10AAA000CF010E947C548CC05B01AE18BF084801E6
:10AAB0008E0C9F1CE091E533F091E633CC24DD242D
:10AAC000C0E0D0E041C0E815F90599F560817181D9
:10AAD000AB014E5F5F4F4A155B0558F1AB014A1958
:10AAE0005B09CC24DD246894C1F8C40ED51E828095
:10AAF000A380E5E0CE16D10448F0F9018282A3825A
:10AB0000408351838D939C93119709C0C70102968E
:10AB1000860F971F8D939C931197E82DFA2D209700
:10AB200019F0EA83FB834CC0E093E533F093E633FE
:10AB300047C040815181C416D50608F46A01EF016F
:10AB400052814381E52FF42F309709F0BCCF40911B
:10AB5000E3335091E43348155905E9F4C816D90692
:10AB6000D0F440910B3150910C314115510541F415
:10AB70004DB75EB76091073170910831461B570B96
:10AB800024173507D8F42093E3333093E4338D93BF
:10AB90009C93119715C00E94E253C82EE6016E01E6
:10ABA000D92EE601209751F08C2DB801A7010E9403
:10ABB0008757C8010E947C54860102C000E010E063
:10ABC000C801DF91CF911F910F91FF90EF90DF901F
:10ABD000CF90BF90AF909F908F9008952F923F920B
:10ABE0004F925F927F928F929F92AF92BF92CF923D
:10ABF000DF92EF92FF920F931F93CF93DF934B015E
:10AC0000EA016115710519F0FB018083918320979A
:10AC100039F09E01225030402332310508F0F4C053
:10AC2000A82EB92EF50111915F017F01812F90E0CF
:10AC30000E9439570097B1F71D3229F4F50111919F
:10AC40007F0101E006C01B3219F4F50111917F016B
:10AC500000E0209719F0C031D105B9F4103381F428
:10AC6000F7018081883711F0883551F4F70111819F
:10AC700082E090E0E80EF91E0260C0E1D0E005C07D
:10AC8000209719F41033C1F422C0C830D105F9F06F
:10AC9000C930D10524F4C230D10509F507C0CA3046
:10ACA000D10551F0C031D105D1F427C0A12CB12C70
:10ACB000C12CF0E4DF2E26C0CAE0D0E0ECECAE2ED2
:10ACC000ECECBE2EECECCE2EECE0DE2E1BC0C8E091
:10ACD000D0E0A12CB12CC12C70E1D72E13C09E0165
:10ACE000442737FD4095542F60E070E080E090E805
:10ACF0000E94915359016A0105C0A12CB12CC12CAD
:10AD000068E0D62E40E060E070E0CB011E014424F4
:10AD100037FC4094542C50ED752E710EE72DEA301F
:10AD200070F0212F21542A3118F439EC732E06C00B
:10AD3000212F21562A3130F529EA722E710E272D46
:10AD400030E02C173D07F4F447FD18C0A616B706EF
:10AD5000C806D90680F0A20191010E945353670DE5
:10AD6000711D811D911D6130F0E07F07F0E08F07BC
:10AD7000F0E89F0710F04FEF01C041E0F70111919B
:10AD80007F01C9CF8114910491F0442339F00894D4
:10AD9000E108F108F401E082F18209C001FF1BC063
:10ADA000970122503040F4012083318314C047FFC3
:10ADB00012C000FF05C060E070E080E090E804C0D1
:10ADC0006FEF7FEF8FEF9FE722E230E02093E733D2
:10ADD0003093E83316C000FF08C0909580957095B9
:10ADE00061957F4F8F4F9F4F0CC097FF0AC082E243
:10ADF00090E08093E7339093E8336FEF7FEF8FEF2E
:10AE00009FE79B01AC0103C020E030E0A901B9013C
:10AE1000CA01DF91CF911F910F91FF90EF90DF90CA
:10AE2000CF90BF90AF909F908F907F905F904F900A
:10AE30003F902F900895FC0188279927E89421914D
:10AE40002032E9F3293010F02E30C8F32B3241F0D4
:10AE50002D3239F4689404C00E941958820F911D54
:10AE6000219120532A30C0F31EF4909581959F4F75
:10AE7000089591114FC6803219F089508550D0F74E
:10AE80000895FB01DC0102C005900D924150504035
:10AE9000D8F70895FC0105900020E9F7809590957A
:10AEA0008E0F9F1F0895EF92FF920F931F93DF93D2
:10AEB000CF930F920F92CDB7DEB7BC01DC010D909E
:10AEC0000020E9F7CD01861B970B69837A830E94E6
:10AED000E2538C0169817A81009711F00E94D0576A
:10AEE000C8010F900F90CF91DF911F910F91FF90AC
:10AEF000EF900895FB01DC0104C08D910190801951
:10AF000021F441505040C8F7881B990B0895FB016C
:10AF1000DC0102C001900D9241505040D8F70895D5
:10AF20006817790768F4FB01DC01E40FF51FA40F33
:10AF3000B51F02C002900E9241505040D8F70895BC
:10AF40000C948757DC0101C06D9341505040E0F7ED
:10AF50000895FB01DC018D9181341CF08B350CF4DC
:10AF6000805E619161341CF06B350CF4605E861B71
:10AF7000611189F3990B0895FC018191861721F0E5
:10AF80008823D9F7992708953197CF010895FB01B8
:10AF9000DC018D91019080190110D9F3990B08956E
:10AFA000FB01DC0101900D920020E1F70895FB0107
:10AFB000DC014150504030F08D910190801919F41E
:10AFC0000020B9F7881B990B0895FB01DC01415063
:10AFD000504048F001900D920020C9F701C01D9229
:10AFE00041505040E0F70895FC0181E090E001906D
:10AFF000061609F4CF010020D1F701970895FB014F
:10B0000051915523A9F0BF01DC014D914517411124
:10B01000E1F759F4CD010190002049F04D91401520
:10B020004111C9F3FB014111EFCF81E090E001979D
:10B0300008957AE0979F902D879F802D910D112480
:10B0400008950F931F93DF93CF93CDB7DEB72E975D
:10B05000CDBFDEBF0E891F89888D998D26E02C8398
:10B0600009831A8397FF02C080E090E801978D83DF
:10B070009E839E01245E3F4FCE0101966A8D7B8D9B
:10B08000A9010E94A8584D815E8157FD0AC02F81F9
:10B090003885421753070CF49A01020F131FF80169
:10B0A00010822E96CDBFDEBFCF91DF911F910F9101
:10B0B0000895DF93CF93CDB7DEB72E97CDBFDEBF18
:10B0C00085E08C838C899D8989839A839E01285E83
:10B0D0003F4FCE0101966E897F89A9010E94635C72
:10B0E0002E96CDBFDEBFCF91DF9108950F931F93B2
:10B0F000DF93CF93CDB7DEB72E97CDBFDEBF8C01E8
:10B10000CB01BA0146E04C8309831A8397FF02C042
:10B1100080E090E801978D839E83CE010196A9017E
:10B120000E94A8584D815E8157FD0AC02F81388545
:10B13000421753070CF49A01020F131FF8011082F3
:10B140002E96CDBFDEBFCF91DF911F910F91089555
:10B150002F923F924F925F926F927F928F929F9227
:10B16000AF92BF92CF92DF92EF92FF920F931F9315
:10B17000DF93CF93CDB7DEB72C97CDBFDEBF6C0189
:10B180001B018A01FC0116821782838181FFD1C1D4
:10B190002E010894411C511CF6019381F10193FD8D
:10B1A000859193FF81911F01882309F4BEC18532E7
:10B1B00039F493FD859193FF81911F01853229F424
:10B1C00090E0B6010E94F05DE7CFEE24FF2420E07E
:10B1D0002032B0F48B3269F08C3228F4803251F096
:10B1E000833271F40BC08D3239F0803349F4216021
:10B1F0002CC02260246029C0286027C0206125C09F
:10B2000027FD2CC0382F30533A3098F426FF08C061
:10B210008E2D880FE82EEE0CEE0CE80EE30E15C016
:10B220008F2D880FF82EFF0CFF0CF80EF30E206206
:10B230000CC08E3221F426FD78C1206406C08C3605
:10B2400011F4206802C0883649F4F10193FD85911C
:10B2500093FF81911F01882309F0BACF982F95544D
:10B26000933018F09052933028F40C5F1F4FFFE397
:10B27000F9830DC0833631F0833771F0833509F0DF
:10B2800060C022C0F801808189830E5F1F4F420198
:10B2900071E0A72EB12C16C062E0662E712C600EF4
:10B2A000711EF8018080918026FF03C06E2D70E032
:10B2B00002C06FEF7FEFC4012C870E94A35D5C0189
:10B2C00083012C852F7717C052E0652E712C600EFC
:10B2D000711EF8018080918026FF03C06E2D70E002
:10B2E00002C06FEF7FEFC4012C870E94985D5C0164
:10B2F0002C852068830123FD20C008C080E290E0F7
:10B30000B6012C870E94F05DFA942C858F2D90E079
:10B31000A816B90698F311C0F40127FD859127FFFF
:10B3200081914F0190E0B6012C870E94F05D2C8541
:10B33000F110FA940894A108B108A114B10461F7BE
:10B34000F1C0843611F0893649F527FF08C0F801AD
:10B3500060817181828193810C5F1F4F09C0F80168
:10B3600060817181882777FD8095982F0E5F1F4F30
:10B370004FE6B42EB22297FF09C090958095709544
:10B3800061957F4F8F4F9F4FF0E8BF2AA2012AE0BF
:10B3900030E00E94375E782E741845C0853731F44E
:10B3A0003FEEB32EB2222AE030E025C099EFB92E4D
:10B3B000B2228F36C1F0803720F4883509F0B5C04D
:10B3C0000DC0803721F0883709F0AFC002C020E1FE
:10B3D000B22AB4FE0BC084E0B82A08C0B4FE09C08B
:10B3E000E6E0BE2A06C028E030E005C020E130E0FB
:10B3F00002C020E132E0B7FE08C0F801608171812F
:10B40000828193810C5F1F4F07C0F80160817181B9
:10B4100080E090E00E5F1F4FA2010E94375E782E01
:10B420007418FFE7BF22B6FE0BC02EEFB2227E14C7
:10B4300038F4B4FE07C0B2FC05C08FEEB82202C0DB
:10B44000A72C01C0AE2C8B2D90E0B4FE0DC0FE01E8
:10B45000E70DF11D2081203319F4E9EEBE2209C069
:10B46000A394B2FE06C004C086789070009709F0DD
:10B47000A3948B2C9924B3FC14C0B0FE0FC0AF145E
:10B4800028F4E72CEF0CEA18AF2C08C0E72C06C014
:10B4900080E290E0B6010E94F05DA394AF14C0F387
:10B4A00004C0AF1410F4FA1801C0FF2484FE0FC0CA
:10B4B00080E390E0B6010E94F05D82FE1FC081FE35
:10B4C00003C088E590E010C088E790E00DC0C4019B
:10B4D00086789070009791F081FC02C080E201C0F4
:10B4E0008BE2B7FC8DE290E0B6010E94F05D06C0F1
:10B4F00080E390E0B6010E94F05DEA947E14C0F310
:10B500007A94F201E70DF11D808190E0B6010E946E
:10B51000F05D7720A9F706C080E290E0B6010E94B6
:10B52000F05DFA94FF20C1F737CEF601268137810E
:10B5300002C02FEF3FEFC9012C96CDBFDEBFCF91E8
:10B54000DF911F910F91FF90EF90DF90CF90BF9010
:10B55000AF909F908F907F906F905F904F903F90B3
:10B560002F90089520FD09C0FC0123FD05C022FF96
:10B5700002C073836283518340830895EF92FF92E8
:10B580000F931F9344FD10C046FD10C0DB01FC016A
:10B59000AA0FBB1FEE1FFF1F1094D1F76A0F7B1F6E
:10B5A0008E1F9F1F31E003C033E001C034E0660FFF
:10B5B000771F881F991F3150D1F77B018C01E20E54
:10B5C000F11C011D111DA8019701B701CA011F91AE
:10B5D0000F91FF90EF900895EF92FF920F931F93BA
:10B5E000CF93DF938C01C8010E94AE5DEC0197FD03
:10B5F00008C00E9439570097B1F7CE01B8010E94E8
:10B600001C5ECE01DF91CF911F910F91FF90EF90C3
:10B6100008958F929F92AF92BF92DF92EF92FF9226
:10B620000F931F93DF93CF930F92CDB7DEB74C01EB
:10B63000D62E5A01122F0E94AE5D8B3219F08D3238
:10B6400049F41068DA9409F46CC0C4010E94AE5D3C
:10B6500097FD67C0312F3D7F232F2073F1F4803396
:10B66000E1F4DA9409F448C0C40139830E94AE5D64
:10B67000398197FD41C03260883711F0883559F41F
:10B680003064DA94C9F1C40139830E94AE5D398116
:10B6900097FF03C031C036FF3061EE24FF248701DD
:10B6A000282F2053283090F034FD09C02A3070F044
:10B6B00036FF05C02F7D422F4151463030F0B40196
:10B6C00039830E941C5E398114C02750C801B7011C
:10B6D000432F39830E94BE5A7B018C01398132602D
:10B6E000DA9469F0C40139830E94AE5D398197FF15
:10B6F000D7CF31FD04C015C0EE24FF24870137FFEA
:10B7000008C010950095F094E094E11CF11C011D17
:10B71000111DC501B801A701232F0E94B25A81E073
:10B7200001C080E00F90CF91DF911F910F91FF90AA
:10B73000EF90DF90BF90AF909F908F9008956F92A1
:10B740007F928F929F92AF92BF92CF92DF92EF92B1
:10B75000FF920F931F93DF93CF93CDB7DEB7A197DF
:10B76000CDBFDEBF6C018A0179019E012F5F3F4F83
:10B7700080E2F90111928A95E9F7F601838080E071
:10B7800090E0BB24992470E0A1E0B0E0F70183FCD5
:10B79000A59083FEA1907F01AA2009F47FC0FA2D15
:10B7A000FE3511F4009751F1472F50E04817590723
:10B7B00044F44A2D4D3551F14D3219F4992001F1DF
:10B7C00003C0992009F4BA2C4A2D46954695469512
:10B7D000F901E40FF11D4A2D47703D0102C0660CCE
:10B7E000771C4A95E2F7908096289082AB1459F026
:10B7F000AB1410F4A394E8CFAA94E6CF71E004C090
:10B800009924939401C099240196C0CF992019F0EE
:10B810008E8180628E83772351F0CE018196FE0166
:10B820003196208120952193E817F907D1F7BB24A1
:10B83000B3944E010894811C911C01C0BB24C60125
:10B8400069A30E94AE5D69A197FD20C0282F2695AF
:10B8500026952695F401E20FF11D208130E0AC0120
:10B860004770507002C0359527954A95E2F720FD44
:10B8700004C0B6010E941C5E09C00115110519F033
:10B88000F80181938F016150C9F602C0BB2031F4E9
:10B890000115110529F0F801108202C0EE24FF24E1
:10B8A000C701A196CDBFDEBFCF91DF911F910F9150
:10B8B000FF90EF90DF90CF90BF90AF909F908F90D0
:10B8C0007F906F9008954F925F926F927F929F92B8
:10B8D000AF92BF92CF92DF92EF92FF920F931F939E
:10B8E000DF93CF930F92CDB7DEB77C016B013A01A6
:10B8F000FC011682178200E0E9C0812F90E00E94CF
:10B900003957009721F0C7010E94EC5ADFC0153269
:10B9100041F4F601A3FC3591A3FE31916F0135325C
:10B9200061F4C7010E94AE5D97FDDCC0181709F4F1
:10B93000CDC0B7010E941C5ED7C03A3239F4A3FCD7
:10B940003591A3FE31916F0111E001C010E09924FF
:10B950000FC01260692D70E080E090E040E20E942C
:10B96000BE5A962EF601A3FC3591A3FE31916F01CC
:10B97000232F20532A3068F311FF03C0992019F4B4
:10B98000B3C099249A94383619F03C3689F409C02A
:10B99000F601A3FC3591A3FE31916F01383641F4D5
:10B9A00018601460F601A3FC3591A3FE31916F017C
:10B9B000332309F499C084E99EE0632F70E0398352
:10B9C0000E948D5D3981009709F48EC0812F10FD92
:10B9D00008C0F3014080518042E050E0640E751EC3
:10B9E00002C0442455243E3651F4F7014681578164
:10B9F00060E070E0C201212F0E94B25A67C0333666
:10BA000091F481FD02C099249394C7010E94AE5D18
:10BA100097FD68C04114510419F0F20181932F0180
:10BA20009A9499F751C03B3559F4C701692DA20189
:10BA300096010E949F5B6C01009709F045C03FC0D2
:10BA4000C70139830E94EC5A398197FD4BC03F36BC
:10BA500059F1303728F4343629F1393639F527C011
:10BA6000333719F0353711F51DC0C7010E94AE5D9F
:10BA70005C0197FD11C00E943957009729F0C5015C
:10BA8000B7010E941C5E08C04114510419F0F20174
:10BA9000A1922F019A9449F741145104A9F0F2019F
:10BAA000108212C0106203C0106101C01064C7018F
:10BAB000692DA201212F0E94095B882329F4F70137
:10BAC0008381807379F410C010FF0F5FF701A380AA
:10BAD000F601A3FC1591A3FE11916F01112309F04A
:10BAE0000CCF02C0002311F010E002C00FEF1FEFD7
:10BAF000C8010F90CF91DF911F910F91FF90EF90B0
:10BB0000DF90CF90BF90AF909F907F906F905F90AD
:10BB10004F900895992788270895FC0105900616EF
:10BB200021F00020D9F7C00108953197CF01089581
:10BB3000FC010590615070400110D8F780959095F8
:10BB40008E0F9F1F0895FC016150704001900110FD
:10BB5000D8F7809590958E0F9F1F0895CF93DF9310
:10BB6000EC013B8130FF36C036FF09C03F7B3B8391
:10BB70008E819F8101968E839F832A8129C032FF07
:10BB80000FC0E881F9818081992787FD9095009702
:10BB900019F430623B831EC03196E883F98311C0EB
:10BBA000EA85FB85CE01199597FF0BC02B813FEFEE
:10BBB0008F3F930711F480E101C080E2822B8B83D9
:10BBC00009C02E813F812F5F3F4F2E833F83282F57
:10BBD00030E002C02FEF3FEFC901DF91CF91089510
:10BBE0000F931F93CF93DF938C01EB018B8181FF28
:10BBF0001BC082FF0DC02E813F818C819D81281743
:10BC0000390764F4E881F9810193E883F98306C078
:10BC1000E885F985802F1995009731F48E819F81F1
:10BC200001968E839F8302C00FEF1FEFC801DF9143
:10BC3000CF911F910F910895FB01238120FF13C025
:10BC400026FD11C03FEF8F3F930769F08283206488
:10BC50002F7D2383268137812150304026833783EF
:10BC6000282F30E002C02FEF3FEFC9010895FA01FD
:10BC7000AA27283051F1203181F1E8946F936E7F2B
:10BC80006E5F7F4F8F4F9F4FAF4FB1E03ED0B4E01C
:10BC90003CD0670F781F891F9A1FA11D680F791F5D
:10BCA0008A1F911DA11D6A0F711D811D911DA11D6E
:10BCB00020D009F468943F912AE0269F112430197E
:10BCC000305D3193DEF6CF010895462F4770405D19
:10BCD0004193B3E00FD0C9F7F6CF462F4F70405DC8
:10BCE0004A3318F0495D31FD4052419302D0A9F723
:10BCF000EACFB4E0A6959795879577956795BA951D
:10BD0000C9F700976105710508959B01AC010A2EE2
:10BD100006945795479537952795BA95C9F7620FB9
:0EBD2000731F841F951FA01D0895F894FFCF78
:10BD2E00200000252D3230732025730A0D00257357
:10BD3E00202D2068657864756D70286C656E3D25C4
:10BD4E0064293A0A0D00253034782020002530323F
:10BD5E00782000202020003A200020202025730A81
:10BD6E000D00082008000A0D00636F6D6D616E6492
:10BD7E00206E6F7420666F756E643A25730A0D001F
:10BD8E0025732000256300240068656C70007072B6
:10BD9E00696E74207468697320696E666F726D6166
:10BDAE0074696F6E002573202D2068657864756D3B
:10BDBE0070286C656E3D2564293A0A0D00253034D5
:10BDCE0078202000253032782000202020003A20D4
:10BDDE000020202025730A0D00737563636573734D
:10BDEE0000756E6B6E6F776E00616C726561647953
:10BDFE0020696E207573650061626F7274656400F0
:10BE0E0073796E63206572726F720063616E636523
:10BE1E006C65642062792072656D6F746500696768
:10BE2E006E6F7265640074696D656F757400707203
:10BE3E006F746F636F6C206572726F7200646973DA
:10BE4E0061626C65640062757379007265747279F3
:10BE5E00206C61746572006261642073697A65009A
:10BE6E006F7574206F662072616E6765006F706506
:10BE7E00726174696F6E206E6F7420737570706F5F
:10BE8E0072746564006E6F207065726D697373698C
:10BE9E006F6E00696E636F6D70617469626C6520A0
:10BEAE00747970650070617468206E6F7420666FAF
:10BEBE00756E640070617273696E67206572726F61
:10BECE007200696E76616C696420737461746500CA
:10BEDE006E6F7420636F6E6E6563746564006F754C
:10BEEE0074206F66206D656D6F72792F6275666650
:10BEFE0065727300696E76616C696420706172613F
:10BF0E006D657465727300756E6B6E6F776E2066FD
:10BF1E0061696C7572650073772076657273696FEF
:10BF2E006E3A25642E25642E25640A0D00636F6E0D
:10BF3E006E5F636220736F636B69643A256420637E
:10BF4E006F6E6E65637465643A25640A0D006F6BDF
:10BF5E000065727200257320256420282573290A36
:10BF6E000D0075736167653A207363616E205B73B4
:10BF7E007369645D0D00494E465241004144484F7D
:10BF8E0043006E6F206E65747320666F756E640A63
:10BF9E000D006661696C656420746F20676574209E
:10BFAE006E6574776F726B206C6973740A0D004244
:10BFBE0053534944202020202020202020202020C0
:10BFCE002020545950452020204348205253534995
:10BFDE0020534E522020415554482020202020200E
:10BFEE00535349440A0D002D2D2D2D2D2D2D2D2D64
:10BFFE002D2D2D2D2D2D2D2D2D2D2D2D2D2D2D2D63
:10C00E002D2D2D2D2D2D2D2D2D2D2D2D2D2D2D2D52
:10C01E002D2D2D2D2D2D2D2D2D2D2D2D2D2D2D2D42
:10C02E002D2D2D2D2D2D2D2D2D2D2D2D0A0D0025AA
:10C03E003032783A253032783A253032783A253017
:10C04E0032783A253032783A253032782020002561
:10C05E0073202025303264202530326420200025C4
:10C06E00303264202020004E2F412020004E4F4EB3
:10C07E004520202020202000574550202020202021
:10C08E002020005750412D50534B20202000575058
:10C09E0041322D50534B202000575041202020205C
:10C0AE002020200057504132202020202020002523
:10C0BE0073000A0D0075736167653A207365745FCE
:10C0CE00706F6C6C5F706572696F64203C70657226
:10C0DE00696F6420696E206D733E0A0D0070657283
:10C0EE00696F642025640A0D0075736167653A20D7
:10C0FE007365745F686561727462656174203C304B
:10C10E007C313E0A0D0075736167653A2073657464
:10C11E005F6C6564203C307C313E0A0D00636170BB
:10C12E00733A3078253032780A0D00756E6B6E6F6B
:10C13E00776E0066772076657273696F6E3A256446
:10C14E002E25642E2564206275696C643A25730A67
:10C15E000D006877207265766973696F6E3A257384
:10C16E000A0D0000687474705F706F7374004C6910
:10C17E007374656E696E67206F6E2025733A256441
:10C18E002F25730A0D0075736167653A2066775F18
:10C19E0075706772616465203C6D6574686F642CA0
:10C1AE0020652E672E2022687474705F706F737412
:10C1BE00223E205B3C69703E203C706F72743E20C4
:10C1CE003C706174683E5D0A0D006C6F6F6B75702C
:10C1DE005F63623A20686F7374206E6F7420666FAF
:10C1EE00756E640A0D006C6F6F6B75705F63622005
:10C1FE0069703A25730A0D002573202564202800E6
:10C20E0069703A257320006D61736B3A25732000B7
:10C21E0067773A25732000646E733A2573290A0DE9
:10C22E000075736167653A206765745F686F737434
:10C23E0062796E616D65203C646E736E616D653EF4
:10C24E000A0D0025732025642028257329200070EF
:10C25E006565723A25730A0D0075736167653A203C
:10C26E006765745F7065657261646472203C736F9C
:10C27E00636B69643E0A0D0073656E64696E6720B8
:10C28E00256420627974657320746F2025733A25B6
:10C29E00640A0D0077726F74653A25642072656DBD
:10C2AE0061696E3A25640A0D0075736167653A20FF
:10C2BE0073656E64746F203C736F636B69643E20AC
:10C2CE003C69703E203C706F72743E203C64617419
:10C2DE0061202E2E2E3E0A0D0073656E64696E6708
:10C2EE002025642062797465730A0D007573616789
:10C2FE00653A2073656E64203C736F636B69643EB0
:10C30E00203C64617461202E2E2E3E0A0D00757342
:10C31E006167653A20636C6F7365203C736F636B66
:10C32E0069643E0A0D0075736167653A20636F6E2E
:10C33E006E656374203C736F636B69643E203C6969
:10C34E00703E203C706F72743E0A0D00757361670B
:10C35E00653A206C697374656E203C736F636B690C
:10C36E00643E205B6261636B6C6F675D0A0D006CEF
:10C37E00697374656E5F636220736F636B69643A91
:10C38E0025642C20616363657074696E67202E2EA0
:10C39E002E200028636F6E6E656374696F6E206C5D
:10C3AE006F73742900726563765F636220736F63C7
:10C3BE006B69643A2564206C656E3A25642025739A
:10C3CE000A0D0052580075736167653A2062696EF6
:10C3DE0064203C736F636B69643E203C69703E2041
:10C3EE003C706F72743E0A0D0073747265616D005D
:10C3FE00646772616D007261770075736167653A8B
:10C40E0020736F636B6574203C73747265616D7C11
:10C41E00646772616D7C7261773E205B70726F74BF
:10C42E006F636F6C5D0A0D0075736167653A2073FB
:10C43E0065745F6468637064203C307C313E0A0D25
:10C44E000025732025642028656E61626C65643A50
:10C45E002564290A0D0075736167653A207365744A
:10C46E005F64686370203C307C313E0A0D0075734A
:10C47E006167653A207365745F69706164647220E8
:10C48E003C69703E205B6D61736B5D205B67775D11
:10C49E00205B646E735D0A0D004E2F4100257320E4
:10C4AE002564200028257320253032783A25303235
:10C4BE00783A253032783A253032783A253032784B
:10C4CE003A253032782000727373693A2564200061
:10C4DE00727373693A4E2F412000736E723A25645F
:10C4EE0000736E723A4E2F4100290A0D00257320FB
:10C4FE0025642028253032783A253032783A253096
:10C50E0032783A253032783A253032783A25303240
:10C51E0078290A0D0075736167653A207365745F3B
:10C52E006368616E6E656C203C6368616E6E656CEF
:10C53E003E0A0D0058202564202564202564202500
:10C54E00642025640075736167653A20636F6E66BB
:10C55E005F7073203C7573655F70735F706F6C6C8A
:10C56E003E203C70735F747261666669635F7469C6
:10C57E006D656F75743E0A0D00202020202020204E
:10C58E0020202020202020203C70735F64656C6189
:10C59E00793E203C72785F616C6C5F6474696D3EAD
:10C5AE00203C6C697374656E5F696E74657276613A
:10C5BE006C3E0A0D0075736167653A207365745F92
:10C5CE007073203C307C313E0A0D00737461006143
:10C5DE0070006164686F63007770730075736167D4
:10C5EE00653A207365745F6D6F6465203C7374618A
:10C5FE007C61707C6164686F633E0A0D00777061C8
:10C60E003200777061007765700075736167653A07
:10C61E00206C696E6B7570205B737369645D205B53
:10C62E006B65795D205B7765707C7770617C777068
:10C63E0061325D0A0D0075736167653A207365742A
:10C64E005F6261756472617465203C6261756472CB
:10C65E006174653E205B7274736374735D0A0D00C2
:10C66E0065727220256420286661696C6564207489
:10C67E006F20636F6E66696775726520686F73747D
:10C68E002075617274290A0D0072657365740077E6
:10C69E006C705F72657365742829007365745F62D0
:10C6AE006175647261746500776C705F7365745F39
:10C6BE0062617564726174652829006C696E6B75B0
:10C6CE007000776C705F6C696E6B75702873736930
:10C6DE00642C206B65792C206175746829006C6957
:10C6EE006E6B646F776E00776C705F6C696E6B64E7
:10C6FE006F776E2829007365745F6D6F64650077C0
:10C70E006C705F7365745F6D6F6465282900676573
:10C71E00745F6D6F646500776C705F6765745F6DD5
:10C72E006F64652829007365745F707300776C7091
:10C73E005F7365745F7073282900636F6E665F7038
:10C74E007300776C705F636F6E665F70732829007D
:10C75E007365745F6368616E6E656C00776C705F95
:10C76E007365745F6368616E6E656C28290067651A
:10C77E00745F68776164647200776C705F6765746C
:10C78E005F6877616464722829006765745F6E65FF
:10C79E0074776F726B00776C705F6765745F6E6530
:10C7AE0074776F726B2829007365745F69706164AA
:10C7BE00647200776C705F7365745F697061646436
:10C7CE00722869702C206D61736B2C2067772C207A
:10C7DE00646E7329006765745F69706164647200CA
:10C7EE00776C705F6765745F697061646472282925
:10C7FE00007365745F6468637000776C705F736557
:10C80E00745F6468637028656E61626C6529006789
:10C81E0065745F6468637000776C705F6765745FE2
:10C82E00646863702829007365745F64686370645C
:10C83E0000776C705F7365745F6468637064282939
:10C84E0000736F636B657400776C705F736F636BEF
:10C85E00657428747970652C2070726F746F29005E
:10C86E0062696E6400776C705F62696E6428736FC4
:10C87E00636B2C2069702C20706F727429006C69A8
:10C88E007374656E00776C705F6C697374656E2877
:10C89E00736F636B69642C206261636B6C6F6729C5
:10C8AE0000636F6E6E65637400776C705F636F6E9E
:10C8BE006E65637428736F636B69642C2069702CCA
:10C8CE0020706F72742900636C6F736500776C70E3
:10C8DE005F636C6F736528736F636B696429007394
:10C8EE00656E6400776C705F73656E6428736F633A
:10C8FE006B69642C2064617461290073656E6474C5
:10C90E006F00776C705F73656E64746F28736F63FE
:10C91E006B69642C20646174612C2069702C20700A
:10C92E006F727429006765745F7065657261646407
:10C93E007200776C705F6765745F706565726164B5
:10C94E00647228736F636B696429006765745F682E
:10C95E006F737462796E616D6500776C705F676579
:10C96E00745F686F737462796E616D6528646E733F
:10C97E006E616D65290066775F75706772616465BB
:10C98E0000776C705F66775F75706772616465289B
:10C99E006D6574686F642C20616464722C20706FF6
:10C9AE0072742C207061746829006765745F7665F7
:10C9BE007273696F6E007072696E7420636C696554
:10C9CE006E742076657273696F6E006765745F664C
:10C9DE00775F76657273696F6E007072696E742020
:10C9EE006669726D776172652076657273696F6EB6
:10C9FE00006765745F66775F63617073007072695C
:10CA0E006E74206669726D77617265206361706104
:10CA1E0062696C6974696573007365745F6C6564D3
:10CA2E0000776C705F7365745F6C656428290073A2
:10CA3E0065745F68656172746265617400776C70AD
:10CA4E005F7365745F6865617274626561742829CD
:10CA5E00007365745F706F6C6C5F706572696F6484
:10CA6E0000776C705F7365745F706F6C6C5F706570
:10CA7E0072696F642829007363616E00776C705F52
:10CA8E007363616E287373696429000D0A0047454C
:10CA9E005420002D2D2D2025732070696E67207374
:10CAAE00746174697374696373202D2D2D0A0D00E2
:10CABE002564207061636B657473207472616E738C
:10CACE006D69747465642C202564207265636569D4
:10CADE007665640A0D00256420627974657320669C
:10CAEE00726F6D2025733A2069636D705F73657187
:10CAFE003D25640A0D0025642062797465732066F5
:10CB0E00726F6D2025733A2069636D705F73657166
:10CB1E003D25642044657374696E6174696F6E207F
:10CB2E00486F737420556E726561636861626C65DF
:10CB3E000A0D0025642062797465732066726F6D2C
:10CB4E002025733A2069636D705F7365713D2564AE
:10CB5E0020547970653A25640A0D006F6B0065727A
:10CB6E0072002D63002D7300257320256420282567
:10CB7E0073290A0D0075736167653A2070696E67D7
:10CB8E00205B2D63203C636F756E743E5D205B2DC4
:10CB9E0073203C73697A653E5D203C69703E0A0DD8
:10CBAE000070696E67000A0D007474637020657200
:10CBBE00723A256420282573290A0D007474637057
:10CBCE00206F6B3A20256420627974657320707231
:10CBDE006F63657373656420696E20256C75206DB7
:10CBEE00732C20256C75204B422F730A0D00747424
:10CBFE006370206F6B3A2025642062797465732010
:10CC0E0070726F63657373656420696E2030206D7A
:10CC1E00730A0D002E002D70002D6E002D6C002D50
:10CC2E0074002D7200257320256420282573290A8F
:10CC3E000D00657272007474637020636F6E6E65A2
:10CC4E0063742025733A2564206E6275663A2564F6
:10CC5E00206275666C656E3A256420736F636B692E
:10CC6E00643A25640A0D0074746370206C697374E1
:10CC7E00656E20706F72743A2564206275666C65FD
:10CC8E006E3A2564206C736F636B69643A25640A8F
:10CC9E000D0075736167653A2074746370205B2DA7
:10CCAE007472706E6C5D0A0D00747463700074742F
:10CCBE006370207468726F75676870757420746520
:10CCCE007374006661696C656420746F20676574A7
:10CCDE00206E74702074696D653A25732825642959
:10CCEE000A0D006E74702074696D653A202530341B
:10CCFE00642D253032642D25303264202530326487
:10CD0E003A253032643A253032640A0D006F6B00DA
:10CD1E0065727200257320256420282573290A0D5B
:10CD2E000075736167653A206E7470203C6E747086
:10CD3E002D7365727665723E0A0D006E7470006713
:10CD4E006574207365727665722074696D652066F0
:10CD5E00726F6D206E7470004E2F41002530327848
:10CD6E003A253032783A253032783A253032783AD0
:10CD7E00253032783A25303278002F002F3F002FA1
:10CD8E00696E6465782E68746D6C3F00746F6767AA
:10CD9E006C653D4C45442564002F696E6465782EA4
:10CDAE0068746D6C002F6C6F676F2E676966006C10
:10CDBE00696E6B5F6362206C696E6B3A25640A0D57
:10CDCE0000616464725F63622069703A6E6F6E65B3
:10CDDE000A0D0068747470642073746F70706564EB
:10CDEE000A0D00616464725F63622069703A257394
:10CDFE000A0D0068747470642073746172746564D3
:10CE0E000A0D006864776972656C657373006864F7
:10CE1E00776972656C65737331323300004E00456D
:10CE2E00004F004D0053002000E933000069202F11
:10CE3E00186E2000000000692969356F2900000076
:10CE4E00007B2998348829000000009B29C333A257
:10CE5E002900000000BE298733C72900000000D634
:10CE6E00290733DF2900000000EE29BE32F7290022
:10CE7E00000000062A52320D2A000000001A2A6213
:10CE8E0031222A00000000302AF7303C2A00000030
:10CE9E00004E2AAA30592A000000006A2A7B2F76FB
:10CEAE002A00000000882ABB2E932A00000000B53D
:10CEBE002A7926C02A00000000D12A4F2EDA2A0035
:10CECE00000000EF2A112EF82A00000000072BA503
:10CEDE002D112B00000000212BF42C282B0000001C
:10CEEE0000402B662C452B000000005E2B0F2B659F
:10CEFE002B00000000812B812A892B00000000A747
:10CF0E002B152AAD2B00000000BF2B3229C42B009D
:10CF1E00000000DB2B1C28E22B00000000052C8EED
:10CF2E0027122C000000002B2C32273A2C00000078
:10CF3E0000562C5A25612C000000008A2CB21F9638
:10CF4E002C00000000AB2CB924BA2C00000000D13C
:10CF5E002C5924DD2C00000000F92CED23012D00AE
:10CF6E000000000F2D5C231D2D00000000312D94BC
:10CF7E0022412D00000000572D0F205C2D000000D7
:10CF8E0000812E1D39812E00000000892FF03C8E6D
:10CF9E002F000000001B30903F1F300000000000EB
:10CFAE00000000FFFFFFFFC920D820E020EB20FE8D
:10CFBE002006210E211D2126212B21372140214D16
:10CFCE00216521732185219421A221B021BE21D476
:10CFDE0021E721AB28AF28B228B82800001F003B5C
:10CFEE00005A0078009700B500D400F3001101300C
:10CFFE00014E016D0100001F003C005B007900989E
:10D00E0000B600D500F400120131014F016E01008F
:0ED01E0001020307FD30FF30013103310531FF
:00000001FF
